:020000040040BA
:1000000038110020D9064000D5064000D506400032
:10001000D5064000D5064000D5064000000000008F
:10002000000000000000000000000000D5064000B5
:10003000D506400000000000D5064000F511400044
:10004000D5064000D5064000D5064000D506400044
:10005000D5064000D5064000D5064000D506400034
:10006000D5064000D506400000000000D50640003F
:10007000D5064000D5064000D5064000D506400014
:10008000D5064000D5064000D5064000D506400004
:10009000891A4000D5064000D5064000D50640002C
:1000A000D5064000D5064000D5064000D5064000E4
:1000B000D5064000D506400000000000000000000A
:1000C0000000000000000000000000000000000030
:1000D0000000000000000000000000000000000020
:1000E0000000000000000000000000000000000010
:1000F000000000000000000000000000D5064000E5
:10010000E5114000D506400000000000000000009E
:1001100000000000000000000000000000000000DF
:1001200000000000000000000000000000000000CF
:1001300000000000000000000000000000000000BF
:1001400000000000000000000000000000000000AF
:10040000803E000010B5054C237833B9044B13B17E
:100410000448AFF300800123237010BD00040020C6
:1004200000000000783C40000C4B43B10C480D49E3
:1004300010B5AFF300800C48036823B910BD0A481B
:10044000036833B97047094B002BF7D0BDE8104063
:100450001847064B002BF5D0184700BF00000000DE
:10046000783C400004040020783C4000000000007C
:10047000144B98420FD9144B984211D9134B984200
:1004800012D9134B984213D9124B984214D9124ADD
:10049000124B1A6070474FF08062104B1A60704721
:1004A0000F4A0E4B1A6070470E4A0C4B1A60704789
:1004B0000D4A0A4B1A6070474FF00422074B1A602E
:1004C000704700BF7F9FD500FF3EAB017FDE8002FB
:1004D000FF7D56037F1D2C0400050004000A0E401A
:1004E00000010004000200040003000410B5A0B0E5
:1004F000334A344B1A60344A936843F0254343F43B
:1005000080139360536913F0800F0CD12F4A2E4B48
:100510001A602D4B5B6913F0800FFAD02C4B9B6E49
:1005200013F0800FF5D00023012262F3070343F498
:100530007C53274A936240F6B73161F31C439362C0
:10054000234B9B6E13F0020FFAD00023012262F3BB
:10055000070343F47C531E4AD3624FF4B76161F33F
:100560001A43D3621A4B9B6E13F0040FFAD0022287
:10057000174B1A63164B9B6E13F0080FFAD0154CED
:1005800015482060154B98472268154B1344154AAF
:10059000934201D920B010BD20216846124B9847E4
:1005A0000949CB6923F4F053109A520202F4F05235
:1005B000134343F0B44343F48073CB61EAE700BFD5
:1005C00000050004000A0E4010140E40080000A5AB
:1005D00000040E40B80900200000DC057104400052
:1005E000C0D3BDF980C3C9010D00002010B50C4B6C
:1005F0009847044601220B4B9A600A4B1B6913F083
:10060000010F0AD0064B984704F114039842F4D91D
:100610000122044BDA60002010BD012010BD00BF94
:10062000D91540000080044010B400240EE04000C2
:1006300080F00700C0B20133DBB2072B05D810F001
:10064000800FF4D14000C0B2F5E70134944204D2E7
:1006500011F8013B58400023EFE710BC7047000041
:1006600070B506460D464FF40032164BC3F8002114
:100670000122154B5A63154B00241C605C609C6082
:10068000DC601C610AE0114A53602C460E4B0F4A95
:100690001A6001229A630E4B984788B1AC420CD283
:1006A000A3190A4A13602B1B4FF6F8729342EAD93A
:1006B0001346064A53601C44E8E7034BD86B70BDF1
:1006C000002070BD00040E4000800440000A00209D
:1006D000ED054000FEE7000008B5104B104A9A42B5
:1006E00009D00E4B0E4A03E011681960043304323E
:1006F0000C498B42F8D30C4B02E000221A60043301
:100700000A4A9342F9D30A4A0A4B23F07F039360C3
:10071000094B9847094B9847FEE700BF0C000020A3
:10072000783C40000402002000040020340B00202C
:1007300000ED00E0000040001D3B40007519400046
:10074000014A024B1A60704700127A0090010020A3
:10075000A0F58000012915D0430A19B1022918D04B
:1007600002207047430B1B0323F07F430E481843BE
:1007700010B5EFF3108404B972B60C4B984794B9D6
:1007800062B610BD830B5B0323F07F430848184318
:10079000EEE7180220F07F4020F0FF0040F0B44068
:1007A00040F01100E4E710BD0702005A710000207C
:1007B0000703005A38B502210A480B4B98470546F3
:1007C00068B90124032C0AD804F120000221400456
:1007D000054B984710B90134E4B2F3E705462846C3
:1007E00038BD00BF00404000510740002DE9F041F6
:1007F00006460C461546EFF3108707B972B6A6F504
:100800008000400A1FFA80FE0EF5005E4FEA4E2E71
:10081000A6EB0E0806EB040CAEEB0C0101F5007123
:10082000002305E04FF0FF324EF8232001339BB246
:10083000B3EB980FF6D3B646002305E055F8232016
:100840004EF8232001339BB2B3EB940FF6D3E64668
:10085000002305E04FF0FF324EF8232001339BB216
:10086000B3EB910FF6D3000220F07F4020F0FF00A1
:1008700040F0B44040F001000E4B9847864670B1FE
:10088000AFB962B613E004339BB29C420AD99A080E
:1008900055F82210F2589142F5D00130F3E70020CC
:1008A0000346F2E707B962B608B14FF0030E70468F
:1008B000BDE8F0817100002010B5EFF3108404B999
:1008C00072B60348034B984704B962B610BD00BF27
:1008D0001300005A7100002010B5EFF3108404B922
:1008E00072B6002307E09A0002F5800250F8231048
:1008F000116001339BB27F2BF5D90348034B984716
:1009000004B962B610BD00BF1200005A7100002089
:1009100038B50246EFF3108404B972B68023034958
:100920000348044DA84704B962B638BD1500005A03
:100930001400005AFD000020154B98421BD003F50F
:10094000A033984219D003F58043984217D0A3F5FD
:100950004043984215D003F58043984213D0A3F545
:10096000A033984211D003F56033984201D0322071
:1009700070471620704708207047092070470E20E6
:10098000704713207047142070471520704700BF30
:1009900000C0004031281BD81F280BD80D4B9A6986
:1009A00001238340934313D0012303FA00F0094B42
:1009B000186170472038074BD3F808210123834082
:1009C000934305D0012303FA00F0024BC3F8000162
:1009D000704700BF00040E404900B0FBF1F003383F
:1009E000002302E040080133DBB2FF28FAD80202FC
:1009F00002F47F4252FA80F01B0403F4E02318440F
:100A000070470368027AD2B2012A21D010B403F5EC
:100A1000C063012202720022C271C1604A78012AB9
:100A200012D00A78120402F4FE025A608C68C2796D
:100A3000D2B2511CC9B2C171A25C5A634FF4417267
:100A40005A62012010BC70470A7852081204ECE781
:100A5000002070470268037ADBB2012B27D010B464
:100A600002F5C064012303720023C371C1604B7897
:100A7000012B12D00B781B0403F4FE0303F5805303
:100A800063600B79012B0ED00123C2F8003640F2CF
:100A900002336362012010BC70470B785B081B04B3
:100AA00003F58053ECE70323C2F80036EFE700209C
:100AB0007047036803F5C063027AD2B2012A17D0E7
:100AC000012202720022C271C1604A78012A0BD051
:100AD0000A78120402F4FE025A60CA785A634FF48C
:100AE00041725A62012070470A7852081204F3E7F3
:100AF00000207047036803F5C063027AD2B2012A6E
:100B000017D0012202720022C271C1604A78012A04
:100B10000BD00A78120402F4FE025A60CA785A63B3
:100B20004FF441725A62012070470A785208120449
:100B3000F3E70020704782B00023ADF8063006E0EE
:100B4000BDF806309BB201339BB2ADF80630BDF85C
:100B500006309BB2B3F52F7FF2D302B0704700008E
:100B60002DE9F0410646884604682046194B98470F
:100B7000312801D9BDE8F0810546174B984703237A
:100B800023602423C4F8003641461448144B984788
:100B9000C4F81006002333720123B3716BB2002B2B
:100BA00007DB5A0905F01F00012181400D4840F87C
:100BB0002210002B08DB03F1604303F56143202280
:100BC00083F80023BDE8F08105F00F05064B2022D5
:100BD0005A55CFE739094000950940000000DC056F
:100BE000D909400000E100E014ED00E008B5837988
:100BF00093B18B78032B11D8DFE803F00205080BC3
:100C0000074B984708BD074B984708BD064B9847C8
:100C100008BD064B984708BD002008BD002008BD50
:100C2000030A4000550A4000B30A4000F50A40009C
:100C3000007A7047F8B50646036803F5C064256A74
:100C4000C76815F0040F0BD0E26A12F0040F07D04A
:100C5000BA78002A4DD0022A4BD0BA78032A5ED047
:100C600015F0020F08D0E26A12F0020F04D0BA7831
:100C7000012A73D0032A71D015F4807F0DD0E36A66
:100C800013F4807F09D040F20733A362002333724C
:100C90000323B371FB6803B1984715F4007F0DD0AF
:100CA000E36A13F4007F09D040F20733A362002304
:100CB00033720423B371FB6803B1984715F0010F39
:100CC00016D0E36A13F0010F12D0BB780BB1022BE0
:100CD00009D140F20533A362002333720223B371BA
:100CE000FB6803B19847BB78012B54D0032B52D03B
:100CF000F8BDF279D2B239798A4208D2B868F2796D
:100D0000D2B2511CC9B2F171825C6263A5E70222C2
:100D1000C3F80026012262620422A2629DE77A786B
:100D2000012A11D03A78120402F4FE0202F5805230
:100D300062603A79012A0DD00122C3F8002604220C
:100D4000A262022262628BE73A785208120402F52C
:100D50008052EDE70322C3F80026F0E7B868F27985
:100D6000D2B2511CC9B2F171216B8154F179C9B26F
:100D70003A79013A91420AD0F379DBB23A79934257
:100D80007FF47AAF012363620223A36274E7022235
:100D9000C3F80026F0E740F20333A3620023337266
:100DA0000223B371FB68002BA2D09847A0E7000094
:100DB000F8B50379202B0BD9A3F12006F3B20B4F22
:100DC00001269E403E603E653E613E63002408E091
:100DD000074FF5E7074DA8477E63A8473E630134F8
:100DE000E4B2092CF6D97E617E60F8BD00100E4099
:100DF000000E0E40370B4000014B1868704700BFD3
:100E00000044400008B5024B9847024B185808BDF3
:100E1000F90D40000040400008B5044B98470146DA
:100E20000348044B9847C04308BD00BFF90D40007C
:100E30000040400061064000F8B5036841681B4A65
:100E40009A4227D81A4D1B4A9A4225D91A4B8B42EF
:100E500024D88D4224D90446184B984700270619F8
:100E600047F10007012F08BF002E1BD2B0F5847F89
:100E70001AD30023BB4208BFB54201D20020F8BDFF
:100E80000F4B984704460F4B9847844214BF0020ED
:100E90000120F8BD0020F8BD0020F8BD0020F8BDFD
:100EA0000020F8BD0020F8BD0020F8BD00000020A3
:100EB000000048000080022000004000F90D4000C2
:100EC000190E4000050E40002DE9F8430378442B2D
:100ED00002D00220BDE8F8834578A5F10803DBB213
:100EE000182B02D90520BDE8F88315F0070F02D0B2
:100EF0000520BDE8F8838678C37806EB03260379DE
:100F000006EB0346437906EB03661E4A1E4B9E42E0
:100F100002D20420BDE8F883964202D30420BDE843
:100F2000F8835FFA85F84FF0000918EB060849F1DD
:100F30000009B9F1010F08BFB8F1000F02D3042076
:100F4000BDE8F88300234B4508BF424502D2042088
:100F5000BDE8F8830446AA1D875C014600200B4BC0
:100F60009847874202D00620BDE8F88306F4FE7653
:100F70002A46A11D06483044064B98470020BDE88C
:100F8000F88300BF000048000040400029064000F0
:100F90001C040020653B4000F8B50378642B01D0A9
:100FA0000220F8BD4678A6F10803DBB2182B01D960
:100FB0000520F8BD8578C37805EB0325037905EB9B
:100FC0000345437905EB0365B5F5007F01D30420A4
:100FD000F8BDF2B20023521943F10003012B08BF00
:100FE000002A01D30420F8BDAB19B3F5007F01D965
:100FF0000420F8BD0446B21D875C01460020084B62
:101000009847874201D00620F8BDC5F38F053246C8
:10101000A11D044800EB8500034B98470020F8BD54
:10102000290640001C060020653B40000378652B24
:1010300001D00220704770B58478C37804EB032494
:10104000037904EB0344437904EB0364214B9C4292
:1010500001D3042070BD204B9C4201D2042070BDFE
:101060004378012B14D01BB1022B18D0022070BD85
:10107000C4F30C030BB1042070BD00260146857932
:1010800006220020154B984785421ED0062070BDD1
:10109000C4F30D030BB1042070BD0126EEE7104B25
:1010A0009C420CD0B4F5840F0BD0B4F5880F0AD055
:1010B000B4F58C0F01D0042070BD0226DEE70226B5
:1010C000DCE70226DAE70226D8E731462046054B60
:1010D000984770BD000048000040400029064000CD
:1010E00000404000510740002DE9F8430378502BA1
:1010F00003D002242046BDE8F88343780BB10524D1
:10110000F8E78478C27804EB0224027904EB024405
:10111000427904EB02641D4E1D4A944201D204241C
:10112000E8E7B44201D30424E4E75FFA83F84FF020
:10113000000918EB040849F10009B9F1010F08BFD3
:10114000B8F1000F01D30424D4E700274F4508BFAE
:10115000464501D20424CDE701469A1D855C002056
:101160000C4B9847854201D00624C3E70A4D2A4616
:101170004FF400712046094B984704464FF4007223
:10118000FF212846064B9847B4E700BF00004800FF
:1011900000404000290640001C040020ED074000EC
:1011A0007B3B400038B50378702B02D002242046E8
:1011B00038BD084B984704460028F8D1064D28460C
:1011C000064B984704464FF40072FF212846044B13
:1011D0009847ECE7B90840001C060020D9084000F9
:1011E0007B3B400008B50020014B984708BD00BF7D
:1011F000C5364000034AD2F800340133C2F8003447
:10120000704700BF1C040020044B01229A63802217
:101210001A604FF48032C3F80021704700040E407A
:101220004FF4C052134B1A61134AD2F8143123F40D
:101230004063C2F81431D2F8203143F00103C2F800
:1012400020310E4B4FF440615960196F21F4406119
:101250001967D2F8141141F02001C2F814114FF4AB
:1012600000721A601A615A6320221A601A615A6366
:10127000704700BF00040E4000020E4000100E40F8
:1012800000207047F8B51C46BDF818501B78223B6B
:101290004E2B00F26D81DFE813F073006B016B01E0
:1012A0006B016B016B016B016B014F006B016B01FB
:1012B0006B016B016B016B016B016B016B016B01CE
:1012C0006B016B016B016B016B016B016B016B01BE
:1012D0006B016B016B016B016B016500C9009C0028
:1012E0006B016B016B016B0161016B016B016B01A8
:1012F000E1006B016B01B4006B016B012A016B0112
:101300006B016B016B016B016B016B016B016B017D
:101310006B016B016B016B016B016B016B010001D8
:1013200087006B016B016B016B016B016B016B0142
:101330006B016B016B011501964C04F204462A46C1
:1013400000213046944B9847944B93E80300C4F82F
:10135000040484F80814EBB2324600210846904C8D
:10136000A047F8BD8F4A936823F07F4323F470634E
:1013700043F0254343F4E06393608B4B1360F8BD67
:101380008A4B98470746834E06F204442A460021BA
:101390002046814B984786F80474EBB22246002120
:1013A00008467F4CA047F8BD2046814B984707462A
:1013B000784E06F204442A4600212046764B984790
:1013C00086F80474EBB2224600210846744CA0470C
:1013D000F8BD2046774B98470446002800F0D88097
:1013E0006C4F07F204462A46002130466A4B984764
:1013F00087F80444EBB2324600210846684CA04707
:10140000F8BD20466C4B98470746624E06F20444EE
:101410002A4600212046604B984786F80474EBB2B8
:101420002246002108465E4CA047F8BD634B984712
:10143000584A82F80704C0F3072382F80634C0F341
:10144000074382F80534000E82F80404EBB202F27E
:10145000044200210846524CA047F8BD584B98471B
:1014600004464C4E06F204472A46002138464A4BB1
:10147000984786F80744C4F3072386F80634C4F374
:10148000074386F80534240E86F80444EBB23A4646
:1014900000210846424CA047F8BD2046494B9847DA
:1014A00007463C4E06F204442A46002120463A4BA9
:1014B000984786F80474EBB2224600210846384C5F
:1014C000A047F8BD2046404B98470746314E06F2EC
:1014D00004442A46002120462F4B984786F804747E
:1014E000EBB22246002108462D4CA047F8BD3748F4
:1014F000374B9847074680B1264E06F204442A46E9
:1015000000212046244B984786F80474EBB222460B
:1015100000210846224CA047F8BD1E4F4FF0000E98
:1015200087F804E407F500740FCCC7F80504C7F882
:101530000914C7F80D24C7F811340FCCC7F81504E7
:10154000C7F81914C7F81D24C7F82134EBB207F205
:10155000044271467046124CA047F8BD1D4BAA22AA
:101560001A6042F601425A600F4A903B1A60F8BD79
:10157000084E2A46002106F20440074B98470223F2
:1015800086F80434EBB2224600210846044CA047FA
:10159000F8BD00BF1C0400207B3B40009C3B40008A
:1015A0009D1A400000140E40080000A5B507400039
:1015B0002D104000C90E4000E9104000050E40000B
:1015C000190E4000990F4000A51140001C06002094
:1015D0001109400090140E40014BD3F800047047ED
:1015E0001C04002030B583B00446064DA847019086
:1015F000A84701E0034B9847019B23449842F9D345
:1016000003B030BDD9154000F0B587B000258DF886
:10161000075010238DF80830A24CA34B23602B23D6
:1016200023712A236371A1492046A14B9847204684
:10163000A04B9847A04F4FF400733B630A209F4E86
:10164000B04720233B630A20B0470595E7238DF878
:101650000B300DF10703049301238DF80C308DF846
:10166000093003238DF80A3002A92046944B98478D
:101670008C48944B98470028FAD19DF8073043F0E6
:1016800001038DF8073002238DF80A3002A985483E
:101690008B4B984783488B4B98470028FAD11223ED
:1016A0008DF8083003238DF80A3002A97D48844B59
:1016B00098477C48834B98470028FAD19DF807301B
:1016C00043F001038DF8073002238DF80A3002A998
:1016D00074487B4B984773487A4B98470028FAD157
:1016E00010238DF8083006238DF80B3003238DF876
:1016F0000A3002A96B48724B98476A48714B984769
:101700000028FAD19DF8073063F07F038DF8073089
:1017100002238DF80A3002A96248694B9847614854
:10172000684B98470028FAD100238DF807300C2326
:101730008DF80B3002A95B48614B98475948614BC3
:1017400098470028FAD10D238DF80B3002A955488F
:101750005B4B984753485B4B98470028FAD10E23C0
:101760008DF80B3002A94F48554B98474D48554BC3
:1017700098470028FAD10F238DF80B3002A9494869
:101780004F4B984747484F4B98470028FAD11223B0
:101790008DF8083006238DF80B3003238DF80A30BE
:1017A00002A94048464B98473E48464B9847002878
:1017B000FAD19DF8073063F07F038DF807300223DC
:1017C0008DF80A3002A937483D4B984735483D4BC4
:1017D00098470028FAD100238DF807300C238DF8A4
:1017E0000B3002A92F48364B98472E48354B984767
:1017F0000028FAD10D238DF80B3002A92948304B6F
:10180000984728482F4B98470028FAD10E238DF887
:101810000B3002A923482A4B98472248294B984766
:101820000028FAD10F238DF80B3002A91D48244B54
:1018300098471C48234B98470028FAD110238DF86D
:101840000830E7238DF80B3003238DF80A3002A906
:1018500014481B4B984713481A4B98470028FAD155
:101860009DF8073023F001038DF8073002238DF82F
:101870000A3002A90B48124B98470A48114B984767
:101880000028FAD112238DF80830E7238DF80B30A9
:1018900003238DF80A3002A90248094B98470148F2
:1018A00012E000BF180A002000C00140A08601001D
:1018B000610B4000B10D400000100E40E5154000E6
:1018C000ED0B4000310C40000B4B98470028E6D14F
:1018D0009DF8073023F001038DF8073002238DF8BF
:1018E0000A3002A90548064B98470448024B98471E
:1018F0000028FAD107B0F0BD310C4000180A0020D2
:10190000ED0B400010B5BFF35F8FBFF36F8F72B662
:1019100000230CE0134A03F120044FF0FF3142F89A
:10192000241003F1600442F824100133DBB2072BCA
:10193000F0D900220C4B1A604FF480720B4B5A679F
:10194000BFF34F8FBFF36F8F20F07F02084B9A6079
:101950004368BFF35F8FBFF36F8F026882F308881D
:10196000984710BD00E100E010E000E000400440B6
:1019700000ED00E010B54FF400422F4B5A6072B6F4
:101980002E4B98472E4B98472E4B1B68AA2B2FD0D7
:101990002D4C20462D4B984758B12A4B1B68BB2B2A
:1019A00041D1284B5B681A2B3DD1264B00221A608F
:1019B0005A604FF40072FF212548264B9847264B6A
:1019C0009847264B264A5A60F021264A82F823106F
:1019D00000229A6007221A60234B9847BFF35F8F5B
:1019E00062B6224B9847224B9847224B9847FCE718
:1019F000144B5B6803F43053B3F5305FC8D1114B1F
:101A00005B68DAB2082A07D90E4B00221A605A60C6
:101A1000194A1A4B1A60BBE742F6014252FA83F3A5
:101A2000084A5360F4E7164B1B68002BC1D02046D0
:101A3000144B9847BDE700BF50140E4041074000CB
:101A4000ED04400090140E4000404000390E40006C
:101A50001C0400207B3B40002112400010E000E00D
:101A6000FF7F010000ED00E0091240000916400070
:101A700095394000612E4000080000A500140E407A
:101A8000940100200519400008B50248024B984710
:101A900008BD00BF180A0020350C4000F8B5054607
:101AA0000F4616461C468C231C4A03FB002359781C
:101AB00000201B4B9847034600B30FB33F2C28BFB1
:101AC0003F2416488C2303FB05F3C2181772083312
:101AD0001844224631460130124B98470134E4B293
:101AE0000E4A8C2000FB05F000F10801104423464B
:101AF0000A44417800200C4CA04703461846F8BD24
:101B0000402C28BF40248C2303FB05F308332246D6
:101B1000314602481844034B9847E1E7600800202B
:101B20009D284000653B4000F528400008B58C2208
:101B300000210248024B984708BD00BF6008002002
:101B40007B3B400008B50020014B984708BD00BF13
:101B50002D1B40004B79032B01D0002070472DE94D
:101B6000F04182B00B79C3EBC305ADB21235ADB213
:101B700095420DD93A4B1B6813F0010F64D000BE9B
:101B8000002002B0BDE8F0818C2202FB06460DE089
:101B9000002353B91E468C22324C02FB034252787A
:101BA000002AF1D00133DBB2F3E7002676B10B78DF
:101BB000CC18C6F888406278212A0FD0284B1B68C1
:101BC00013F0010F44D000BE0020DAE7244B1B685D
:101BD00013F0010F3AD000BE0020D2E70F46804636
:101BE000C95C3A79731C0193B31C0093032321440D
:101BF0001D4CA04730B91A4B1B6813F0010F29D0B8
:101C000000BEBEE7BB79012B0CD001233371BB783A
:101C10003370D6F88830B3F80730F380B17821B943
:101C20002846AEE7FB79F370EFE7402306F1480260
:101C300040460E4CA04778B9094B1B6813F0010FC2
:101C40000CD000BE28469CE700209AE7002098E7C9
:101C5000002096E7002094E7284692E7284690E780
:101C6000F0ED00E06008002019284000F528400051
:101C70002DE9F04182B0137803F01F04012C04D049
:101C80000023184602B0BDE8F0819488E5B2002434
:101C9000ACB1FF24002C40F00A81154606462746C9
:101CA00013F0600339D1002940F0038153881B0AE7
:101CB0005278062A0DD0062A1CD00023E1E78C2694
:101CC00006FB04F6824FBE5DB542E3D00134E4B2B8
:101CD000DEE7212BEFD18C237D4A03FB0427D7F8C5
:101CE0008820002A00F0E78013782946794CA04725
:101CF0000346C6E7222B01D00023C2E72046764BDD
:101D000098478C23724A03FB0727FB880246294623
:101D10003046704CA0470123B3E7202B01D00023AD
:101D2000AFE75378013B0A2B00F2C780DFE803F0EE
:101D3000068C9AC5C5C5C5C54275A800002940F0E6
:101D4000BE806B881A0ADFF888C18C2000FB04F083
:101D500008300CEB0008B5F806E013F0FF010CD0DA
:101D6000BEF1010F1CD908F101030CF800100EF1AF
:101D7000FF3E1FFA8EFE012701E043460027CDF803
:101D800000E02046554CA0473B189BB25BB9544B32
:101D90001B6813F0010F00F0948000BE002370E771
:101DA00043460027EBE7424629463046494CA047C8
:101DB000012366E779B9EB88402B01D9002360E75E
:101DC0008C2202FB04F2483241490A442946414C24
:101DD000A047012355E7022901D0012351E7698873
:101DE0000A0ADFF8ECE08C2606FB04F648360EEB18
:101DF0000603E88811F0FF0105D0012803D91EF879
:101E00000650A94205D000902046364CA047012339
:101E100037E70133013880B2F5E7002953D16988EB
:101E2000090A8C232A4A03FB042779712E4B2BB114
:101E300020469847034600283FF423AF2946304602
:101E40002A4B984701231CE709B1012319E78C228B
:101E50001F4B02FB04320123053229461D4CA047CB
:101E600001230EE709B101230BE78C22184B02FB7B
:101E70000432012304322946164CA047012300E70F
:101E800019B1022906D00123FBE62946174B9847D2
:101E90000123F6E66988C9B28C220D4B02FB043798
:101EA0003971134B8BB1204698470123E9E6002393
:101EB000E7E60123E5E60023E3E60023E1E601236C
:101EC000DFE60023DDE60123DBE60123D9E600BFE0
:101ED0006008002059314000B13A400081124000B2
:101EE000F0ED00E0851240000000000019314000D4
:101EF00000000000F0B583B0254D002444B1A4B12A
:101F0000244B1B6813F0010F3ED000BE002314E0E9
:101F10008C251F4A05FB0425AA788A42EFD06A78EF
:101F20009142ECD00134E4B2E8E706466A78914287
:101F300006D0AA7891420DD00123184603B0F0BD17
:101F4000154A1AB3DAB205F108012046124B984738
:101F50000123F2E705F148079BB200933B460022BC
:101F6000114620460D4CA04740233A46A9783046FA
:101F70000B4CA04703460028DFD1064A126812F036
:101F8000010FDAD000BED8E70023D6E70123D4E75B
:101F900060080020F0ED00E0000000008512400025
:101FA000F52840000A4492B2914202D883899A42AD
:101FB00002D94089024492B2104670478A1A92B2FE
:101FC000914202D383899A4202D94089121A92B26D
:101FD00010467047838801E0C91A89B28B42FBD949
:101FE00008467047F8B504460F4611461D46D31AF9
:101FF0009BB2AA4202D242899B1A9BB2A6889E42F9
:1020000005D2324620460A4B9847208233460BB908
:102010000020F8BD29462046064B98472168E388F2
:102020001A4603FB00113846034B98470120F8BDC0
:10203000BD1F4000D51F4000653B400038B5044639
:10204000C289038A9BB292B2054DA8470546218AF0
:1020500082B289B22046034B98472082284638BD79
:10206000E51F4000A51F4000F8B5C589ADB2028A42
:1020700092B2AB1A9BB2954202D242899B1A9BB292
:1020800082889A4215D00E46044629460B4B984743
:102090002768E3881A46314603FB0070084B9847CF
:1020A000012229462046074B9847E0810123184624
:1020B000F8BD037A002BE6D1F9E700BFD51F400039
:1020C000653B4000A51F40000023C3810382838835
:1020D0005B009BB2013B9BB28381DB4343810120C8
:1020E0007047000038B5054600240CE0E31ADBB267
:1020F000DBB903EB4303DA00194B13445B68284652
:1021000098470134E4B2174B1B795A1C94420EDAFB
:10211000154A42B19C42E9D204EB4403DA00114B68
:102120001B681344EAE72346E2E70023E6E70D4C89
:102130002B22002104F108000C4B98474FF0FF338D
:10214000C4F80B30C4F80F30C4F81330C4F817309B
:10215000C4F81B30C4F81F30C4F8233038BD00BFAA
:10216000A43B4000EC080020000000007B3B400046
:1021700008B5024B9847024B984708BDE520400040
:10218000F131400070B505460C461646C868044B50
:102190009847E368324600212846984770BD00BF43
:1021A000053240002DE9F84F80460139C8B26E4B28
:1021B000984718B182464378022B09D06B4B1B68B5
:1021C00013F0010F00F0BB8000BE0020BDE8F88FC7
:1021D000C279C2F3401066490B7A60F30413C2F36C
:1021E000801262F345130B720AF10905BAF8023046
:1021F0009A447DE02B78A9461D4481E05B4B1B6827
:1022000013F0010F00F09E8000BE0020BDE8F88FA3
:10221000564B1B6813F0010F00F0978000BE0020A2
:10222000BDE8F88FE31ADBB203BB03EB4303514A6B
:1022300002EBC3039B6832462946404698478346D3
:10224000B0B90134E4B22746494B1B795A1C944279
:1022500049DA494A42B19C42E4D204EB4403444A7D
:10226000126802EBC303E5E72346DDE70023E1E75D
:10227000082814D9864212D3AA783D4B1344DC7245
:10228000B9F1000F28D099F80220AB789A420FD10B
:1022900099F804206B799A420AD1012318E0334B54
:1022A0001B6813F0010F53D000BE0020BDE8F88F6B
:1022B0002E4B1B6813F0010F4DD000BE0020BDE86F
:1022C000F88FAA7899182A4A0A44D4720133DBB2EB
:1022D00099F803209342F4D323465A4629462748C7
:1022E000274CA0475D44224B1B7901339F4217DAEC
:1022F00055451ED26B780B2B3FF47CAF4FF0000995
:102300006B78042B7FF47AAFAAEB0506B6B2AA78F5
:10231000174B1344DB7AFF2B7FF47AAF002492E74C
:10232000124B1B6813F0010F18D000BE0020BDE84F
:10233000F88F144BABB198470120BDE8F88F00200F
:10234000BDE8F88F0020BDE8F88F0020BDE8F88FC9
:102350000020BDE8F88F0020BDE8F88F0020BDE820
:10236000F88F0120BDE8F88FB93A4000F0ED00E0A9
:10237000EC080020A43B40000000000007090020FA
:102380007D3A40000000000038B505460C464888FC
:10239000020AC0B2531E0E2B4BD8DFE803F0081C14
:1023A000344A4A3F1C4A4A4A4A4A4A4A1100284B80
:1023B00098471223024621462846264CA04738BD9E
:1023C000254B002B37D098470246438821462846A4
:1023D000204CA04738BD022A0BD0204B002B2CD01C
:1023E000984748B14388024621462846194CA047E1
:1023F00038BD1B4B9847F4E71A4B1B6813F0010FCD
:102400001DD000BE38BDA188174B98470246C0B109
:102410000378214628460F4CA04738BD134B93B193
:102420009847024688B1037821462846094CA047C0
:1024300038BD002038BD002038BD002038BD002048
:1024400038BD002038BD002038BD002038BD00BF99
:10245000A93A40005931400000000000000000008F
:10246000B93A4000F0ED00E0C13A40000000000041
:10247000014B93F833007047EC080020234B93F88E
:1024800033300BB11846704770B505461F4C2B22F0
:10249000002104F108001E4B98471E4E301D1E4BB4
:1024A000984766631D4B13B1201D98472060002498
:1024B0000FE0E31ADBB23BB903EB4303DA00184B3E
:1024C000134402E02346F6E700231B6898470134D3
:1024D000E4B20E4B1B795A1C94420BDA0F4A002AC5
:1024E000F0D09C42E5D204EB4403DA00074B1B68B2
:1024F0001344EAE728460B4B984728460A4B98476F
:102500000123024A82F83330184670BDEC080020DF
:102510007B3B4000DC010020C9204000000000009F
:10252000A43B4000753440003D34400070B584B099
:1025300004460D464378023B032B00F2B880DFE8E7
:1025400003F002832F5A6B4B1A7A6FF300021A7250
:102550001A7A6FF341021A72002159721A7A61F3E2
:1025600082021A725E6B15B93378012B10D02146A6
:10257000301D614B9847044615B93378012B0BD0B9
:102580009CB95E4B1B6813F0010F0ED000BE0CE02F
:1025900008465B4B9847EAE700205A4B9847EFE71D
:1025A000544B1B7A13F0010F01D104B070BD514B95
:1025B0001A7A42F004021A725E6B11B93378012B59
:1025C00011D02146301D4C4B9847044615B933783D
:1025D000012B0CD0002CE8D1484B1B6813F0010FE5
:1025E000E3D000BEE1E70020454B9847E9E7002033
:1025F000444B9847EEE73F4B1B7A13F0010FD4D0C2
:102600003C4A137A6FF382031372566B11B9337815
:10261000012B11D02146301D374B9847044615B980
:102620003378012B0CD0002CBFD1344B1B6813F036
:10263000010FBAD000BEB8E70020314B9847E9E758
:102640000020304B9847EEE72A4B1B7A13F0040F1B
:10265000ABD0284A137A6FF38203137200230193DD
:102660000293039303788DF8043005238DF8053029
:10267000546B11B92378012B11D001A9201D1E4BD9
:102680009847064615B92378012B0CD0002E8CD123
:102690001A4B1B6813F0010F87D000BE85E700209E
:1026A000174B9847E9E70020164B9847EEE7114B88
:1026B0005E6B11B93378012B13D02146301D0E4BC0
:1026C0009847044615B93378012B0ED0002C7FF4BF
:1026D0006CAF0A4B1B6813F0010F3FF466AF00BEEE
:1026E00063E70020064B9847E7E70020054B984733
:1026F000ECE700BFEC08002069204000F0ED00E0AE
:102700004D3440003D34400000B585B000230193B6
:10271000029303938DF804008DF80510114601A86B
:10272000024B984705B05DF804FB00BF2D25400023
:1027300000B585B000230193029303938DF8040044
:1027400001238DF805308DF80810114601A8024BC1
:10275000984705B05DF804FB2D25400000B585B015
:10276000002301938DF8040006238DF8053002AB99
:102770000868496803C3114601A8024B984705B091
:102780005DF804FB2D25400010B584B000240194B1
:1027900002948DF8040007208DF805008DF80810CC
:1027A00003928DF809309DF8181001A8014B984745
:1027B00004B010BD2D25400038B58B7803F07F03A1
:1027C000052B08D9104B1B6813F0010F19D000BE60
:1027D0000023184638BD0C4605460C4B997A204616
:1027E0000B4B9847034630B9074A126812F0010FA5
:1027F000EFD000BEEDE721462846064B984703463A
:10280000E7E70023E5E700BFF0ED00E0EC0800207B
:10281000C9394000D53440002DE9F04780460C46C8
:1028200016461F46DDF82090DDF824A0002513E0B1
:10283000184B1B6813F0010F2AD000BE002324E0C0
:10284000144A126812F0010F1FD000BE1DE08AF872
:10285000003023781C440135B54215DA6378052B26
:10286000E6D1E37803F00303BB42E1D121464046C1
:10287000094B984703460028E2D0A37813F0800F55
:10288000E5D189F80030E4E701231846BDE8F08778
:102890000023FAE7F0ED00E0B927400010B401F0A2
:1028A0007F04C909124B03EB44030B442033DB794B
:1028B00013F0010F0AD10E4A02EB44020A4492F8C7
:1028C000273013F0040F10D0002200E00022104641
:1028D0004AB1074B03EB4403194491F8273043F006
:1028E000040381F8273010BC70470122EFE700BFD6
:1028F000EC080020F8B501F07F06CD091C4C04EB74
:1029000046042C442034E47914F0010F08D0194B0C
:102910001B6813F0010F29D000BE00231846F8BD34
:10292000134C04EB46042C4494F8277047F001073D
:1029300084F82770104CA04703460028EED10C4ABB
:1029400002EB4606354495F827206FF3000285F820
:10295000272095F827206FF3820285F82720054A63
:10296000126812F0010FD9D000BED7E70023D5E7D7
:10297000EC080020F0ED00E09935400038B501F09A
:102980007F05CC090E4B03EB450323442033DB7951
:1029900013F0020F00D038BD0A4B9847084B03EBE9
:1029A0004503234493F8272042F0020283F82720AE
:1029B00093F8272042F0010283F82720EBE700BFBD
:1029C000EC0800203D36400038B501F07F05CC0909
:1029D0000E4B03EB450323442033DB7913F0020F46
:1029E00000D138BD0A4B9847084B03EB45032344FD
:1029F00093F827206FF3410283F8272093F82720CC
:102A00006FF3000283F82720EBE700BFEC080020FB
:102A10007536400001F07F02044B03EB420303EBE9
:102A2000D11191F82700C0F340007047EC08002056
:102A30002DE9F04182B005460C4600209D4B984799
:102A40002378C3F34113022B0BDD9B4B1B6813F060
:102A5000010F00F0D58100BE0023184602B0BDE88A
:102A6000F081237803F06003402B12D0227802F02B
:102A70001F02012A00F0E880CAB1022A00F04E814C
:102A80008D4B1B6813F0010F00F0D28100BE0023B4
:102A9000E3E78A4B002B00F0B5811E461846854BB4
:102AA0009847224600212846B0470346D5E7202B09
:102AB0000AD0002B30D0804B1B6813F0010F00F0C0
:102AC000A78100BE0023C8E7A388DBB20F2B00F26A
:102AD0009B817B4A1344DB7A7A4AA2B1784A127905
:102AE00093420ED203EB4303DA00754B196811448D
:102AF000002900F08B8122462846734B98470346F5
:102B0000ABE79B1ADBB22BB903EB4303DA006F4947
:102B10001144EDE70021EBE76378092B00F28B808D
:102B2000DFE803F07464895489054E891420204637
:102B3000674B98476188C9B22846664B9847604AF8
:102B4000137A43F002031372012386E75C4B5B7A2E
:102B500002AA02F8023D0123214628465E4CA04706
:102B600001237AE76688F6B2554B5B7ADBB29E4268
:102B700003D0534B5B7A43B99EB9514B5E722146E9
:102B80002846564B9847012367E72846544B9847F9
:102B90004B4F97F80A802846524B984787F80A808F
:102BA000EAE731462846504B984703460028E4D1CF
:102BB000414A126812F0010F3FF44FAF00BE4CE7DC
:102BC00021462846494B9847034646E76388012B30
:102BD00001D0002341E73A4A137A43F00803137205
:102BE000214628463D4B9847012336E76388012B51
:102BF00001D0002331E7324B1A7A6FF3C3021A7205
:102C000021462846354B9847012326E72C4B1B7A53
:102C1000C3F3401213F0080F0BD10023134302AA91
:102C200022F8023D0223214628462B4CA0470123CF
:102C300013E70223F2E7204B1B6813F0010F00F0AB
:102C4000E98000BE002308E7A388DBB20F2B00F267
:102C5000E3801B4A1344DB7A1A4A002A4AD0184AF6
:102C60001279934244D203EB4303DA00144B196800
:102C70001144002900F0D28022462846124B984782
:102C8000034600287FF4E9AE227812F0600F7FF44B
:102C9000E4AE62780A3A012A3FF6DFAE054B984768
:102CA00063780A2B2FD0214628460C4B98470123E6
:102CB000D3E600BF05324000F0ED00E00000000068
:102CC000EC0800200000000085214000A43B4000EB
:102CD000113240002936400059314000193140007E
:102CE00095354000E5204000A521400089234000A3
:102CF0009B1ADBB22BB903EB4303DA004D491144B5
:102D0000B7E70021B5E702AA002302F8023D01233C
:102D100021462846484CA04701239EE6A288D1B20E
:102D200001F07F06C2F3C012052E07D9434B1B6882
:102D300013F0010F74D000BE00238EE6404800EB74
:102D400046000244D27E3F48A8B13D480079824205
:102D50000FD202EB4202D000394A166806449BB1FA
:102D6000002E5FD0224631462846374B984703460F
:102D700073E6121AD2B22AB902EB4202D0002D4EEB
:102D80000644ECE70026EAE76378012B17D04BB145
:102D9000032B14D0294B1B6813F0010F46D000BE43
:102DA00000235AE62846294B984702AA22F8020D2A
:102DB000022321462846204CA04701234DE6628885
:102DC00022B9012B18D02846214B984766B32246DA
:102DD000314628461C4B984700201E4B9847184BFD
:102DE00093F8283013F001037FF437AE21462846CC
:102DF000194B9847012330E62846184B9847E5E7DA
:102E000000232AE6002328E6002326E6002324E602
:102E1000002322E6002320E600231EE600231CE612
:102E200000231AE6002318E6012316E6002314E621
:102E3000002312E6A43B400059314000F0ED00E0D1
:102E4000EC0800200000000085214000152A400009
:102E50007D2940000532400019314000C929400059
:102E600030B585B0884B984788B905B030BD002093
:102E7000864B984710E00020854B984714E09DF85A
:102E80000400844B98479DF80820834B9A72824B2C
:102E90005C6B2378012BEAD001A9201D7F4B98475A
:102EA00005462378012BE6D0002DDED09DF80530B5
:102EB000013B072B00F2E08001A252F823F000BF93
:102EC0007F2E4000E12E400067304000E52F40009B
:102ED00007304000F32E40004F2F40006B30400081
:102EE0009DF804006B4B98476D4B002BCFD0984753
:102EF000CDE7694B1A7A42F001021A7293F8272043
:102F00006FF3000283F8272093F827206FF38202E3
:102F100083F8272093F828206FF3000283F82820F5
:102F200093F828206FF3820283F8282002A99DF8E5
:102F300004005C4B98470028A9D100219DF80400AB
:102F4000594CA04780219DF80400A0479FE79DF8B9
:102F5000081001F07F00CC094F4B03EB40032344E2
:102F600093F827206FF3000283F8272093F8272097
:102F70006FF3820283F8272088B1474B03EB4003AD
:102F80002344DB7E494AA2B1434A127993420ED2CE
:102F900003EB4303DA00404B1B6813440FE0039B31
:102FA0009DF809209DF80400414CA0476FE79B1A4B
:102FB000DBB26BB903EB4303DA003E4B13444BB176
:102FC0001C69039B9DF809209DF80400A0475EE75B
:102FD0000023F4E7384B1B6813F0010F3FF445AFB3
:102FE00000BE42E72C4B1B7A13F0010F3FF44FAFAA
:102FF000324B002B3FF44BAF274B187AC0F3C00085
:103000002E4B984743E7244B1B7A13F0010F3FF4F4
:103010003EAF2B4B002B3FF43AAF984737E7E31A0C
:10302000DBB2F3B903EB4303DA00224B13445B69D1
:1030300013B19DF8040098470134E4B2164B1B7994
:103040005A1C9442BFF623AF184A42B19C42E6D2C2
:1030500004EB4403DA00104B1B681344E7E72346F4
:10306000DFE70023E3E70024E8E7029B002B3FF4BF
:103070000EAF039898470AE70F4B1B6813F0010F38
:103080003FF405AF00BE02E7B93940004D344000BF
:103090003D34400071214000EC0800203D204000FC
:1030A00000000000312A40003D36400000000000D2
:1030B00031324000A43B4000F0ED00E00000000091
:1030C0000000000038B50546104BB3F84C40B3F88B
:1030D0004E20A41AA4B2402C28BF402493F94030BB
:1030E000002B07DB00217CB9002223462846084C30
:1030F000A04738BD0CB98021F5E704482246816C11
:10310000044B98478021EEE7004AEEE724090020AF
:10311000F5284000653B400038B505460C460C4B91
:1031200003F140020868496803C200229A64A3F8C8
:103130004E20A3F84C2094F90030934206DB802106
:1031400000231A462846034CA04738BD1146F7E72E
:1031500024090020F5284000F8B507460C46204D0C
:1031600005F140060868496803C6AA640021A5F86D
:103170004E10E1888B4228BF0B46A5F84C30E18801
:10318000A9B103B15AB13846164B9847034600BB64
:10319000154A126812F0010F1BD000BE19E0124B45
:1031A0001B6813F0010F18D000BE002311E094F942
:1031B0000030002B0FDB802100231A4638460B4CD1
:1031C000A047034628B9084A126812F0010F00D040
:1031D00000BE1846F8BD0021EEE70023F9E700BF66
:1031E00024090020C5304000F0ED00E0F528400043
:1031F000034900230B644B648B64CB640B657047FD
:1032000024090020014B1865704700BF24090020E5
:103210000146064B03F140020068496803C20022E0
:103220009A64A3F84E20A3F84C207047240900208C
:1032300038B505461C463C4B93F84030DB09B3EBF0
:10324000D11F17D03CB1394B1B6813F0010F65D06B
:1032500000BE00230CE0364B0BB136499847324B89
:103260001B6D002B5CD0334A02212846984701236E
:10327000184638BD2C4B93F94030002B07DB2A4B06
:10328000986C00284ED0224619462B4B9847264A68
:10329000B2F84E3023449BB2A2F84E30916C2144D8
:1032A0009164B2F84620934201D03F2C29D81E4B9E
:1032B0001B6DCBB11F4A012128469847C0B11A4B5C
:1032C00093F94030002B11DB802100231A46284659
:1032D0001A4CA04703460028CAD1144A126812F0BB
:1032E000010FC5D000BEC3E70120E7E70021ECE7EE
:1032F00000212846124CA04780212846A0470123E0
:10330000B6E728460F4B984703460028B0D1074A36
:10331000126812F0010FABD000BEA9E70023A7E7A7
:103320000123A5E70023A3E724090020F0ED00E036
:103330009934400064090020653B4000F5284000B6
:103340003D364000C5304000002393420CD270B49B
:10335000CE5C00F11404054D45F8246001339BB2A6
:103360009342F5D370BC7047704700BF00400440E3
:10337000002393420CD230B400F11404054D55F8EB
:103380002440CC5401339BB29342F5D330BC7047F8
:10339000704700BF004004400181704710B582B003
:1033A000104C4822002120460F4B984740212046D0
:1033B0000E4B98474FF400420D4B1A6300230193C4
:1033C00003E000BF019B01330193019B132BF8D94C
:1033D000074B42F201321A615A6F22F480725A6727
:1033E00002B010BDEC0A00207B3B40009933400046
:1033F00000400440016082800023C38070470023A6
:1034000003608380C38070478388C28892B29B1A0E
:103410009BB20089984228BF1846704710B50446F1
:10342000054B9847236803442360E38810FA83F030
:1034300080B2E08010BD00BF093440004FF48032FC
:10344000014B5A60704700BF00E100E04FF480324A
:10345000034BC3F88420BFF34F8FBFF36F8F7047C8
:1034600000E100E04FF44072014B5A67704700BF23
:103470000040044010B50446482200210348044B94
:1034800098472046034B984710BD00BFEC0A002028
:103490007B3B4000653440000B7813F07F0F04D174
:1034A0004B78052B02D0092B0CD070474B88084A6B
:1034B000516841F00101516003F07F0343F48073D0
:1034C00093607047024A536843F002035360ECE78D
:1034D00000400440F0B583B08C78CB7803F0030350
:1034E000012B48D004F07F0564B2E70F052D44D8C6
:1034F00005F10C03234A52F8233013F4004F07D090
:10350000214B1B6813F0010F3AD000BE002035E0BC
:103510000E460979737903F0070305EB4500820035
:1035200041EA032119481044194B9847F37803F0F6
:10353000030303EB87031B0203F4E06343F400433C
:1035400005F10C020F4941F822300023019303E0FA
:1035500000BF019B01330193019B132BF8D9002C71
:1035600001DB01200AE0074A1369012000FA05F592
:103570001D43156102E0002000E0002003B0F0BD13
:103580000020FBE700400440F0ED00E0EC0A0020E2
:103590009933400070470000F0B583B0174601F042
:1035A0007F044DB204EB440082001A4E16441A46C2
:1035B00039463046184B9847002D0ADB34B117497D
:1035C0000B69012202FA04F41C430C61012003B0D0
:1035D000F0BD04EB440293000E4AD5583046104B20
:1035E00098470246294620460E4B98470B4A0C3412
:1035F00052F8243043F05F0342F824300023019353
:1036000003E000BF019B01330193019B132BF8D909
:10361000DCE700BFEC0A0020F53340000040044026
:10362000093440004933400010B500231A46802178
:10363000014CA04710BD00BF99354000802915D02E
:1036400082B001F07F010A4A0C3152F8213043F078
:103650006F0342F821300023019303E000BF019B78
:1036600001330193019B132BF8D902B0704700BFBF
:103670000040044082B001F07F01114A01F10C00CA
:1036800052F8203023F0200343F04F0342F820305B
:103690000023019303E000BF019B01330193019BD1
:1036A000132BF8D9064B986A012202FA01F108435C
:1036B00098629A6A22EA0101996202B0704700BFDB
:1036C000004004402DE9F0478AB00646A54B9D69AD
:1036D000DA6915401D6215F4805F12D115F4807F00
:1036E00017D115F4007F1AD115F4005F1DD115F024
:1036F000010F04D09B4B1B6B13F0040F38D1002437
:10370000F9E0994B9847012200213046974B9847A2
:10371000E4E7012204213046954B9847E1E7012276
:1037200005213046924B9847DEE7012205213046BD
:103730008F4B9847DBE78B4A116D0AAA1A4402F8AF
:10374000081C0133DBB2072BF5D9012208A930464A
:10375000884B98479DF92030002B0BDB814A136B77
:1037600023F0800343F04F0313630023039315E01A
:103770000023E8E77B4A136B43F0CF031363002376
:10378000029303E000BF029B01330293029B132BC1
:10379000F8D906E000BF039B01330393039B132B6F
:1037A000F8D9704A136B23F07F031363002304934B
:1037B00003E000BF049B01330493049B132BF8D94F
:1037C0009DE740466C4B984740466C4B98470246F5
:1037D00040B304EB44018B006949C9582046694B4A
:1037E0009847604A04F10C0152F8213043F05F031E
:1037F00042F821300023059303E000BF059B01330D
:103800000593059B132BF8D9564A07F10C0152F882
:10381000213023F0010343F04E0342F8213000230E
:10382000069317E004EB44039A00554B1344DA88DF
:1038300001230093002392B244F080013046DFF868
:103840005091C8474046504B9847DDE700BF069B64
:1038500001330693069B132BF8D963E007F10C03A1
:1038600052F8232007EB47018B00C2F30A42444978
:10387000C9582046454B984740463F4B98474046DD
:103880003E4B9847C0B92CB136494B690122BA402A
:1038900013434B6107EB47039A00394B1344DA8813
:1038A00001230093002392B221463046DFF8E0A0C6
:1038B000D0474046344B98472A4A07F10C0152F84A
:1038C000213043F04F0323EA090342F8213000235B
:1038D000079303E000BF079B01330793079B132B5C
:1038E000F8D927E000BF089B01330893089B132BEE
:1038F000F8D90134E4B2052C30D8274625FA04F370
:1039000013F0010FF5D004EB44034FEA83081C4B7E
:10391000984404F10C03134A52F8233013F0010FBA
:103920007FF44FAF07F10C030E4A52F8233013F027
:10393000420993D107F10C030A4A52F8233013F0DD
:10394000080FD6D00C3752F8273023F0080343F085
:10395000470342F8273000230893C7E70AB0BDE8C1
:10396000F08700BF004004409D33400031274000F5
:10397000092740005D2740001D3440000934400005
:10398000EC0A002049334000FF334000713340000F
:103990008927400008B50020054B9847034628B901
:1039A000044A126812F0010F00D000BE184608BD8C
:1039B0007D244000F0ED00E008B5024B984700B1CF
:1039C000012008BD712440000279437903F0070308
:1039D00042EA0322C37803F00303022B13D029D851
:1039E000012B37D102290BD040F2FF33934233D25F
:1039F000214B1B6813F0010F30D000BE0020704730
:103A00004FF48063F2E7022909D0402A2CD91A4BDF
:103A10001B6813F0010F29D000BE00207047B2F5DB
:103A2000007F1DD0144B1B6813F0010F1AD000BE8D
:103A30000020704702290AD04023934218D20E4B2F
:103A40001B6813F0010F15D000BE002070474FF423
:103A50008063F2E700207047012070470020704724
:103A600001207047002070470120704700207047F8
:103A70000120704700207047F0ED00E070B4002492
:103A800003E00D782C44A4B2294494420AD24D7824
:103A9000052DF6D18D7805F07F0600EB4606ED0981
:103AA0007355EEE770BC704700487047BC3B400060
:103AB00000487047D03B400000487047F43B40004E
:103AC00010B560B9124B1B681A88124B5A8001203E
:103AD000431C5B0043F440730E48038010BD032871
:103AE00014D80B4A52F8204020460B4B9847C0B2DE
:103AF0001F2800D91F20002305E05A1CE15C054B5C
:103B000023F81210D3B29842F7D8E1E7002010BD95
:103B1000F4010020780900208B3B400070B50D4E69
:103B20000D4CA41BA4100025A54209D10B4E0C4C32
:103B300000F092F8A41BA4100025A54205D170BD89
:103B400056F8253098470135EEE756F82530984766
:103B50000135F2E7643C4000643C4000643C4000B6
:103B6000683C400010B5431E0A44914200D110BD8C
:103B700011F8014B03F8014FF7E702440346934263
:103B800000D1704703F8011BF9E7034613F8012B36
:103B9000002AFBD1181A013870470000302E312E50
:103BA00033000000451B40002D1B4000551B40000A
:103BB000711C4000F51E40000000000012010002D0
:103BC00000000040BD350440000101020301000077
:103BD0000600FF0901A1010902150026FF00750872
:103BE000954081020903150026FF00750895409154
:103BF00002C000000902290001010080320904000E
:103C00000002030000000921110100012222000727
:103C100005020340000A0705810340000A00000076
:103C20000904000042696773637265656E000000F5
:103C300042696773637265656E2055534220466919
:103C4000726D7761726520557067726164650000FE
:103C50003132333435360000F8B500BFF8BC08BC4B
:103C60009E46704729044000F8B500BFF8BC08BC68
:103C70009E4670470504400082B0154B1A6842F416
:103C800080321A60134A5A60114B9B680193019B62
:103C900013F0010FF8D1002306E09A0002F580022C
:103CA000126840F8232001338B42F6D30A4A084BAE
:103CB0005A60074B9B680193019B13F0010FF8D0EA
:103CC000034A136823F48033136002B0704700BFC7
:103CD000000A0E400E00005A0F00005A82B00F4B2F
:103CE00058600E4B9B680193019B13F0010FF8D0B5
:103CF000019B13F0020F02D0022002B07047019B1B
:103D000013F0080F01D00320F7E7019B13F0040F15
:103D100001D10020F1E70120EFE700BF000A0E40CB
:103D200082B0104B58600F4B9B680193019B13F0BE
:103D3000010FF8D0019B13F0020F02D0022002B055
:103D40007047019B13F0080F01D00320F7E7019B98
:103D500013F0040F04D1034BDB680B600020EEE787
:103D60000120ECE7000A0E4010B483B0214C6060E3
:103D7000204880680190019810F0010FF8D1019857
:103D800010F0020F03D0022003B010BC704701985E
:103D900010F0080F01D00320F6E7019810F0040F8F
:103DA00026D1002005E0144C54F8204042F8204071
:103DB00001309842F7D30F4B59600E4B9B6801932B
:103DC000019B13F0010FF8D0019B13F0020F01D0FB
:103DD0000220D9E7019B13F0080F01D00320D3E79D
:103DE000019B13F0040F01D10020CDE70120CBE7A8
:103DF0000120C9E7000A0E400000400000127A00CE
:103E00000100000040000000887B002019114100E3
:103E10001511410015114100151141001511410006
:103E2000151141000000000000000000000000002B
:103E300000000000B1144100151141000000000015
:103E40001115410075154100010000002C0A0020E9
:103E500010000C000000E0FF1F0000000000000048
:103E6000203C4000243C4000303C4000503C40009E
:103E7000FFFFFFFFFFFFFFFFFFFFFFFFFD28E12127
:103E8000FFFFFFFFFFFFFFFFFFFFFFFFFFFFFFFF42
:103E9000FFFFFFFFFFFFFFFFFFFFFFFFFFFFFFFF32
:103EA000FFFFFFFFFFFFFFFFFFFFFFFFFFFFFFFF22
:103EB000FFFFFFFFFFFFFFFFFFFFFFFFFFFFFFFF12
:103EC000FFFFFFFFFFFFFFFFFFFFFFFFFFFFFFFF02
:103ED000FFFFFFFFFFFFFFFFFFFFFFFFFFFFFFFFF2
:103EE000FFFFFFFFFFFFFFFFFFFFFFFFFFFFFFFFE2
:103EF000FFFFFFFFFFFFFFFFFFFFFFFFFFFFFFFFD2
:103F0000FFFFFFFFFFFFFFFFFFFFFFFFFFFFFFFFC1
:103F1000FFFFFFFFFFFFFFFFFFFFFFFFFFFFFFFFB1
:103F2000FFFFFFFFFFFFFFFFFFFFFFFFFFFFFFFFA1
:103F3000FFFFFFFFFFFFFFFFFFFFFFFFFFFFFFFF91
:103F4000FFFFFFFFFFFFFFFFFFFFFFFFFFFFFFFF81
:103F5000FFFFFFFFFFFFFFFFFFFFFFFFFFFFFFFF71
:103F6000FFFFFFFFFFFFFFFFFFFFFFFFFFFFFFFF61
:103F7000FFFFFFFFFFFFFFFFFFFFFFFFFFFFFFFF51
:103F8000FFFFFFFFFFFFFFFFFFFFFFFFFFFFFFFF41
:103F9000FFFFFFFFFFFFFFFFFFFFFFFFFFFFFFFF31
:103FA000FFFFFFFFFFFFFFFFFFFFFFFFFFFFFFFF21
:103FB000FFFFFFFFFFFFFFFFFFFFFFFFFFFFFFFF11
:103FC000FFFFFFFFFFFFFFFFFFFFFFFFFFFFFFFF01
:103FD000FFFFFFFFFFFFFFFFFFFFFFFFFFFFFFFFF1
:103FE000FFFFFFFFFFFFFFFFFFFFFFFFFFFFFFFFE1
:103FF000FFFFFFFFFFFFFFFFFFFFFFFFFFFFFFFFD1
:10400000205400204DDF400019504000B9524000BC
:104010000DE040000DE040000DE040000000000019
:1040200000000000000000000000000001E340006C
:104030000DE040000000000061E34000C5E34000E7
:104040000DE040000DE040000DE040000DE04000BC
:104050000DE040000DE040000DE0400000000000D9
:104060000DE04000550541000000000019BB400074
:104070002DBB40005DD740000DE040000DE040004A
:104080000DE040000DE040006DD74000B5904000CD
:10409000690541000DE040000DE040005D54400026
:1040A0000DE040000DE040000DE040000DE040005C
:1040B0000DE04000A94A40000DE040000000000073
:1040C00000000000000000000000000000000000F0
:1040D00000000000000000000000000000000000E0
:1040E00000000000000000000000000000000000D0
:1040F0000000000000000000000000000DE0400093
:104100002DCC40000DE04000000000000000000049
:10411000000000000000000000000000000000009F
:10412000000000000000000000000000000000008F
:10413000000000000000000000000000000000007F
:10414000000000000000000000000000000000006F
:104400005C1D010010B5054C237833B9044B13B182
:104410000448AFF300800123237010BDE80C002096
:1044200000000000745041000C4B43B10C480D4992
:1044300010B5AFF300800C48036823B910BD0A48DB
:10444000036833B97047094B002BF7D0BDE8104023
:104450001847064B002BF5D0184700BF000000009E
:1044600074504100EC0C002074504100000000002A
:104470000120704770470120704700207047704747
:1044800001207047014B1878704700BF0C0D0020C9
:104490007047000058B908B5054B1B78012B00D0B8
:1044A00008BD044B1B68002BFAD09847F8E770470B
:1044B000100D0020040D002008B50C4B9847C37860
:1044C0000B4A1370012B0CD101220A4B1A700022E7
:1044D000094B1A80094B9847094B1B681BB1984739
:1044E00001E0084B9847012008BD00BF61B74000BC
:1044F0000C0D0020100D00200E0D00203505410090
:10450000040D00204105410008B5054B1B78012B27
:1045100000D008BD0022034B1A70034B9847F8E700
:104520000C0D0020100D00204105410010B582B097
:10453000074B00930B46024600218420054CA04700
:1045400018B9054A13680133136002B010BD00BFEB
:104550009544400065D34000080D0020014B1860D1
:10456000704700BF040D00202DE9F0474FF40046CE
:10457000BF4B5E600B20BF4CA0470C20A047BE4B3A
:104580004FF0400CC3F810C0C3F8A0C0C3F834C04B
:104590004FF0807EC3F810E0C3F8A0E0C3F834E029
:1045A000B64A01271761C2F8A0705763022414614C
:1045B000C2F8A04054631C61C3F8A0405C631F664E
:1045C000C3F890705F655F62C3F88070196F3943FC
:1045D0001967596F21F0010159675F604FF480310D
:1045E0001966C3F8901059655962C3F88010186FA6
:1045F00008431867586F20F48030586759601C6171
:10460000C3F8A0405C6304205861C3F8A00058665A
:10461000C3F8900058655862C3F88000196F21F004
:1046200004011967596F21F00401596718211966AF
:10463000C3F8901059655962C3F880101D6F25F0BA
:1046400018051D675D6F25F018055D675960082521
:104650001D66C3F890505D655D62C3F88050196FA8
:1046600021F008011967596F21F0080159675D6051
:1046700010211966C3F8901059655962C3F880106B
:10468000D3F8708028F01008C3F87080D3F87480D5
:1046900028F01008C3F8748059604FF48028C3F8DC
:1046A0001480C3F8A0804FF02009C3F81490C3F819
:1046B000A090C3F810C0C3F8A0C0C3F834C0C3F8BA
:1046C00010E0C3F8A0E0C3F834E01761C2F8A070AE
:1046D00057631461C2F8A04054634FF4007CC3F8E0
:1046E00060C0C3F890C0C3F854C0C3F824C0C3F876
:1046F00080C01C6F44EA0C041C675C6F24F40074D7
:104700005C67C3F804C04FF480641C66C3F8904033
:104710005C655C62C3F880401F6F27431F675F6F53
:1047200027F480675F675C604FF4006EC3F810E0A9
:10473000C3F8A0E0C3F834E04FF400275F61C3F88A
:10474000A0701F66C3F890705F655F62C3F88070E9
:104750001F6F27F400271F675F6F27F400275F672D
:104760004FF480175F61C3F8A0701F66C3F89070A4
:104770005F655F62C3F880701F6F27F480171F6743
:104780005F6F27F480175F674FF480575F61C3F84E
:10479000A0705F66C3F890705F655F62C3F8807059
:1047A0001F6F27F480571F675F6F27F480575F677D
:1047B0004FF400575F61C3F8A0704FF480775761E2
:1047C000C2F8A0704FF48048C3F86080C3F89080AE
:1047D000C3F85080C3F82480C3F88080D3F870A059
:1047E0002AF4804AC3F870A0D3F874A02AF4804A4F
:1047F000C3F874A0C3F81080C3F8A080C3F8308059
:104800005E61C3F8A0604FF400365E61C3F8A0603B
:104810001066C2F8900050655062C2F88000166FB2
:1048200026F004061667566F26F004065667506099
:104830001566C2F8905055655562C2F88050106FE9
:1048400020F008001067506F20F008005067556096
:104850000B4DD5F8140140F03000C5F8140151613A
:10486000C2F8A0105166C2F890105165516209E07B
:1048700050140E4095DC4000000E0E4000100E401B
:1048800000020E40C2F88010116F21F01001116774
:10489000516F21F010015167C2F81090C2F8A0903A
:1048A000C2F83490C2F810C0C2F8A0C0C2F830C03C
:1048B0004FF400015961C3F8A0105966C3F8901075
:1048C00059655962C3F88010196F21F40001196706
:1048D000596F21F400015967C2F860E0C2F890E016
:1048E000C2F854E0C2F824E0C2F880E0116F21F46D
:1048F00000611167516F21F400615167C2F804E053
:104900001466C2F8904054655462C2F88040116F3A
:1049100021F480611167516F21F480615167546007
:104920001F66C3F890701F655F62C3F880701A6FCE
:1049300022F480721A675A6F22F480725A671F61DC
:10494000C3F8A0701F63BDE8F08700BF08B5034B34
:1049500053F8203003B1984708BD00BF6C10002009
:1049600010B582B0036B0193002400E00134172CD2
:1049700009D8064B53F82420019B1A42F6D0204652
:10498000034B9847F2E702B010BD00BFF04341006F
:104990004D49400000230360064A4260064A826097
:1049A0004FF48022C2600222027442748374C37482
:1049B000037570470000DC05808D5B00036C1943B4
:1049C0000164704710B58B7C23B34FF000434A68F5
:1049D0008C686400B2FBF4F2013A120292B2134303
:1049E0000A7C120602F0706213434A7C120702F03E
:1049F00040521343CA6813434360CB7C63B14FF00A
:104A000080730A7D52B90022134303640968054B81
:104A1000984710BD0023DAE70023F2E74FF4801235
:104A2000F2E700BFBD49400008B5036B13F0807F7B
:104A300001D0192008BD01230360064B98470023CD
:104A400004E00021044A42F823100133172BF8D95F
:104A5000002008BDC54940006C100020B1F1FF3FA7
:104A600004D0044B53F82130436270474FF0FF33BA
:104A700043627047F043410010B5084C44F82120D0
:104A8000074A4FF00054C2F880411B01DBB282F8A4
:104A90001D331460034B984710BD00BF6C100020FD
:104AA00000E100E05D4A400008B50248024B98472B
:104AB00008BD00BF008003406149400042F26663C8
:104AC00003FB00F008E000BF00BF00BF00BF00BF55
:104AD00000BF00BF00BF01380028F4D170470000BC
:104AE000124B1A68126802601A6853684360936830
:104AF0008360D368C3600E4B1B68D9680161196974
:104B00004161596981619969C161D9690162196A13
:104B10004162596A81629B6AC36213690363054BF0
:104B20001B68436353698363704700BFC41300204D
:104B30006C110020781100200D4B1A6892690260F8
:104B40001B68DB6943600B4B1B681A6882605A68FC
:104B5000C2609B680361002306E05A1D064951F8B4
:104B6000231040F822100133092BF6D9704700BFFB
:104B7000C41300206C110020E01000200A2308E07C
:104B800003F180420A3A044951F8231040F82210F8
:104B90000133182BF4D97047E0100020192308E0E6
:104BA00003F18042193A064951F8231040F82210C7
:104BB00001331F2BF4D9024BD3F88030C361704707
:104BC000E0100020FEE70000284B5B6A13F0010FA5
:104BD00005D0EFF30583042B01D004207047234B4D
:104BE0005B6A13F0020F05D0EFF30583052B01D0AC
:104BF000052070471D4B5B6A13F0080F05D0EFF3DB
:104C00000583062B01D006207047184B5B6A13F012
:104C1000800F05D0EFF305830B2B01D00B207047DD
:104C2000124B5B6A13F4807F05D0EFF305830C2BE6
:104C300001D00C2070470D4B5B6A13F4806F05D0D8
:104C4000EFF305830E2B01D00E207047074B5B6AF4
:104C500013F4006F05D0EFF305830F2B03D00F2063
:104C60007047002070470020704700BF00ED00E053
:104C700000230FE0114AD2F80412A3F12000012210
:104C80008240114205D0EFF3058203F110009042FB
:104C900013D10133312B0FD81F2BEBD8074AD2F891
:104CA000001201229A401142F3D0EFF3058203F182
:104CB00010009042EDD070470020704700E100E006
:104CC00010B5EFF308831C4613F0070F00D01C1F2C
:104CD000174B5B6813F0010F01D0B7EE000A154BBC
:104CE0005B6813F4006F15D0134A22F001026FF0D5
:104CF000060E002303F1807344F8043C44F8082CAA
:104D00000E4B44F80C3C203C84F3088884F309885B
:104D1000704710BD0A4B9847034628B1094A22F054
:104D200001026FF00E0EE5E7074B98470346F5E7E3
:104D300030EF00E000ED00E0E14D4000C54B4000E9
:104D4000C94B4000C14C4000714C4000064A93687A
:104D500023F07F4323F4706343F0254343F4E0637F
:104D60009360024B1360704700140E40080000A5CA
:104D7000024B1860024B1960704700BF641100209D
:104D8000C0130020014B1870704700BF110D0020A8
:104D9000C0F30800014B1880704700BFDC100020F2
:104DA00008B5024650B9084B0849196008495960CE
:104DB000002199601046074B984708BD024B0649F1
:104DC000196006495960F5E7FC01002098020020AF
:104DD000080200207DB04000E0000020F800002024
:104DE00070B564201B4B984700221B4B1A7062B6AB
:104DF00061B60120194B9847194B9847194B9847B2
:104E000007E01948194B98470028FAD0184B1B782F
:104E1000DBB9114B1B78002BFBD0154B1B7813B95A
:104E200000210D4A117010484D220270114A157868
:104E300045708370104E34682A46214604300F4B6B
:104E400098472C4434600020DEE7013B084A137089
:104E5000DFE700BFBD4A400070110020A14D4000B7
:104E60006DB740004D0541008013002089B040001F
:104E700068110020D4100020D8100020011A410031
:104E8000F8B505464F4B4FF0FF32C3F88020C3F80A
:104E90008420C3F88021C3F8842103F540635A6855
:104EA00042F020625A605A6A22F400425A62464B2B
:104EB0009A6D5A6C22F040625A645A6C42F0006259
:104EC0005A64424C4FF4804363634FF4006363635E
:104ED0004FF48073636302203D4EB0474FF0807300
:104EE00063630420B0473B4F01237B630420B0473A
:104EF00002237B6340236363374A136823F0010373
:104F00001360364B5A6F42F480725A675A6F42F4FC
:104F100000725A67324AD2F8143143F44063C2F83F
:104F20001431002383F311882E4B1D60EA6A12F0BE
:104F3000040F26D069682C4B19602B4B1B6820335B
:104F40002A490B6012F0100F1FD148330B60284D17
:104F50002846284B9847244B1F6807F12004403D02
:104F600007F1600E2E4620686168A268E3680FC6EC
:104F7000103435467445F5D13A6E1F4BC3F8802086
:104F800006E02968184B1960D7E71B481B4B984768
:104F9000144B1B689B6813F4007F03D0134A1368FB
:104FA00004331360164B1B7813B90322154B1A8078
:104FB000154BD96A154A11609A6A154B1A60154B40
:104FC0009847F8BD00E100E000000140000E0E40EF
:104FD000BD4A400000100E4010E000E000400440D8
:104FE00000020E406C110020C41300207811002034
:104FF00020110020F1524000E0100020E552400056
:10500000110D0020DC10002000ED00E0D010002089
:1050100074110020C14C40006FF0060E70477047BD
:1050200070B58AB00446402200218048804B9847E2
:1050300023782A3B2A2B39D8DFE813F02B003800DD
:1050400038003800380038003800380038003800A0
:105050003800380038003800380038003800380090
:10506000380038003800380038003800F000ED0013
:10507000380038003800880038008E0038003800CA
:105080003800C40038003800380038003D004D00BA
:10509000790066490B462A2203F8012B654A1068FD
:1050A000C1F801009188927999809A715F48624BAA
:1050B00098470AB070BD5D4B52221A705F4A127851
:1050C0005A705F4A12885A805E4A12685A605E4A75
:1050D00012689A60EAE7554B53221A7062785A7048
:1050E0006378032BE2D8DFE803F0020A121A574C68
:1050F0002046574B98473C2304F8013CD6E7534CD5
:105100002046544B98473C2304F8013CCEE74F4CD3
:105110002046514B98473C2304F8013CC6E74B4CD2
:1051200020464E4B9847202304F8013CBEE73F4CF5
:10513000542323704A4D102128684A4B9847C2B225
:1051400062702968A01C484B9847AFE7374B47224D
:105150001A7004225A70A9E7344B49221A706278F7
:105160005A7063784BB1012B10D0022B14D0032B53
:105170001BD02E4B5E609D6098E73C4E3C4D3D4BF6
:105180003D4A92E8030018601971F2E73B4E3C4D2E
:105190003C4A384B1A60ECE73B4E3C4D354B3C4AA1
:1051A00092E8030018609980E3E73A4E68463A4B6C
:1051B0009847009D35442F4B384A92E80300186009
:1051C0001971D6E72579637905EB0325A37905EBFA
:1051D0000345E37905EB0365314B1D6013484D230F
:1051E000037063784370A378837062782946043033
:1051F0001D4B9847A378002B3FF458AF627829499C
:105200000A70013B28490B701544254B1D60012293
:10521000264B1A704AE7264B984747E7254BBB2297
:105220001A601A225A60224B98473FE780130020E9
:10523000FD1B41005044410089B04000110D002089
:10524000DC100020D01000207411002084130020F6
:10525000E14A4000394B40007D4B40009D4B4000EF
:10526000C01300209D1F4100011A410010000020C2
:10527000E80C00208C13002058444100E80C00206A
:105280001C2400206273730020240020205400207E
:105290006044410020540020B11C4100684441009A
:1052A000D8100020D41000206811002070110020B8
:1052B0004D4D400090140E4072B671B6EFF303836B
:1052C000EFF30982EFF30881DFF814D02DE9FE4FE8
:1052D0006846FFF7D5FDBDE8FE4F8D4670470000DC
:1052E00080130020F1EE101AA0EC200A0160704734
:1052F000A0EC108A704700BF10B51720234CA047C0
:105300001820A047224B4FF480321A66C3F8902031
:105310005A655A62C3F88020196F11431967596F93
:1053200021F4803159675A6001225A66C3F89020EF
:105330005A655A62C3F88020196F11431967596F73
:1053400021F0010159675A60A3F5206340F212620F
:10535000DA644FF400621A600E4B0F4A5A60412221
:105360005A62052119600D4A5A644FF4F572DA65E4
:1053700000229A6519640A4B1A700A4B4FF4000216
:105380001A60702283F8172310BD00BF95DC40001F
:10539000000E0E40000001400406090001C4000A8E
:1053A000CC13002000E100E010B54FF40002124BD6
:1053B000C3F88020BFF34F8FBFF36F8F0F4B4FF4B5
:1053C00080321A66C3F890205A655A62C3F880206A
:1053D000196F21F480311967596F21F480315967B1
:1053E0001A601A61C3F8A0205A631720044CA04722
:1053F0001820A04710BD00BF00E100E0000E0E40E5
:10540000E9DC4000642800D964200F4AD36D03FB17
:1054100000F30E49A1FB03135B09936548B10A4BE6
:105420005A6C22F040625A645A6C42F080625A64AC
:1054300070471346526C22F040625A645A6C42F034
:1054400000625A64704700BF000001401F85EB51A5
:10545000014B1888704700BFD01300200F4B1B6A08
:1054600013F0010F06D000220D490A700D490A60A1
:105470000D490A6013F0400F0ED00122084B1A703C
:10548000064B9A69094BB3FBF2F3064A1360C3EB70
:1054900003139A00044B1A60704700BF00000140DC
:1054A000CC130020C8130020D01300201F1A0500C1
:1054B000014B1870704700BF00010020064B1B789D
:1054C00023B94FF40062054B1A6370474FF4006232
:1054D000024B5A63704700BF00010020000E0E40CF
:1054E000064B1B7823B94FF40062054B5A63704793
:1054F0004FF40062024B1A63704700BF00010020A6
:10550000000E0E402DE9F04186B00F461646984633
:10551000B8B9344B984704460025049598238DF874
:10552000043001238DF805308DF8065002238DF8E4
:10553000083005AB03938DF8075020462A4B984757
:105540000EE02A4B98470446E6E72046284B98474A
:10555000002044E09DF8153008F805300135EDB223
:10556000B54238D28DF814708DF8155000238DF89F
:105570000630322201A920461E4B9847A379DBB2A0
:10558000022B0BD020461C4B9847322201A9204603
:10559000184B9847A379DBB2022BD6D101238DF8A3
:1055A0000630322201A92046124B9847A379DBB27C
:1055B000022BCFD02046104B9847322201A920461B
:1055C0000C4B9847A379DBB2022BC3D02046084B83
:1055D0009847002003E02046054B9847012006B07D
:1055E000BDE8F08125054100317440002D054100E2
:1055F000457440005D7440000D7640002DE9F04197
:1056000086B00C4617469846D8B9264B98470546AB
:105610000026049698238DF8043001238DF8053078
:1056200002238DF8063003238DF8083005AB039371
:105630008DF807408DF8156028461B4B9847344677
:1056400005E01A4B98470546E2E70134E4B2BC4254
:1056500021D28DF8144018F804308DF8163032221B
:1056600001A92846124B98470646AB79DBB2022BBC
:10567000EBD028460F4B9847322201A928460C4B05
:1056800098470646AB79DBB2022BDED028460A4BA0
:105690009847002602E02846074B9847304606B058
:1056A000BDE8F08125054100317440002D05410021
:1056B0005D7440000D764000457440002DE9F043D4
:1056C00087B00C4690461F46DDF83890D8B9274B76
:1056D000984705460026049698238DF80430012348
:1056E0008DF8053002238DF8063003238DF808303D
:1056F00005AB03938DF807408DF8156028461C4BC9
:105700009847344605E01B4B98470546E2E70134CD
:10571000E4B2BC4223D204EB08038DF8143019F82C
:1057200004308DF81630322201A92846124B9847D2
:105730000646AB79DBB2022BE9D028460F4B9847DF
:10574000322201A928460C4B98470646AB79DBB2BA
:10575000022BDCD028460A4B9847002602E0284658
:10576000074B9847304607B0BDE8F0832505410058
:10577000317440002D0541005D7440000D764000FD
:1057800045744000F8B506460D461746344BAA222C
:105790001A7011225A700222F021324CA0470128BF
:1057A00001D00020F8BD2C0AEDB22D4B1C705D70AD
:1057B0009C70DD701C715D7100229A719022DA710B
:1057C00067B182221A72264B0922C2213046254F28
:1057D000B847012806D001280BD0F8BD0222204B83
:1057E0001A72F0E71E4B0922C22130461E4EB04706
:1057F000F1E71B4B1B789C4201D00020F8BD184BF1
:105800009B789C4201D00020F8BD154B1B799C422F
:1058100001D00020F8BD124B5B789D4201D00020E2
:10582000F8BD0F4BDB789D4201D00020F8BD0C4B3A
:105830005B799D420BD10A4B9B7953B9084BDB79BD
:10584000902B08D1064B1B7A022B06D1F8BD002005
:10585000F8BD0020F8BD0020F8BD0020BDE700BF66
:10586000D4130020FD5540000555400010B500221E
:10587000054B1A7029B91121034B0122034CA04793
:1058800010BD1021F8E700BFD4130020FD554000E3
:1058900010B50022054B1A7029B92821034B0122AB
:1058A000034CA04710BD2921F8E700BFD413002006
:1058B000FD55400070B506460A4CAA2323701123FB
:1058C000637023460222F021074DA847FF2323706F
:1058D000012800D070BD23460122C0213046A847D0
:1058E000F8E700BFD4130020FD55400010B539B9CA
:1058F0000022044B1A7001223621034CA04710BD30
:105900000322F6E7D4130020FD55400038B50546C4
:105910000C4BAA221A7012225A700222F0210A4C51
:10592000A047012801D0002038BD064B0322BF212B
:105930002846064CA047012801D0002038BD014B65
:10594000987838BDD4130020FD554000055540001F
:1059500038B50D46094B0E228421094CA047012879
:1059600001D0002038BD054B186859689A68286036
:105970006960AA609B89AB810E2038BDD4130020DA
:105980000555400010B50B462C227021014CA04754
:1059900010BD00BFFD5540002DE9F04184B000234B
:1059A0008DF80F300139052942D8DFE801F00705ED
:1059B000030C0E101F4D02E01F4D00E01F4D8046EE
:1059C000012000240FE01E4DF9E71E4DF7E71E4DA4
:1059D000F5E70DF10F03024640461C4EB0473C442C
:1059E000E4B20134E4B201280BD123462F5D47B164
:1059F000621CA95C012FECD902332B44781EC0B283
:105A0000E9E7012804D0012809D004B0BDE8F081FD
:105A10000F4B0222FF2140460C4CA047F3E70D4BF1
:105A200000930D230B22F92140460B4CA047ECE7D5
:105A30000020EAE7C4444100F445410074464100B7
:105A4000744441004845410098454100FD554000DF
:105A500070444100F8464100BD56400008B506219B
:105A6000014B984708BD00BF9959400010B5274920
:105A700000238B72CB720B7340F2DC528A8064225B
:105A8000CA800B8021F8083F0620214B98470B2045
:105A9000204B984780B90C201E4B984788B90022AC
:105AA0001A4B5A801C4B984701211C4B98470128E0
:105AB0000CD0164B987A10BD19490B20144B9847FF
:105AC000E9E718490C20124B9847E8E701220F4BF1
:105AD0009A72114B98470521134B9847034650B1D2
:105AE0000A4AD372002BE4D00B4B98470F4B9847D0
:105AF000064B5880DDE7084CA0470021074B98472C
:105B0000A0470321084B98470346E9E734140020D7
:105B1000A57D4000D97D40002D054100155C400069
:105B2000381400203A140020455E4000D55D400046
:105B3000014B987A704700BF3414002008B5224BFF
:105B40009B7A8BB9214A13781F490888204921F88C
:105B500013000133DBB213700F2B02D900221B4B51
:105B60001A7000231A4615E01A4B98471A4B9847AB
:105B7000154B1B89984203D80022134B1A80E1E78A
:105B8000C01A114B1880DDE7114931F813100A448F
:105B90000133DBB20F2BF7D912090B4B1B7B4BB137
:105BA00009498B88C9885B1A9A420CD80022064B97
:105BB0001A7308BD04498B88C9880B449A4202D3E2
:105BC0000122014B1A7308BD34140020120D00206D
:105BD000141400202D054100655D4000014B187B29
:105BE000704700BF34140020014B1888704700BF75
:105BF0003414002008B5014B984708BD155F4000DC
:105C000008B5024B9847024B984708BD2D05410047
:105C10001D5F400030B587B005460C4600238DF867
:105C2000073072228DF808208DF80B3001228DF894
:105C300009208DF80C200DF10702049202228DF844
:105C40000A200593434B9847322202A92846424B2B
:105C50009847002C43D1012402238DF80A30802379
:105C60008DF80B3001238DF807309C4244D08F23F0
:105C70008DF80B3003238DF80A30012C43D09DF8AA
:105C8000073003F0F00343F005038DF807300223DB
:105C90008DF80A30012C3DD0AA238DF80B3001235A
:105CA0008DF807309C423CD007238DF80730F9234C
:105CB0008DF80B30012C3BD005238DF80730802365
:105CC0008DF80B30012C3AD02846244B9847012CF4
:105CD0003CD00022224B1A70204607B030BDA823CA
:105CE0008DF80B3001238DF80730322202A92846A7
:105CF000194B98470446AFE7322202A92846164BB3
:105D000098470446B3E7322202A92846124B984727
:105D10000446B4E7322202A928460F4B98470446AE
:105D2000BAE7322202A928460B4B98470446BBE744
:105D3000322202A92846084B98470446BCE7322283
:105D400002A92846044B98470446BDE70122044BAC
:105D50001A70C1E7317440005D7440004574400022
:105D6000130D002030B587B004460023059301AB26
:105D7000049372238DF8083001238DF809309C2399
:105D80008DF80B3002238DF80C3003238DF80A3088
:105D90000C4B9847322202A920460B4B98470546E8
:105DA00020460A4B9847012D04D00020084B18705C
:105DB00007B030BD9DF804009DF8053000EB0320CE
:105DC00080B2F5E7317440005D74400045744000D6
:105DD000130D002030B587B004460023059301ABB6
:105DE000049372238DF8083001238DF80930C02305
:105DF0008DF80B3002238DF80C3003238DF80A3018
:105E00000C4B9847322202A920460B4B9847054677
:105E100020460A4B9847012D04D00020084B1870EB
:105E200007B030BD9DF804009DF8053000EB03205D
:105E300080B2F5E7317440005D7440004574400065
:105E4000130D0020F0B587B00646002305930DF131
:105E50000703049372238DF8083001238DF809306D
:105E6000D9228DF80B208DF80C3002238DF80A30E2
:105E70004901C9B241F010018DF80710214B984734
:105E8000322202A93046204B98470546D7238DF889
:105E90000B3021238DF8073001280BD030461B4BE7
:105EA0009847DC238DF80B3003238DF80A3000244B
:105EB000274608E0322202A93046134B9847054690
:105EC000ECE70134A4B2012D18D1BFB9092C15D8C3
:105ED00019200F4B984730460A4B9847322202A9A7
:105EE0003046094B984705463046084B98479DF881
:105EF000073013F0010FE4D00127E2E7384607B07E
:105F0000F0BD00BF317440005D7440004574400036
:105F1000D5F140000048704744140020A84BDB78BE
:105F2000032B00F24081A64B1B793F2B00F23D81F1
:105F3000A34B5B79072B00F23A81A14B9B79082B8D
:105F400000F237819E4B1B7A013BDBB2022B00F241
:105F500032819B4B5B7A032B00F22F81984B9B7A0B
:105F6000072B01D90020704710B586B004460023E6
:105F7000059372238DF8083001238DF809300DF157
:105F8000070204928DF80C308E4B984780238DF8D1
:105F90000B3003238DF80A30322202A920468A4BA7
:105FA0009847012817D1864B1B78D3B19DF807304D
:105FB00043F010038DF8073002238DF80A303222A7
:105FC00002A92046804B9847012811D020467F4BDC
:105FD0009847002003E020467C4B9847002006B0FD
:105FE00010BD9DF8073023F010038DF80730E3E76C
:105FF00082238DF80B30724B5B788DF8073032229C
:1060000002A92046704B9847012817D18D238DF89F
:106010000B3040238DF80730694B9B7813B1482330
:106020008DF80730322202A92046674B9847012895
:1060300009D02046654B98470020D0E72046634BA7
:1060400098470020CBE78E238DF80B305C4AD3783D
:106050009B01DBB2127902F03F0213438DF8073047
:10606000322202A92046584B9847012804D02046E6
:10607000564B98470020B2E78F238DF80B30504ADB
:1060800053795B01DBB2927902F00F0213438DF872
:106090000730322202A920464B4B9847012804D0F2
:1060A00020464A4B9847002099E7A9238DF80B30EA
:1060B000434BDB798DF80730322202A92046424B50
:1060C000984701280CD1AA238DF80B303C4B1B7A42
:1060D000022B18D0032B1AD0012B06D000207EE70C
:1060E00020463A4B9847002079E78DF80730322256
:1060F00002A92046344B984701280CD02046334B48
:10610000984700206BE702238DF80730EFE7032361
:106110008DF80730EBE7B3238DF80B30284B5B7A13
:1061200003F003038DF80730322202A92046264BE4
:106130009847012804D02046244B984700204EE77A
:10614000D9238DF80B3003238DF80A30322202A9AF
:1061500020461D4B9847012804D020461B4B9847EA
:1061600000203CE79DF8073003F0F80343F01003EC
:10617000134A927A02F0070213438DF80730022384
:106180008DF80A30322202A920460F4B9847012889
:1061900004D020460D4B9847002020E720460B4BAB
:1061A000984701201BE7002070470020704700201F
:1061B000704700207047002070470020704700BFE4
:1061C00044140020317440005D7440004574400068
:1061D00000FB01F0C0F3C71070470000F0B587B0B6
:1061E00004460E46234B9847002304938A238DF8D8
:1061F000043001238DF805308DF808300DF11703B8
:10620000039334278DF8077002238DF80630337816
:106210008DF81730322201A92046174DA8478DF876
:10622000077033788DF81730322201A92046A8472D
:106230008DF8077033788DF81730322201A9204687
:10624000A84735238DF8073073788DF81730322240
:1062500001A92046A84736238DF80730B3788DF87A
:106260001730322201A92046A8472046034B984701
:1062700007B0F0BD317440005D74400045744000CB
:10628000F0B587B00446002505958A238DF80830BF
:1062900001268DF809608DF80C600DF10703049359
:1062A000254B984755238DF807308DF80B50022366
:1062B0008DF80A30322202A92046204DA847032338
:1062C0008DF807308DF80B60322202A92046A847CE
:1062D0008DF8076004238DF80B30322202A9204686
:1062E000A84707238DF8073030238DF80B30322272
:1062F00002A92046A8470F278DF8077031238DF893
:106300000B30322202A92046A8478DF807703226AA
:106310008DF80B60324602A92046A8478DF8077019
:1063200033238DF80B30324602A92046A847204679
:10633000034B984707B0F0BD317440005D744000D6
:1063400045744000F0B583B007460C46802900D95B
:1063500080240C4B1C700C4E214630780B4DA84706
:106360008DF8040021467078A8478DF80500214675
:10637000B078A8478DF8060001A93846044B984725
:1063800003B0F0BD01010020140D0020D1614000D8
:10639000DD61400010B5054B0C888A781C809A702E
:1063A000034B1978034B984710BD00BF140D002014
:1063B000010100204563400010B586B004468DF809
:1063C000081000230593E7238DF80B300DF1070328
:1063D000049301238DF80C308DF8093003238DF8D8
:1063E0000A30322202A90A4B9847012801D006B090
:1063F00010BD9DF8073043F001038DF807300223EC
:106400008DF80A30322202A92046014B9847EEE768
:106410005D74400010B586B004468DF80810002366
:1064200005930DF10703049301238DF80C308DF8CB
:10643000093006238DF80B3003238DF80A30322201
:1064400002A9224B98479DF8073063F07F038DF82F
:10645000073002238DF80A30012818D000238DF868
:1064600007300C238DF80B30012816D00D238DF842
:106470000B30012817D00E238DF80B30012818D0CF
:106480000F238DF80B30012819D006B010BD322231
:1064900002A920460D4B9847E0E7322202A9204688
:1064A0000A4B9847E2E7322202A92046074B984759
:1064B000E1E7322202A92046044B9847E0E7322266
:1064C00002A92046014B9847DFE700BF5D744000FA
:1064D00010B586B004468DF8081000230593E72315
:1064E0008DF80B300DF10703049301238DF80C3068
:1064F0008DF8093003238DF80A30322202A90A4BA5
:106500009847012801D006B010BD9DF8073023F050
:1065100001038DF8073002238DF80A30322202A9D8
:106520002046014B9847EEE75D74400070B5044685
:106530002022214B1A630A20204B98472046204BEB
:106540009847102120461F4EB0470546122120468D
:10655000B0470646012D0ED0012E12D0012D16D0C7
:10656000012E1AD02046184B9847012D1BD0012E22
:106570001DD0284670BD10212046144B9847054673
:10658000EAE712212046114B98470646E6E710211C
:1065900020460F4B98470546E2E7122120460C4B58
:1065A00098470646DEE701220A4B1A70DFE7012210
:1065B000094B1A70DDE700BF00100E40D5F1400016
:1065C00031744000B96340004574400015644000D8
:1065D000D1644000170D0020180D002010B1034BAE
:1065E00018787047024B1878704700BF180D0020CC
:1065F000170D002030B587B004460D4600220592E5
:10660000A8238DF8083001238DF809308DF80B2070
:106610000DF1070204928DF80C3002238DF80A3038
:10662000124B9847012D0ED0022D15D000238DF866
:106630000730322202A920460D4B984720460D4BC9
:10664000984707B030BD03238DF80730322202A9E6
:106650002046074B9847F1E702238DF80730322296
:1066600002A92046024B9847E8E700BF317440007A
:106670005D7440004574400030B587B072238DF8DA
:10668000003001238DF8013000238DF802308DF8A1
:10669000033008228DF8042004AA029203938DF897
:1066A0001000C0F307238DF81130C0F307438DF8B5
:1066B0001230000E8DF813008DF81410C1F307236B
:1066C0008DF81530C1F307438DF81630090E8DF89B
:1066D0001710084CA047084B9847A047322269463C
:1066E000064B98470546A047054B9847284607B0F4
:1066F00030BD00BF25054100317440005D7440008D
:106700004574400030B587B00D4672238DF80430D3
:1067100001238DF8053000238DF806308DF8073001
:1067200004228DF8082005AA039204938DF8140022
:10673000C0F307238DF81530C0F307438DF81630EA
:10674000000E8DF81700184CA047184B9847A0472B
:10675000322201A9164B98470446012808D0124B53
:106760009847144B9847012C0DD0204607B030BDF8
:1067700001238DF806300C4B9847322201A90C4BAF
:1067800098470446EBE79DF814309DF8152003EB7D
:1067900002239DF8162003EB02439DF8172003EB1C
:1067A00002632B60E1E700BF250541003174400022
:1067B0005D744000457440002DE9F04E82B0824681
:1067C000894693461BB11E46002501272FE001276D
:1067D000012F40D0012F49D0012F4DD0012F51D092
:1067E0004FF4000301932F4B98470446012F4FD1DC
:1067F000019B13F4000F4BD00A9920462A4B98476F
:1068000000284DD101A92948294B98470746EDE7B3
:10681000EA18B25C4FEAC30E02FA0EF211440133D9
:10682000DBB2A342F4D3012F0DD02544EDB22846AC
:106830004D45CDD2A9EB0504042C28BF0424E4B2B5
:1068400000231946EDE700F1201000F58070194B88
:1068500098470746E9E74FEA0A4101F4FE0101F5CE
:1068600000011248134B98470746B3E749461248C0
:10687000104B98470746AFE7594610480D4B9847CD
:106880000746ABE7F2210E480A4B98470746A7E7B1
:106890001FB9052002B0BDE8F08E9DF80700F9E7AA
:1068A0000620F7E7957A4000AD7A400010012000FD
:1068B000056740007966400018012000140120009F
:1068C000FC00200010B584B00A4B93E8030002904E
:1068D0008DF80C103223009302AB00220521012019
:1068E000054CA047034610B90121044A117018460F
:1068F00004B010BD08474100B9674000190D0020E1
:1069000070B5074D4FF480466E630A20054CA047D2
:106910002E6340F21310A047034B984770BD00BF91
:10692000000E0E40D5F14000C568400030B583B080
:106930000D46322300930023024604213120074CE8
:10694000A047044610B1204603B030BD2946044894
:10695000044B98470128F6D00524F4E7B9674000B6
:10696000200120000567400010B584B08DF80C10A0
:106970000B0A8DF80D300B0C8DF80E30090E8DF8CA
:106980000F103223009303AB024604212120024C56
:10699000A04704B010BD00BFB967400008B5044B64
:1069A0001B780BB1002008BD024B984708BD00BF03
:1069B000190D0020C56840002DE9F04383B059B19E
:1069C000012904D00124204603B0BDE8F08340F63D
:1069D0005D0740F6050503E040F2DD7740F285757E
:1069E00080464FF000094C4601E0002CEBD1BD423F
:1069F000E9D225F00306002CF7D101A93046164B49
:106A0000984704460028F0D1019B8DF80030C3F36D
:106A100007228DF80120C3F307428DF802201B0ED8
:106A20008DF80330E9B2F3B2C91AC9B2C1F1040357
:106A3000BE1B9E4228BF1E46042E28BF0426F6B267
:106A40003246694408EB0900044B984735444E44EC
:106A50005FFA86F9C9E700BF2D694000011A4100BD
:106A600028B1012801D000207047094800E00948FA
:106A700000B583B001A9084B984728B9019B13F4CE
:106A8000006F02D0012000E0002003B05DF804FB9D
:106A900040003500400031002D69400010B52DED5B
:106AA000028B82B0044601A93548364B984703460D
:106AB000F8B14BB3002B32D0002B3BD0DFED328A44
:106AC000002B49D09FED308A73B9DDED017AB8EE25
:106AD000677AC8EE077A9FED2D7A67EE877AFCEE2B
:106AE000E77A17EE902A6281184602B0BDEC028B5D
:106AF00010BD02A951F8043D23801B0C638024487B
:106B0000204B98470346D4E702A951F8043DA380DF
:106B10001B0CE3801F481B4B98470346CAE702A99A
:106B200051F8043D03F01F0323721B48154B98478F
:106B30000346C1E702A951F8043DC3F3094308EE37
:106B4000903AF8EE688A9FED158A68EE888A1448B4
:106B50000C4B98470346B3E702A951F8043DDBB25A
:106B600008EE103AB8EE488A28EE888ADFED077AF8
:106B700028EE278A0B48034B98470346A4E700BF3B
:106B8000300822002D694000000000000000C842CB
:106B900038082200540822000800200000401C464B
:106BA000040822001408220000B583B001A941F2B4
:106BB0003070094B9847034618B1184603B05DF88A
:106BC00004FB019921F00601019141F23070034B61
:106BD00098470346F1E700BF2D694000696940000E
:106BE00030B583B015460C4AA2FB01231B090F33B5
:106BF0000093002302461120084CA047044610B120
:106C0000204603B030BD29460548064B9847012869
:106C1000F6D00524F4E700BF1F85EB51B9674000AB
:106C2000200120000567400010B582B09623009334
:106C3000134602462020024CA04702B010BD00BF00
:106C4000B9674000072801D90120704710B584B00A
:106C50008DF80C0030238DF80D3041F2883300930D
:106C600003AB002202211420014CA04704B010BD48
:106C7000B967400010F0800F11D110B584B08DF8C5
:106C80000C0010238DF80D3041F28833009303ABD4
:106C9000002202211420034CA04704B010BD0120A3
:106CA000704700BFB9674000F0B583B0032832D801
:106CB000DFE800F00209050747F6F07604E0184E19
:106CC00002E0184E00E0184E002401273D4604E083
:106CD0009CB10F2C11D00134E4B20F2C13D801AAAF
:106CE0000121A019114B9847B8B9002DF0D09DF89B
:106CF0000430FF2BECD00025EAE79DF80430002B90
:106D0000E9D10027E7E717B11DB1002006E0002018
:106D100004E0012002E0002000E0002003B0F0BD0C
:106D2000F0FF0100F0FF0300F07F0200E16B400084
:106D300070B582B006460020114B984720B14FF441
:106D4000BE65002423460BE001200D4B984718B97F
:106D50000323184602B070BD0A4DF2E70134E4B2D5
:106D60000E2CF6D8002BF9D101AA01212819064BC7
:106D7000984703460028F1D19DF804203255EDE7ED
:106D8000A96C4000F0050200E16B400030B587B00F
:106D90001D201C4B98471C4C236C23F400132364C8
:106DA00068461A4B984769462046194B98476368CE
:106DB00023F47F436360636843F47F436360042389
:106DC00023610823236101232361626822F08F027B
:106DD0006260104A032120460F4DA847002120463B
:106DE0000E4B9847636813F0800F01D10822226090
:106DF0000B4B4FF000521A60702283F81D2307B02E
:106E000030BD00BF95DC4000008003409549400044
:106E1000294A4000456E4000794A4000BD49400083
:106E200000E100E00222014B1A607047008003403D
:106E3000024B1880024B1980704700BF02010020EE
:106E40000401002010B5064C206D80B2054B984718
:106E5000A06DE16D89B280B2034B984710BD00BFB1
:106E600000800340397F4000316E4000014B18889C
:106E7000704700BF02010020014B1888704700BF17
:106E8000040100200D4B1B8840F68962934205D90E
:106E90000B4A12883E2A01D803207047084A1288FC
:106EA00040F689618A4203D93E2B01D804207047FD
:106EB000934201D802207047012070470201002050
:106EC0000401002008B50120034B9847034B1860CC
:106ED00000B1012008BD00BF4DE840005014002063
:106EE00008B54FF0FF31024B1868024B984708BDB8
:106EF0005014002009EA400010B500231A46194634
:106F000002480068024CA04710BD00BF501400208A
:106F100015E74000154B98421BD003F5A03398426B
:106F200019D003F58043984217D0A3F54043984207
:106F300015D003F58043984213D0A3F5A0339842AF
:106F400011D003F56033984201D0322070471620EB
:106F5000704708207047092070470E2070471320A3
:106F60007047142070471520704700BF00C00040D4
:106F70004900B0FBF1F00338002302E04008013380
:106F8000DBB2FF28FAD8020202F47F4252FA80F004
:106F90001B0403F4E0231844704700002DE9F84374
:106FA000D0F80090037ADBB2012B00F0E68009F5FF
:106FB000C0650B7913B91846BDE8F88317460E462D
:106FC0000446012303720023C371E1606E4B9847AE
:106FD0008046B378022B08D07378012B18D0337811
:106FE0001B0403F4FE036B6050E07378012B09D09F
:106FF00033781B0403F4FE0303F580736B60F378AE
:10700000EB6043E033785B081B0403F58073F5E71E
:1070100033785B081B04E6E70323A3710023237284
:10702000237A002B00F0AB802B6A13F4807F53D1BE
:1070300013F4007F78D113F0400F7AD113F0800F52
:107040007CD113F0040F4BD1394640464F4B984743
:107050000028E9D00723A371002323724C4BC9F801
:1070600000363DE00423A37100232372D8E70523F3
:10707000A37100232372D3E70623A3710023237295
:10708000CEE739464046414B9847E8B93379E27933
:107090009B1A002BC4DD2B6A13F4807FBCD113F440
:1070A000007FDFD113F0400FE1D113F0800FE3D167
:1070B00013F0040FE5D0B168E379DBB25A1CD2B209
:1070C000E271CB5C6B63DCE70723A37100232372BF
:1070D0002F4BC9F80036A3E70323A37100232372C3
:1070E000237A002B4DD00223C9F800362B6A13F007
:1070F000010F28D113F4807F2BD113F4007F2DD101
:1071000013F0400F2FD113F0800F31D13946404694
:107110001E4B98470028E9D00723A3710023237250
:107120001B4AC9F8002646E70423A37100232372F3
:10713000D6E70523A37100232372D1E70623A371A9
:1071400000232372CCE7002323720223A3710123BF
:1071500031E70323A371002323722CE70423A371D7
:107160000023237227E70523A3710023237222E75C
:107170000623A371002323721DE700231BE70023CE
:1071800019E7002317E700BF957A4000AD7A400069
:10719000028000052DE9F84FD0F800B0037ADBB289
:1071A000012B00F0CE800BF5C0670B7913B91846A0
:1071B000BDE8F88F90460E46054601230372002372
:1071C000C371E960614B98478146B378032B14D0B3
:1071D0007378012B24D033781B0403F4FE0303F5EA
:1071E00080537B6096F804A0BAF1010F1ED00123F2
:1071F000CBF800364FF0000A64E07378012B09D019
:1072000033781B0403F4FE0303F588537B60F378A3
:10721000FB60E7E733785B081B0403F58853F5E769
:1072200033785B081B0403F58053DAE70323CBF8BC
:10723000003647E00323AB7100232B722B7A002B1F
:1072400000F081803B6A13F0010F60D113F4807F5E
:1072500063D113F4007F65D113F0400F67D113F0B1
:10726000800F69D141464846394B98470028E9D0FC
:107270000723AB7100232B72364ACBF8002696E722
:107280000423AB7100232B72D8E70523AB710023D5
:107290002B72D3E70623AB7100232B72CEE70723B3
:1072A000AB7100232B722B4BCBF80036C6E714F0E2
:1072B000020F07D0B168EB79DBB25A1CD2B2EA7187
:1072C0003A6BCA54EB79DBB232799342B6D23C6A5C
:1072D00014F4807FAED114F4007FD1D114F0400FAC
:1072E000D3D114F0800FD5D141464846184B98476A
:1072F0000028D4D1BAF1000FD9D13379EA799B1A99
:10730000012BD4D102233B604FF0010ACFE70023C9
:107310002B720223AB71012349E70323AB710023D6
:107320002B7244E70423AB7100232B723FE7052344
:10733000AB7100232B723AE70623AB7100232B724B
:1073400035E7002333E7002331E700BF957A40009B
:10735000AD7A4000028000052DE9F04106468846DE
:10736000046820461B4B9847312801D9BDE8F081BD
:107370000546194B9847032323602423C4F800369D
:1073800041461648164B9847C4F81006002333723E
:107390000123B3716BB2002B07DB5A0905F01F0004
:1073A000012181400F4840F82210002B0BDB03F134
:1073B000604303F56143202283F8002301200A4B38
:1073C00098473061D2E705F00F05084B20225A5547
:1073D000F4E700BF156F400095DC40000000DC05BD
:1073E000716F400000E100E04DE8400014ED00E066
:1073F00008B500680B4B9847312811D843B2002BD1
:107400000CDB5B0900F01F0101228A402033064992
:1074100041F82320BFF34F8FBFF36F8F034B984783
:1074200008BD00BF156F400000E100E0E9DC40004E
:1074300008B54FF0FF310069014B9847C0B208BD55
:1074400009EA400010B500231A4619460069024CAB
:10745000A047C0B210BD00BF15E7400008B5837952
:1074600063B18B78032B0BD8DFE803F0020502052C
:10747000044B984708BD044B984708BD002008BD41
:10748000002008BD9D6F40009571400080797047D5
:10749000F8B50646036803F5C064256AC76815F0A9
:1074A000040F0BD0E26A12F0040F07D0BA78002A5A
:1074B0004DD0022A4BD0BA78032A5ED015F0020FC5
:1074C00008D0E26A12F0020F04D0BA78012A73D011
:1074D000032A71D015F4807F0DD0E36A13F4807F06
:1074E00009D040F20733A362002333720323B37140
:1074F000FB6803B1984715F4007F0DD0E36A13F4DD
:10750000007F09D040F20733A362002333720423C3
:10751000B371FB6803B1984715F0010F16D0E36A09
:1075200013F0010F12D0BB780BB1022B09D140F23E
:107530000533A362002333720223B371FB6803B1E6
:107540009847BB78012B54D0032B52D0F8BDF27969
:10755000D2B239798A4208D2B868F279D2B2511CD3
:10756000C9B2F171825C6263A5E70222C3F800260A
:10757000012262620422A2629DE77A78012A11D078
:107580003A78120402F4FE0202F5805262603A79FF
:10759000012A0DD00122C3F800260422A262022291
:1075A00062628BE73A785208120402F58052EDE7E6
:1075B0000322C3F80026F0E7B868F279D2B2511C72
:1075C000C9B2F171216B8154F179C9B23A79013AAA
:1075D00091420AD0F379DBB23A7993427FF47AAFE1
:1075E000012363620223A36274E70222C3F8002628
:1075F000F0E740F20333A362002333720223B37136
:10760000FB68002BA2D09847A0E7000070B4056883
:1076100005F5C0660379202B0BD9A3F12001CBB26D
:107620001A4C0121994021602165216121630022CA
:1076300011E0174CF5E701339BB2B3F52F7FFAD376
:107640006163002301E001339BB2B3F52F7FFAD3CE
:1076500021630132D2B2092A01D80023EDE761612A
:10766000616032698023C5F80036002301E00133F0
:107670009BB2B3F52F7FFAD332612423C5F80036CD
:10768000002303720123837170BC704700100E4009
:10769000000E0E4030B591B000238DF835308DF8D6
:1076A00036308DF837308DF839308DF83A30ADF806
:1076B0003E300F238DF834300223ADF83C300124E6
:1076C0008DF838400DAA0B4907A80B4DA8470DAA05
:1076D0000A4901A8A8471023079A1360019A13606A
:1076E000074B1C70074B1C7045F6FF72064B1A8047
:1076F00011B030BD00C002407DD740000000034003
:107700001C0D002034160020FE16002042B110B4DB
:1077100020B119B1034B586099605A805DF8044B51
:10772000704700BF1C0D0020154B1B783BB3144B5A
:107730005B8823B3124A52680AB311498968F1B1D0
:10774000F0B583B0009201930E4D6A466946284613
:107750000D4FB8474FF480362E62094B9B6800935B
:107760000A4C6A4669462046B847266201212846E7
:10777000074DA84701212046A84703B0F0BD704738
:107780001C0D002000C10240B9D64000000103409A
:10779000D1D640000223034A136202F580421362ED
:1077A000704700BF00C1024010B58CB00A4B98472B
:1077B000069A136823F010031360009A136823F0ED
:1077C000100313600D20054CA0471220A047002293
:1077D000034B1A700CB010BD95774000E9DC4000F7
:1077E0001C0D0020064B1B783BB1054B5888054B00
:1077F000D3F80431C01A80B270470020704700BF30
:107800001C0D002000C00240094AD36D23F4FF4341
:1078100023F07F03C0F30E000343D36502F58042DB
:10782000D36D23F4FF4323F07F031843D0657047E3
:1078300000C00240014B1880704700BFFE160020B8
:10784000014B1870704700BF341600200048704785
:1078500000170020004870475414002070477047FC
:107860002DE9F8434F4B984705464F4B9847044640
:107870007FE0A0EB070E1FFA8EFE0EF1F00E1FFA4E
:107880008EFE85E03121002308E02F21FBE74748E9
:107890000078C0B2012831D001339BB2994259D946
:1078A000DA1992B2EF2A01D9F03A92B23F48007841
:1078B0000028ECD13E48B0F9000035F9126006FB13
:1078C00000F6F6134FEA8308DFF8ECC00CF82360EB
:1078D00008F10109C6F307260CF8096034F91220F3
:1078E00000FB02F2D21308F102000CF8002008F1AC
:1078F0000308C2F307220CF80820CDE735F912007F
:1079000034F91220024402EBD272521012F5004FE9
:1079100005DBB2F5004F03DB47F6FF7200E0254AB6
:107920002348B0F9000012B202FB00F2D213980013
:107930005FFA82FC204E06F823C000F10108C2F372
:10794000072206F8082000F1020806F808C00330F4
:107950003254A1E7194BA3F800E07744BFB2184BAB
:107960001F80EF2F01D9F03F1F8089001248154B6F
:1079700098474FF0FF310120134B9847134B98471E
:107980000F4B1F88B842FFF474AFC01B1FFA80FE74
:10799000BEF1300F3FF676AFBEF12F0F7FF675AF19
:1079A000302170E74D7840005578400034160020B3
:1079B000FE1600200080FFFF38160020FC16002075
:1079C000280D00202D454000E1F64000E5774000FD
:1079D000F8B5084C4FF4804666630A20064DA84768
:1079E000402767630A20A84727630A20A847266321
:1079F000F8BD00BF000E0E40D5F14000F8B578B9D3
:107A0000114D4FF480736B630220104CA0474FF070
:107A100080736B630420A04701220D4B5A63F8BDAD
:107A2000094E4FF480737363094F02253D63284666
:107A3000064CA04701233B630420A0474FF080730E
:107A400033632846A047F8BD000E0E40D5F1400034
:107A500000100E4010B5084C4FF4804363630020C3
:107A6000064B98470220064B98470222054B5A6363
:107A70004023636310BD00BF000E0E40FD7940003F
:107A8000D5F1400000100E400322014B1A607047F0
:107A900030140E40044B986801E0034B9868024B89
:107AA0009B689842F9D1704730140E4010B584B0ED
:107AB00001900C46064B98470390039B019A9B1A32
:107AC000A34202D2002004B010BD0120FBE700BF9A
:107AD000957A400030B585B01E4B1B68002B31D025
:107AE0001D4B98474FF0FF311A4B18681B4B9847B6
:107AF000EFF31083B3FA83F35B09039372B6BFF31A
:107B00005F8F0022164B1A70039D80230093154B44
:107B1000152214211448154CA04704462DB101220A
:107B20000F4B1A70BFF35F8F62B600231A461946D7
:107B3000084800680E4DA8470E4B984744B10020F6
:107B400005B030BD01200C4B9847024B1860C7E7C9
:107B50000120F5E72C0D0020E16E400009EA40000D
:107B60002F030020E0180020000A0E401100002022
:107B700015E74000F96E40004DE8400010B5074B96
:107B80009847002213210648064B98470446064BA7
:107B90009847B4FA84F0400910BD00BFE16E400080
:107BA000000A0E40F5D94000F96E400038B5114B7F
:107BB0009847EFF3108404B972B6002308E09A00E6
:107BC00002F580020C4951F82310116001339BB279
:107BD0007F2BF4D9002212210848094B9847C5B2DF
:107BE00004B962B6074B98470DB1002038BD01209B
:107BF00038BD00BFE16E4000E0180020000A0E40D2
:107C0000F5D94000F96E400010B400240EE04000A9
:107C100080F00700C0B20133DBB2072B05D810F0AB
:107C2000800FF4D14000C0B2F5E70134944204D291
:107C300011F8013B58400023EFE75DF8044B704713
:107C400070B50646002501E02C44A5B2B5F5007FCD
:107C500015D20E4BE918EA5CFF2A14D06B1C0B48B6
:107C60001B5C0333DCB2B242EED1621EFF20084B34
:107C700098472B19074A9B5C9842E5D101E04FF6E3
:107C8000FF75284670BD4FF6FF75FAE7E018002033
:107C9000097C4000DF18002008B5094B1B781BB198
:107CA000022B01D0074808BD074B9847012804D193
:107CB0000122034B1A70034808BD002008BD00BF15
:107CC000300D0020E0180020D57A400008B5094B9F
:107CD0001B781BB1022B01D0074808BD074B984702
:107CE000012804D10122034B1A70034808BD00206B
:107CF00008BD00BF300D0020E0180020D57A4000FC
:107D0000A8B108B50346B1F5007F12D28818B0F5C6
:107D1000007F01D9002008BD08461946064B1844CB
:107D2000064B98470222064B1A70012008BD00201E
:107D30007047002008BD00BFE0180020011A410074
:107D4000300D002008B5064B1B78022B01D0002017
:107D500008BD044B98470128FAD1034B984708BD4A
:107D6000300D00207D7B4000AD7B400090B110B510
:107D700004460268094B9A4201D0002010BD9A22A5
:107D80000146FF20064B984794F89A30984203D05A
:107D9000002010BD00207047012010BD5FE1AD5AEA
:107DA000097C400010B50C46084B9847B0F5007FA1
:107DB00001D3002010BD811C054B5A1C125C1944D4
:107DC0002046044B9847012010BD00BF417C400075
:107DD000E0180020011A410008B5044B9847B0F59F
:107DE000007F01D2012008BD002008BD417C400079
:107DF00008B5054B9847B0F5007F02D2034BC05C35
:107E000008BD002008BD00BF417C4000E1180020F3
:107E1000FF292FD02DE9F843D61CF6B28419B4F50A
:107E2000007F03D94FF6FF70BDE8F88317460C4674
:107E300005460221114A1170DFF84C8000EB080959
:107E400000F80840421C02F8087008443A461946F7
:107E500040440B4B98477C190234721E4946FF2060
:107E6000084B984708F80400E81980B2033080B244
:107E7000BDE8F8834FF6FF70704700BF300D00205B
:107E8000011A4100097C4000E018002010B5A8B09C
:107E9000224B98470446224B984708B928B010BD9A
:107EA0009B22214601A81F4B98474FF40072FF21E7
:107EB0001D481E4B984702AB1022012100201C4C8C
:107EC000A0474FF6FF73984203D026AB032202214E
:107ED000A0474FF6FF73984205D00DF19B03012296
:107EE0000321134CA0474FF6FF73984204D027ABF1
:107EF000012204210E4CA0474FF6FF73984205D093
:107F00000DF19D0301220521094CA0474FF6FF7397
:107F10009842C3D0074B9847C0E700BF997C400008
:107F20006D7D4000011A4100E0180020FD1B41005A
:107F3000117E4000457D4000044B1880044A1378B0
:107F4000591C1170034A22F813007047E41C0020EA
:107F5000310D0020E41A002008B5194B1B8807EEEC
:107F6000903AF8EE677A9FED177A67EE877A164BAC
:107F7000C3ED007AF7EE006A76EEE76A87EEA67A3E
:107F8000DFED126A67EE267A114BC3ED007A86EEBA
:107F9000A77A17EE100A0F4B9847DFED0F7A07EE1E
:107FA000100A27EE277ADFED0D7A77EEC77ADFED3C
:107FB0000C6A86EEA77A0B4B83ED007A08BD00BFF2
:107FC000E41C002001088039E01A002000401C4613
:107FD000EC1C0020950541003313954300F05745F4
:107FE000C47D7B49E81C0020BFF35F8F024B1868FB
:107FF000BFF35F8F704700BFE81C002068B90F4ACD
:108000001368B3F1FF3F0AD00320B3F1333F0ED022
:1080100013B9536803B902207047094AF0E7516861
:10802000B1F1FF3F01D00320EFE70020EDE75168F9
:10803000B1F1333FECD10120EAE700BF00C04700B7
:1080400000E0470018B101280FD0022070470B480C
:1080500041F6F87383B130B4C518C4588C4206D0C9
:10806000083B002BF8D1012004E00548F0E76B68DD
:108070001360002030BC70470120704700C04700EB
:1080800000E0470070B505460020124CA0470646A8
:108090000120A0471DB1012D12D0022070BD022881
:1080A00003D0022E07D0022070BD012E01D0012086
:1080B00070BD002070BD012801D0002070BD70BDD2
:1080C000022E05D0022801D0022070BD012070BD13
:1080D000002070BDFD7F4000F8B504460F461646EF
:1080E000450A094B984704F4FE7000F580031F60B1
:1080F0005E602A4601210548054B98470446054B1A
:1081000098472046F8BD00BFE16E4000000A0E40CF
:10811000F5D94000F96E4000012909D002290CD19F
:10812000002108B538B906480A46064B984708BDED
:108130004FF03331F5E70448F6E70120704700BF00
:1081400000C04700D980400000E0470038B518B1B2
:1081500001280DD0022038BD0A4C0823B3F5005F7A
:108160000ED2E018E558B5F1FF3F03D00833F5E72C
:10817000054CF2E7054B984708B1022038BD38BDE1
:10818000012038BD00C0470000E04700D980400012
:1081900010B568B140F2F234074B984722460721E8
:1081A0000648074B98470446064B9847204610BDA3
:1081B00040F2E234F0E700BFE16E4000000A0E40FA
:1081C000F5D94000F96E400070B582B000230193EC
:1081D000044668B90125184E18490023B3F5006F0D
:1081E00028D251F82320B2F1FF3F05D10133F5E742
:1081F0000025134E1349F0E72046134B98470446D9
:1082000010B1204602B070BD01AA314628460F4B7E
:10821000984748B9019A0132314628460C4B984795
:108220000028EED00124ECE7012231462846084B15
:108230009847F5E70024E4E70120FFFF00C047006E
:108240000220FFFF00E04700918140004580400090
:108250004D81400070B582B005460E460846294B58
:108260009847012806D001213046274B98470446FD
:10827000002844D1002400E00134244B1B689C42B8
:1082800015D201AA224B53F824102846214B9847B7
:10829000022833D00028EFD1019A1D4B53F8241047
:1082A00030461D4B98470028E6D0012427E0284699
:1082B0001A4B9847044610BB02213046124B984790
:1082C0000446E0B995B9164D02AA002342F8083DCC
:1082D000294630460F4B984750B9009A013229463B
:1082E00030460D4B984750B1012408E00D4DEBE7A7
:1082F000012229463046084B9847F4E701242046DE
:1083000002B070BDFD7F40001981400020010020B7
:1083100008010020458040004D81400091814000CF
:108320000120FFFF0220FFFF10B50020104B9847EF
:10833000044608B1204610BD01200D4B9847044665
:108340000028F7D102210B4B984704460028F1D1B1
:1083500001220949094B984708B10124EAE70122A3
:108360000749064B98470028E4D00124E2E700BF04
:1083700091814000198140000120FFFF4D814000A4
:108380000220FFFF38B50120384B9847384B186062
:10839000002869D00020374DA84704460120A8478F
:1083A000012C2BD05CB1022C46D0334B98470346AE
:1083B00018B90122314B1A700023184638BD012824
:1083C00008D0022814D100202D4B984703460028DE
:1083D000EFD0F2E700202A4B984703460028ECD163
:1083E00002210120274B984703460028E1D0E4E70B
:1083F000214B984703460028DBD0DEE748B102282E
:1084000014D100210120204B984703460028D0D0EA
:10841000D3E701201A4B984703460028CDD102210B
:10842000184B984703460028C3D0C6E7124B98471D
:1084300003460028BDD0C0E738B102280CD10E4B4E
:10844000984703460028B4D0B7E701200C4B984763
:1084500003460028ADD0B0E7012100200A4B984721
:1084600003460028A5D0A8E70123A6E74DE8400071
:10847000F01C0020FD7F400029834000320D0020C9
:10848000C9814000198140005582400070B50E4BF3
:108490001B7813B90324204670BD0D4604460B4ECD
:1084A0004FF0FF3130680A4B98470120094B98473D
:1084B0002A462146084B9847044600231A46194687
:1084C0003068064DA847E6E7320D0020F01C00207A
:1084D00009EA4000858040004580400015E74000E3
:1084E000F8B5194B1B7813B903242046F8BD0E4686
:1084F00005464FF0FF31154B1868154B9847002083
:10850000144B9847074632462946134B9847044672
:10851000012807D000231A4619460C4800680F4D61
:10852000A847E2E7B7FA87F46409214638460C4BBE
:10853000984708B10224EDE7324629462046064B0B
:1085400098470446E6E700BF320D0020F01C0020EB
:1085500009EA4000858040004D81400015E7400059
:108560005582400008B50020094B984708B101200A
:1085700008BD2022074B5A630A20074B9847074B38
:108580009847074B9847012801D0002008BD08BD37
:10859000DD65400000100E40D5F140002D05410082
:1085A0002D65400030B587B0174B984704468A23A5
:1085B0008DF808300025059501238DF809308DF8D8
:1085C0000C300DF107030493104B98478DF80B50B6
:1085D00003238DF80A30322202A920460C4B98471B
:1085E00020460C4B9847022806D0002520460A4B0F
:1085F0009847284607B030BD9DF80730092B01D0B9
:108600000025F3E70125F1E72D0541003174400015
:108610005D7440008D7440004574400030B587B0F3
:108620001A4B9847044600220592A8238DF808307B
:1086300001238DF809308DF80B2001AA0492022243
:108640008DF80C208DF80A30114B9847322202A980
:108650002046104B984720460F4B9847022806D0DB
:10866000002520460D4B9847284607B030BD9DF8A1
:10867000043033B99DF8053013F0F80F03D000250E
:10868000EFE70025EDE70125EBE700BF25054100F9
:10869000317440005D7440008D74400045744000AA
:1086A00008B5034B984708B1002008BD012008BD5C
:1086B0009D69400030B587B0184B984704460023A9
:1086C000059372238DF8083001238DF8093092222A
:1086D0008DF80B200DF1070204928DF80C30032366
:1086E0008DF80A300E4B9847322202A920460D4BD6
:1086F000984720460C4B9847022806D00025204674
:108700000A4B9847284607B030BD9DF80730442BE8
:1087100001D00025F3E70125F1E700BF2D05410059
:10872000317440005D7440008D7440004574400019
:1087300070B586B0002832D11C4B984704460025FE
:10874000059598238DF8083001268DF809608DF87D
:108750000A5002238DF80C3001AB04938DF80B50B6
:108760002046134B984736238DF804308DF805507A
:10877000322202A920460F4DA8478DF80A60322206
:1087800002A92046A84720460B4B984702280AD04A
:1087900000252046094B9847284606B070BD084B77
:1087A00098470446CBE73546F3E700BF250541006F
:1087B000317440005D7440008D7440004574400089
:1087C0002D05410038B50020064CA0470546012084
:1087D000A047012D01D0002038BD0128FCD0002089
:1087E00038BD00BF318740002DE9F0473D4BD3F83D
:1087F000588019203C4B98474FF496703B4B984754
:10880000002409E03A4B98473A4B23F81400032020
:10881000364B98470134E4B21F2CF3D9364B9847B6
:10882000824600263746354634463FE0314931F826
:1088300013100A440133DBB21F2BF7D94FEA521948
:10884000B9F10A0F17D92A4B9847631CDBB2294AA2
:1088500022F814001F2B1DD81C46A9F1FA039842D8
:108860001AD309F1FA02904225D80135EDB2202D34
:1088700013D9012611E0B8F1000F05D0194BC3F848
:1088800058800020BDE8F0870020174B9847002053
:10889000BDE8F0870024E0E700250320134B98474C
:1088A0004FF47A615046154B984707462FB926B9C1
:1088B00000231A46C0E70025EFE7B8F1000F07D004
:1088C000084BC3F8588057B936B10120BDE8F0878E
:1088D0000020054B9847F6E70020BDE8F087002010
:1088E000BDE8F0870000014005544000D5F140008C
:1088F00051544000F41C0020957A4000AD7A4000AD
:108900000048704710474100072070472DE9F843A1
:1089100005460E4617460A469C211E4B98470446BC
:10892000451B40B1731B052B05D94378552B07D048
:1089300010237B7001E000237B702046BDE8F883A4
:1089400090F80280C37888EA0303FF2B02D011233A
:108950007B70F2E790F80490437909EB03291FFA42
:1089600089F9B9F13A0F06D84D440635AE4205D221
:1089700000237B70E1E712237B70DEE74A46811D0E
:10898000381D054B9847A7F8029087F8008001230F
:108990007B70D2E701194100011A410010B55388DC
:1089A0009C1D8C4219D83A2B01D9002010BD1146CC
:1089B0009C23037055234370137883701378DB4333
:1089C000C3709378037153881B0A43715288043132
:1089D0000630034B9847012010BD002010BD00BF9A
:1089E000011A410070B582B004460378253B332B51
:1089F00000F21982DFE813F0450017021702170290
:108A00001702340017021702170217021702170283
:108A1000170217021702170217021702170217028E
:108A2000170217021702170217021702170217027E
:108A30003E0117021702FA00170217021702170267
:108A40001702BA0113015C0017021702170217027E
:108A500017021702170265017900CB00A600E30098
:108A60009C4C2A2323709C4DA84760809B4B9847C1
:108A70000646A84702463146201D994B984702B04A
:108A800070BD0120974B984780B2924B588010B927
:108A900045221A70F3E794490120944B984718B186
:108AA00025228C4B1A70EAE745228A4B1A70E6E7BA
:108AB0004388032B05D0874B00225A8045221A7029
:108AC000DDE703798DF8043043798DF8053083793B
:108AD0008DF80630864B984701A9864B98477D4B09
:108AE00000225A8024221A70C9E74388012B05D03E
:108AF000784B00225A8045221A70C0E703790F2B69
:108B000005D9744B00225A8045221A70B7E77A4B78
:108B10009847704A5523137020235380237900EB24
:108B20004310066845688468C16856609560D460E3
:108B30001161066945698469C16956619561D461AD
:108B400011629CE74388212B05D0624B00225A809A
:108B500045221A7093E701790F2905D95D4B002250
:108B60005A8045221A708AE7202249010530634B5A
:108B70009847012805D0574B00225A8045221A7089
:108B80007DE7544B00225A8024221A7077E74388ED
:108B90002BB1504B00225A8045221A706FE7584B78
:108BA0009847012805D04B4B00225A8045221A7065
:108BB00065E7484B00225A8024221A705FE74388F9
:108BC0002BB1444B00225A8045221A7057E74D4B77
:108BD000984728B93F4B00225A8024221A704EE74A
:108BE0003C4B00225A8045221A7048E74388012BEB
:108BF00005D0384B00225A8045221A703FE7007991
:108C0000414B984728B9334B00225A8024221A70CE
:108C100035E7304B00225A8045221A702FE74388EF
:108C2000082B05D02B4B00225A8045221A7026E7CC
:108C30000379427903EB0223827903EB0243C07983
:108C4000217A627A01EB0221A27A01EB0241E47AF5
:108C500001AA01EB046103EB00602C4B984700284C
:108C60007FF40DAF1B4B019A5A604B221A700422FD
:108C70005A8004E74388063B9BB21F2B05D9154B4E
:108C800000225A8045221A70F9E64379807903EB75
:108C90000023E07903EB0043207A04F109022179F3
:108CA00003EB00601A4B984728B90A4B00225A8000
:108CB00024221A70E3E6074B00225A8045221A70DC
:108CC000DDE6438833B3034B00225A8045221A70F5
:108CD000D5E600BF341D002009894000018940000D
:108CE000011A4100F17D4000381D0020A57D4000A3
:108CF0002D05410095634000CD7C4000017D400082
:108D0000457D40009D694000456C4000E16B40009E
:108D1000296C40000020474B1871474B984720B101
:108D2000444A137943F0010313710120424B9847E1
:108D300020B1404A137943F00203137102203E4BE5
:108D4000984720B13B4A137943F004031371032081
:108D5000394B984720B1374A137943F00803137110
:108D6000344B01225A8054221A7088E64388012B22
:108D700005D0304B00225A8045221A707FE60379D5
:108D8000463B102B49D8DFE803F03F4809484848E4
:108D9000124848362D48481B48482400274B98471E
:108DA000244B18714A221A7001225A8067E6244B1C
:108DB0009847204B18714A221A7001225A805EE6A9
:108DC000204B98471B4B18714A221A7001225A8077
:108DD00055E61D4B9847174B18714A221A7001220D
:108DE0005A804CE6194B9847124B18714A221A7058
:108DF00001225A8043E6164B98470E4B18714A22BF
:108E00001A7001225A803AE6124B9847094B1871A2
:108E10004A221A7001225A8031E6064B45221A7006
:108E200000225A802BE6034B00225A8045221A70FA
:108E300025E600BF341D0020A96C40006585400078
:108E4000A58540001D864000A1864000B5864000F3
:108E5000C5874000E987400000487047341D002066
:108E6000F0B583B0EFF31083B3FA83F35B0901939A
:108E700072B6BFF35F8F0022364B1A70019E364BDD
:108E80001B68364A15682B447F2B2AD8324B1C6846
:108E90002246334933482844334B98472C442F4BC0
:108EA0001C6000222C4B1A602EB10122294B1A7033
:108EB000BFF35F8F62B62D4A284B196829482C4BA7
:108EC00098470146D0B1274BC31A284842881A4414
:108ED000951D4478012C15D044BB802B1CD900244F
:108EE0002AE01D4A136814682C441B1B03F18004FC
:108EF000204A137843F001031370C9E70024174B8D
:108F00001C6019E01748154F3E68761B3246411920
:108F1000194B98473E600FE0104D2C68E41A22462A
:108F20001048154B98472C60002405E00133802B36
:108F300005D90024094B1C60204603B0F0BD094848
:108F4000064D2C68E41A2246C1180B4B98472C603A
:108F50000024F1E72F0300207C2000208C2000203B
:108F6000D42000207C1F0020011A41009020002006
:108F70000D89400088200020351B410010B50DE010
:108F8000144B195D1448154B98470134E4B2144B47
:108F90001B689C42F4D30022114B1A600120114B34
:108FA0009847114B98470128F8D11048104B984723
:108FB000104B98470246802106480F4B98470128DE
:108FC000ECD10C4B984743880633054A13600024C4
:108FD000DDE700BFFC1F0020008201407FDE400073
:108FE00084200020D5F14000618E400090200020B8
:108FF000E5894000598E40009D89400030B583B01E
:109000008024224600211C481C4DA84722460021EE
:109010001B48A84700231B4A13601B4A13601B4AC6
:1090200013701B4A10215166C2F8901051655162AD
:10903000C2F88010116F21F010011167516F21F0FB
:1090400010015167134A4FF400211160202182F86A
:1090500013130121104A9160104A01920093224695
:109060000F491048104CA047012802D00F48104B60
:10907000984703B030BD00BFD4200020FD1B410045
:10908000FC1F00207C20002084200020882000205D
:10909000000E0E4000E100E0008201408020002030
:1090A000184741007D8F400001EF400020474100FC
:1090B00055134100104B1B6913F0010F12D00E4BDA
:1090C0005B6913F0010F0DD00C4B1B687F2B0AD985
:1090D0000B4A137843F001031370074B9A69094B4D
:1090E00083F87F207047054A1368591C1160024AB3
:1090F0009169044AD1547047008201407C200020CD
:1091000088200020D4200020064A936823F07F4363
:1091100023F4706343F0254343F4E0639360024B10
:109120001360704700140E40080000A570B5064695
:109130000D46094B98470446002040B92946204671
:10914000064B984728B93046054B9847F5E701206C
:1091500070BD002070BD00BF957A4000AD7A400020
:1091600089B0400010B54FF47A722B4B1A8004E09E
:109170004022002129482A4B9847274B188880B263
:10918000284B9847254C2323237014236370264BC8
:109190009847C0F30F23A370E070244B9847C0F3A7
:1091A0000F2323716071224B9847C0F30F23A371E3
:1091B000E071204B9847C0F30F23237260721E4B5F
:1091C0009847C4F80A001D4B1B7807EE103AB8EE1A
:1091D000477A9FED1B6A27EE067ADFED1A6A37EEB3
:1091E000667A17EE103AC4F80E30174B1B7807EE6C
:1091F000903AF8EE677A67EE867A77EEE67A17EEBF
:10920000903AC4F81230114B98470028B0D0322160
:1092100020460F4B9847ABE7C8210020782100205B
:10922000FD1B4100D5F1400051544000E95B400076
:109230006D6E4000796E4000E97F4000F80100202B
:10924000B4C8363F6FDB4A42F90100204F054100A8
:109250002D914000F0B583B0402200219A489B4BED
:1092600098470BE29A4B98479A4B984711E2984BD4
:109270009847994BBB221A601A225A60954B98471F
:109280000AE291490B462A2203F8012B934A1068FF
:10929000C1F8010091889279104699809A71FEE197
:1092A00001208F4B984728B9874B45221A7002221C
:1092B0005A70F7E18449252301F8013B0120894BCD
:1092C0009847EFE10820864B984728B97E4B452206
:1092D0001A7002225A70E8E17B49262301F8013B0B
:1092E0000820804B9847E0E109207D4B984728B93A
:1092F000754B45221A7002225A70D9E172497E23B9
:1093000001F8013B0920774B9847D1E1C4F30723CB
:10931000032B09D8DFE803F0020B0406724807E0CC
:10932000724805E0724803E04FF0FF3000E07148FA
:10933000B0F1FF3F10D001A96F4B984730B9624B95
:109340005A221A70019AC3F80120B5E15E4B4522FA
:109350001A7002225A70AFE15B4B45221A7001224B
:109360005A70A9E1C4F30723032B09D8DFE803F0FF
:10937000020B04065C4807E05C4805E05C4803E03B
:109380004FF0FF3000E05B48B0F1FF3F0ED05B4B89
:1093900019685B4B984718B924224B4B1A708EE121
:1093A000494B45221A7003225A7088E1464B4522E8
:1093B0001A7001225A7082E12422434B1A7081E113
:1093C000414B45221A704F4A12785A707DE14E4B3C
:1093D0001B780F2B05D93C4B45221A7001225A707D
:1093E00076E14A4B9847384A55231370202353702F
:1093F000454B1B7800EB4310D0F800E047688668C7
:10940000C168C2F802E0C2F80670C2F80A60C2F889
:109410000E10D0F810E047698669C169C2F812E001
:10942000C2F81670C2F81A60C2F81E1050E1264B3E
:109430004B221A7004225A706A44354B1968354B16
:109440001868354B984720B91F4B019AC3F8022082
:1094500041E10022314B1A603DE11B4B54221A704E
:10946000002058702E4B984720B1174A537843F08C
:109470000103537001202A4B984720B1124A5378B8
:1094800043F0020353700220254B984720B10E4A47
:10949000537843F0040353700320214B984700286E
:1094A00000F01C81084A537843F00803537015E11B
:1094B0001C4B1878072837D9802841D0024B452209
:1094C0001A7001225A700CE1D0210020FD1B4100CE
:1094D000A90441000991400090140E4050444100FD
:1094E000F17D4000A57D40000110FFFF0310FFFF4C
:1094F0000410FFFF0210FFFF8D844000C4210020F4
:10950000E1844000CA210020C0210020CD7C400021
:10951000CC210020BC210020E16B4000D2210020A2
:10952000A96C4000542100207C4B984718B9242294
:109530007B4B1A70D5E07A4A452111705070D0E00B
:10954000784B187810F0800FB8D1774B984718B93E
:109550002422734B1A70C4E0714B45211970587066
:10956000BFE0724A724B1968724B1868724B984789
:1095700018B924226A4B1A70B6E0694B452119705C
:109580005870B1E066484E2300F8013B6B4B98479A
:10959000002800F0AC806A4B4FF020321A605A600D
:1095A0009A60C3F80B20A2E014F47F4F5C4E314662
:1095B0004FF05E0301F8023B14BF01200020614B15
:1095C00098477070002840F095804522327091E0F5
:1095D0004A22534B1A70C4F30723463B102B2DD855
:1095E000DFE803F0272C092C2C2C0E2C2C221D2C10
:1095F0002C132C2C1800544B9847494B58707CE086
:10960000524B9847464B587077E0514B9847444B24
:10961000587072E04F4B9847414B58706DE04E4B7D
:1096200098473F4B587068E04C4B98473C4B5870FC
:1096300063E04B4B98473A4B58705EE0384B4522FD
:109640001A7001225A7058E0464B98472422344B36
:109650001A7054E09A000232434951F8230030490D
:1096600050500133DBB20B2BF4D9404B9847002804
:109670004ED1402200212A483D4B98474FF0FF3100
:1096800001203C4B984704460028F7D043283FF47C
:10969000E9AD422C3FF4EBAD2A2C3FF4F2AD252C82
:1096A0003FF4FEAD262C3FF40DAE7E2C3FF41CAEF5
:1096B000E5B25A2D3FF42AAE7A2D3FF453AE242C56
:1096C0003FF47AAE452C3FF47BAE552C3FF47FAE91
:1096D0004B2C3FF4ACAE542C3FF4BFAE442C3FF4C3
:1096E000E7AE412C3FF43DAF4E2C3FF44BAF5E2D27
:1096F0003FF45AAF4A2D3FF46BAF3D2CA4D0732CEE
:10970000B3D1074B73221A7030225A700023AAE794
:1097100032210348184B9847ABE700BF456C400027
:10972000D0210020B8210020756C40005821002075
:10973000CC210020BC210020296C4000316D40006C
:10974000D12100205159400065854000A585400089
:109750001D864000A1864000B5864000C5874000B8
:10976000E98740003DA84000B42300204F05410098
:10977000FD1B4100E1F640002D91400010B5002393
:109780000322014602480068024CA04710BD00BFFA
:10979000340D002009F8400010B584B0002304AA5D
:1097A00042F8043D09490C68009203220146204614
:1097B000074CA047039B3BB14FF08052054B1A600A
:1097C000BFF34F8FBFF36F8F04B010BD340D002077
:1097D000B5F8400004ED00E010B582B00F4B0193E6
:1097E00001230093002380220D490E480E4CA04710
:1097F000012802D00D480E4B984700230193012207
:10980000009280220B490C48074CA047012802D047
:109810000A48074B984702B010BD00BF340D002026
:10982000404741005592400001EF40005047410041
:109830005513410080474100659140008C4741002D
:1098400070B584B0044603782A2B00F09580237805
:10985000252B00F095802378262B00F09580237827
:109860007E2B00F0958023785A2B00F0958023788A
:109870007A2B00F098802378532B00F0A780237870
:10988000472B00F0B0802378672B00F0BD80237851
:10989000462B00F0C4802378522B00F0C780237839
:1098A000502B00F0D78023785E2B00F0FB802378CC
:1098B000492B00F008812378432B00F0178123788F
:1098C000422B00F017812378552B00F01781237865
:1098D000572B00F01A812378562B00F0298123782A
:1098E0004C2B00F0328123784D2B00F042812378FD
:1098F0004B2B00F087812378542B00F09F81237835
:10990000442B00F09F812378412B00F0B281237813
:10991000592B00F0D08123784E2B00F0E58123787D
:109920004A2B00F0E5812378402B00F0E781237873
:109930006F2B00F0FC812378642B00F00A822378DF
:10994000702B00F0288223785B2B00F03D82237877
:109950003D2B00F03F822378732B00F03F82257867
:109960002C2D00F03F822E2D00F0458223783E2BD7
:1099700000F0538204B070BD2A20934B984766E7ED
:109980002520914B984766E726208F4B984766E73E
:109990007E208D4B984766E76078000240F05A00C1
:1099A000894B984763E7A378E27803EB0223227997
:1099B00003EB0243627903EB0263844A136060782D
:1099C000000240F07A00804B984754E7637833B93F
:1099D00001207F4B984724207B4B98474FE700207E
:1099E0007B4B9847F7E76378A07800EB032080B2C1
:1099F00010F4004F05D1774B98472420724B9847BD
:109A000041E747F6FF70F6E76378A07800EB0320A4
:109A100000B2714B984724206B4B984737E760782A
:109A20006E4B98472420684B984734E76278A378B8
:109A300003EB02239BB2092B05D9694A138024202A
:109A4000614B98472BE70122664B1A7045205E4B0D
:109A5000984724E763785BB1012B16D00022624B54
:109A60001A7001225F4B1A704520574B98471AE72E
:109A700002205E4B984730B904225A4B1A70452099
:109A8000514B98470FE72420FAE70120574B98479E
:109A900020B90422534B1A70452000E024204A4B81
:109AA000984700E763782BB1012B07D04520464B40
:109AB0009847FCE65E20444B9847F8E64FF4AF70B9
:109AC000414B9847F3E66278A37803EB0223484AB8
:109AD00013800520454B984720B90422414B1A704A
:109AE000452000E02420384B9847E4E64320364BDD
:109AF0009847E4E64220344B9847E4E662783D4BD1
:109B00001A705520304B9847E1E661780F2908D844
:109B100020224901A01C384B984724202A4B984703
:109B2000D9E601222F4B1A704520274B9847D2E6E1
:109B300008202E4B984720B904222A4B1A70452042
:109B400000E02420204B9847C9E62C4B62781A701D
:109B5000A2785A70E2789A700720244B984720B96F
:109B60000422204B1A70452000E02420164B984711
:109B7000B9E6234B98476378003318BF012303707D
:109B8000A3784370E378003318BF012383702379EF
:109B9000C37063790371A3794371E3798371237A85
:109BA000C371637A0372A37A4372E37A83720920E2
:109BB0000E4B984720B904220A4B1A70452000E04A
:109BC0002420014B984792E699974000C421002039
:109BD0004178400009784000357840000554400045
:109BE000C8210020CA2100207B22002039AF40007C
:109BF00096220020C0210020017D40007822002014
:109C0000F55B40006378A27803EB0223E27803EB74
:109C10000243227903EB02638F4A13606379A279CE
:109C200003EB0223E27903EB0243227A03EB0263A4
:109C30008A4A13604B208A4B98475CE65420884B35
:109C400098475CE609228749E01C874B984748B94A
:109C50006278864B1A70A278854B1A704420804B2C
:109C6000984750E60122834B1A7045207C4B984759
:109C700049E66278531EDBB21F2B06D901227D4BC9
:109C80001A704520764B984741E6744B1A60A378CA
:109C9000E17803EB0123217903EB0143617903EBC5
:109CA00001636D490B60A11D7348744B98474120B7
:109CB0006B4B98472BE6002604AD45F8046D704BBE
:109CC000984700953346012204216E4DA847039B17
:109CD000002B3FF420AE4FF080526B4B1A60BFF365
:109CE0004F8FBFF36F8F16E64E205D4B984716E6F9
:109CF000607800024A305A4B984714E60120634BC3
:109D000098475F4B984703AB00930023012204213F
:109D10005C4DA847039B002B3FF409AE4FF08052E7
:109D2000594B1A60BFF34F8FBFF36F8FFFE5E21CF3
:109D30006178A078564B98470620564B984720B933
:109D400004224C4B1A70452000E02420444B9847D5
:109D5000F1E56078504B9847012803D04520404BEF
:109D60009847ECE524203E4B9847454B984703AB7A
:109D70000093002301220421424DA847039B002B9E
:109D80003FF4DDAD4FF080523F4B1A60BFF34F8F71
:109D9000BFF36F8FD3E5414B9847394B984703ABDF
:109DA0000093002301220821364DA847039B3BB1B5
:109DB0004FF08052344B1A60BFF34F8FBFF36F8F59
:109DC0002420274B9847BEE5354B98472420244B49
:109DD0009847BCE53D20224B9847BCE57320204BBB
:109DE0009847BCE508222F49601C1F4B9847002864
:109DF0007FF4B9ADFFDE08222A49601C1A4B984750
:109E000000287FF4B3AD284B4FF400421A60402184
:109E100083F80F13C3F80021A8E508222149601C2C
:109E2000114B984700287FF4A5AD154B984703AB1D
:109E30000093002301224FF48011124CA047039B92
:109E4000002B3FF497AD4FF080520F4B1A60BFF3D9
:109E50004F8FBFF36F8F8DE5BC210020CC210020F8
:109E600099974000B8474100A119410054210020B2
:109E7000B8210020CA21002058210020011A4100E9
:109E8000B5A04000B5F8400004ED00E019A1400085
:109E900031AE400039AF400039A1400059A8400020
:109EA00069A84000C447410000E100E08388B3F5A1
:109EB0009F5F0DD0B3F5706F1DD0B3F5206F27D025
:109EC000B3F5A05F30D0B3F5706F39D00020704784
:109ED000C288B2F51F6FEDD14289A2F5E751093969
:109EE00089B2C6293DD9A2F5DD521D3A92B2C62AE1
:109EF000E0D802207047C288B2F5F06FDDD1428908
:109F0000A2F50B52053A92B2C62AD6D80320704762
:109F1000C288B2F5206FD3D14289A2F6553292B2EF
:109F2000C62ACDD805207047C288B2F5206FCAD1A5
:109F30004289A2F6553292B2C62AC4D8052070478B
:109F4000C388B3F5F06F01D0002070474389A3F5B3
:109F5000B8530D3B9BB2C62B01D80420704700209C
:109F6000704701207047000000B9704710B50446E3
:109F70000120034B9847601EFFF7F6FF10BD00BF9E
:109F8000D5F1400038B50125044B1D70002108466D
:109F9000034CA04700212846A04738BD390D0020BA
:109FA0009158400010B50024022C09D80B4B1A78A8
:109FB000002108460A4B9847012801D00134F3E7F5
:109FC0000024022C09D8054B1A7800210120044BEB
:109FD0009847012801D00134F3E710BD3A0D002065
:109FE0008557400038B51A4B1B786BB90024022CFA
:109FF0001FD8184B1A78184B19880020174B984710
:10A00000012816D00134F2E701210020144CA047AA
:10A0100001210846A0471420124CA0470020124DF1
:10A02000A8470120A8471420A0470022084B1A7017
:10A03000DCE70024022C0AD8064B1A78064B198854
:10A040000120064B9847012801D00134F2E738BDC2
:10A05000390D00203A0D00202C01002085574000CA
:10A0600091584000D5F14000B5584000F8B505467C
:10A070000E460024204601E00134A4B22746B4EB8A
:10A08000960F14D215F8241005EB84035A7801EBCF
:10A0900002219A7801EB0241DB7801EB0361002891
:10A0A000EAD107F540608000014B9847E4E7F8BD2E
:10A0B00069694000014B1868704700BF400D0020DF
:10A0C000014B1878704700BF3D0D002010B582B0DD
:10A0D000084B0193002300934FF480720649074810
:10A0E000074CA047012802D00648074B984702B00A
:10A0F00010BD00BF400D0020D04C410085A14000A4
:10A1000001EF4000DC4C410055134100014B187831
:10A11000704700BF380D002018B9044A044B1A607C
:10A120007047044A024B1A60704700BFD04B410091
:10A1300028010020D0474100032817D8DFE800F0AD
:10A1400002070C110A4A0B4B1A60012070470A4A99
:10A15000084B1A6001207047084A064B1A6001201C
:10A160007047074A034B1A60012070470020704770
:10A17000D04B410028010020D04A4100D049410085
:10A18000D0484100F0B585B001238DF80B307B4BF2
:10A19000009300231A467A497A487B4CA0477B4BB0
:10A1A000186004A9502301F8063D0320784CA0470D
:10A1B00004A9002301F8073D0D20A04710B9002392
:10A1C00003930BE09DF80900724B9847F7E74FF0B7
:10A1D000FF3303AA002108466F4CA047039B13F0EE
:10A1E000010FF4D040F213106C4B98476C4B98471A
:10A1F0004FF480716B4B18686B4B984706E04FF03B
:10A20000FF3303AA00210846634CA047039B13F0C9
:10A21000020FF4D01920614B9847644B4FF48072C1
:10A220001A63DB6B13F4004F19D0614B98470F2072
:10A23000604B984701465D485F4B984700225F4B53
:10A240001A700DF10B010420514B984728B19DF86D
:10A250000B3083F001038DF80B30002403E0584BE2
:10A260009847E4E7002414204C4B9847002303AAA6
:10A270001C211846484DA847039B13F0080F00D037
:10A28000012413F0100F40F0B780039B13F0040F6C
:10A290002ED04A4B1B78002B40F0FF800F20454BFF
:10A2A000984701464148474B9847454B9847464B8E
:10A2B00098473B4B98473B4D4FF4807128683A4B89
:10A2C00098472A68414B9A4200F0F380374BDB6B8A
:10A2D00013F4004F00F0F080354B98470F20354BBA
:10A2E000984701463148344B98472420384B9847CB
:10A2F000039B13F4801F40F0E280304B1B78002B4F
:10A3000040F0E180334B9847002840F0FE80002267
:10A310002A4B1A709DF80B3093B12F4B1B787BB1F1
:10A320002E4B1B78002B00F01E822D4B984738B91E
:10A3300000222A4B1A702B4B9847002840F00182CC
:10A34000002C90D0254B1D78002D8BD11B4B1C78F9
:10A35000002C88D00122244B1A70244B98470B4BB9
:10A3600018680A23009300231A460321204CA047B3
:10A370000022204B1A702C4675E700BF859F4000D5
:10A38000E0930400044D41009DFB4000102200209A
:10A39000A57D400039A1400065F74000D5F140009F
:10A3A000C5684000280100206DA04000000E0E404E
:10A3B000E154400073D840004FD840003D0D0020CC
:10A3C000BD54400053D8400001694000D0474100CF
:10A3D0007D9740007D054100240100202E010020D2
:10A3E000DD5B4000C1A04000380D0020E59F40002B
:10A3F000D9FB4000390D00200F20924B9847924E18
:10A4000001463046914B9847914B98474FF480470F
:10A4100077630A208F4DA8478F4B98474FF4FA7007
:10A42000A8478E4B9847776301208D4B984719209A
:10A43000A8474FF48073336300208A4EB047012051
:10A44000B04700210846884EB04700210120B047A0
:10A4500001210020854EB04701210846B047142055
:10A46000A8470020824EB0470120B0470127814B0A
:10A470001F70814B98479DF80A100023032241F476
:10A4800080717E4EB0477E4B984700233A460221AA
:10A49000B0474FF0FF30A847F7E60022754B1A701F
:10A4A000694D4FF480766E6319206A4B98472E638E
:10A4B000F4E6744B984709E7654B98470EE7402050
:10A4C000714B984719E7714B984720B1704B9847EB
:10A4D00000287FF417AF0025664B1D70664B984728
:10A4E0002B4603224FF48071644EB047644B98476B
:10A4F0002B4601220421B047534D4FF480766E6302
:10A500001920544B98472E63FCE6614B984700286E
:10A510003FF4FDAE574B1B78002B7FF4FBAE0020C1
:10A520005C4EB0475C4D28700120B0475B4B187003
:10A530002B78002B3FF4EEAE00283FF4EBAE012267
:10A540004C4B1A70564D2846564B98472846564B4A
:10A5500098470746052816D00022544B1A704FF42E
:10A56000FA703C4B984700204A4EB0474A4D28703D
:10A570000120B047494B18702B7803B138B900223D
:10A580003C4B1A70C6E60122484B1A70E7E73A4B7B
:10A5900098479DF80A100023032241F48071374D3B
:10A5A000A847374B9847002301220221A847394684
:10A5B00000203F4DA84739460120A8470A203D4BBF
:10A5C0009847D8B93C4D002128463C4B98472B78FA
:10A5D000112B18D000210846234DA8470021012047
:10A5E000A8470025022D20D8304B1A7800210846B4
:10A5F000334B9847012818D00135F3E731490A2039
:10A60000314B9847DEE76B78002BE3D1AB78002B1A
:10A61000E0D1EB78892BDDD12E46294600202B4D49
:10A62000A84731460120A847D4E70025022D4FD87E
:10A630001E4B1A7800210120214B9847012847D052
:10A640000135F3E773D84000000E0E4053D84000A8
:10A65000BD544000D5F14000557A4000D17940000A
:10A66000FD7940005D5A40006D584000915840000F
:10A67000B55840003D0D002091AF400009F8400062
:10A680009DAF4000A96B4000699F40007D054100DF
:10A6900089054100616A40003B0D00203C0D00200F
:10A6A0006C2200209D6A4000AD9E40003A0D0020C3
:10A6B00099594000F17D400014220020B969400002
:10A6C000855740002C010020A57D400085594000A1
:10A6D00001210020334DA84701210846A847142036
:10A6E000314B98470020314DA8470120A8479DF8DD
:10A6F0000B3003B32E4B9847E8B12E4B1B78D3B1E8
:10A700002D4B1B782BB101222C4B1A702C4B9847E8
:10A7100000E60025294B1D702A4B98472A4B1E68DE
:10A720002A4B98470A2300932B46024601213046C4
:10A73000274DA847EEE50122204B1A70204B984781
:10A74000E8E500251D4B1D701E4B98471E4B1E68EB
:10A750001E4B98470A2300932B46024601213046A0
:10A760001B4DA847ECE51B4B984700283FF4E8AD8C
:10A770000122114B1A70184B984700283FF4E0ADA6
:10A7800001220E4B1A700E4B98470F4B18680A2384
:10A79000009300231A4603210D4DA84700220F4BBA
:10A7A0001A70CDE591584000D5F14000B5584000F1
:10A7B000315B4000240100202E010020380D0020D4
:10A7C000E59F4000A59F400010220020FDEF4000C3
:10A7D000D9FB4000DD5B4000C1A04000390D0020E6
:10A7E000124A1080124A12787AB138B50446002510
:10A7F000022D0CD80F4B1A78214600200E4B98479B
:10A800000346012803D00135F2E7012070471846BE
:10A810000025022D09D8074B1A7821460120064B46
:10A820009847012801D00135F3E738BD2C010020FD
:10A83000380D00203A0D00208557400010B5044B1C
:10A840009847002303221021024CA047012010BD8D
:10A85000B5A0400009F840000022024B1A70012008
:10A86000704700BF240100200120014B1870704781
:10A870002401002038B50024204609E000F47F437D
:10A88000B3F5007F0CD000F47F43B3F5807F0CD08C
:10A890000028F3D14FF0FF310120134B9847EDE72B
:10A8A0000020124B98470020EDE7C5B2002008E0D9
:10A8B0000134A4B220460D4B98470A2101200A4BCF
:10A8C000984758B9AC42F3D308E0013CA4B2204603
:10A8D000064B98470A210120034B98470028D7D1FF
:10A8E000AC42F2D8D4E700BFE1F640000554400086
:10A8F000F0B583B00224002010F0010F0AD14FF010
:10A90000FF310120314B984700F00E03042BF3D1A7
:10A910000424F1E72E4B1B68ADF804301B0C8DF8B6
:10A92000063001A902202B4B9847042C07D02A4B54
:10A93000984701A9294B984700252E4607E0264B4A
:10A9400098470021264B9847F1E72E4602253221F1
:10A9500001201E4B984700F00E00042812D0022858
:10A9600014D0042CF3D1C5B1022D22D0032DEED189
:10A970000136F6B2182EEAD900252E46E7E7032560
:10A980000026E4E700252E460424E8E7124B98470A
:10A990008021134B98470224E3E70F4B9847771C1D
:10A9A000FFB2104B995D0E4B9847632FCDD83E46B2
:10A9B000CDE7094B9847771CFFB20B4B995D084BCD
:10A9C0009847632FDBD83E46C1E700BFE1F6400061
:10A9D000184D4100A57D40002D05410095634000C4
:10A9E00045634000940100203001002008B5044B6D
:10A9F00098476420034B9847034B9847F7E700BFFD
:10AA0000256E4000D5F14000597F400070B582B0FE
:10AA1000944B9847944B98470120944B984702A930
:10AA2000002301F8013D0520914B984728B19DF87E
:10AA3000073013B100208D4B98478E4B98478E4BB3
:10AA400098478E4A8E4B1A6001208E4B98470446D9
:10AA500090B98A4D8C4C0FCC28606960AA60EB607D
:10AA60008A4B98478A4B984702228A4B1A638A4B33
:10AA700098470546002416E0814B196801207C4B5D
:10AA8000984705E07E4B1B6800221A550134E4B25A
:10AA90000F2CF7D9E4E70520804B98477E4B984769
:10AAA00005460134E4B20DB9132CF4D97C4B984718
:10AAB00029467C4B98477C4B98477C4DA847002300
:10AAC000012211467A4CA04701207A4B9847A847AB
:10AAD000002301220221A047774B98476B4B9847F0
:10AAE000764B984700230122052175480068A0474E
:10AAF00000252C4680E01146002341F8043B7148B4
:10AB0000714B984738B9714B5968013159606D489C
:10AB10006F4B98477BE001216A486D4B984776E080
:10AB20001146002341F8043B6A48674B984798B99F
:10AB3000694B5968013159606648654B98476749C8
:10AB40006748614B984760B9634B59680131596058
:10AB500063485F4B984768E001215E485C4B98472B
:10AB6000EDE701215E485A4B98475EE0134600220C
:10AB70001A605A6801325A6069465A48524B9847DF
:10AB800050B9594B5968009B994201D8002514E0EF
:10AB900054484F4B9847F9E7534B596851484C4B31
:10ABA0009847F3E7514A136801331360052B44D9E2
:10ABB0004D4B00251D605D6015604D4BA3FB0423CC
:10ABC000DB0803EB83035A00944238D0494B984783
:10ABD000002840F09D80484BA3FB04235B096422BE
:10ABE00002FB1343002B00F096800A202B4B984762
:10ABF0000134632C00D900240135B5F57A7FDCD30C
:10AC0000324A1368013313603B2B3FF674AF3B4B62
:10AC100098470028C6D00022344B1A602E4A136889
:10AC2000013313603B2B3FF67BAF2F4A1368013390
:10AC300013603B2B9AD80025BFE70025BDE7304BBA
:10AC4000984728B947232F4A13702F4A1370BDE73E
:10AC500000202E4EB0472B4B18700120B0472A4BD6
:10AC60001870B3E7858340008D7E4000B1544000EA
:10AC7000A57D4000BD544000F95240009C220020B8
:10AC80007C220020F17D4000D04D41002D05410087
:10AC90002D654000000E0E40856E4000D5F140004D
:10ACA00025054100F5654000D1794000B5A0400080
:10ACB00009F84000FD7940006D5A40008162400073
:10ACC000680D00200110FFFF8D844000580D00200A
:10ACD000E18440000210FFFF480D00204C0D0020D1
:10ACE0000410FFFF0310FFFF500D0020440D002053
:10ACF000CDCCCCCC315B40001F85EB510DA1400089
:10AD0000C1A04000F8010020F90100200D594000C9
:10AD1000024B984769E7024B984766E73D5B400066
:10AD20006D5A400008B509E000210846314CA047A3
:10AD300000210120A04700222F4B1A704FF0FF3155
:10AD400001202E4B98472C4B1B78013B082BF2D847
:10AD500001A252F823F000BF7DAD400029AD4000B4
:10AD600097AD4000A7AD40008DAD4000DFAD400085
:10AD7000C7AD4000D3AD4000D9AD40000121002057
:10AD80001C4CA04701210846A047D4E71C4B18885B
:10AD90001C4B9847CFE7002108461B4CA0470021D9
:10ADA0000120A047C7E701210020174CA04701213F
:10ADB0000846A0471420154B98470020144CA04784
:10ADC0000120A047B7E7134B98471349134B984707
:10ADD000B1E7134B9847AEE7124B9847ABE7124ADF
:10ADE000D01E134612F8032C817840780F4CA047F0
:10ADF000A1E700BFED5840007B220020E1F64000B3
:10AE000096220020E1A7400091584000D5F1400073
:10AE1000B55840002D054100782200209563400080
:10AE2000457D4000015C4000AF220020FD55400000
:10AE300010B51446044B1870597002462146981CF0
:10AE4000024B984710BD00BFAC220020011A410000
:10AE500010B582B0234B019303230093002380227B
:10AE600021492248224CA047012802D02148224BE8
:10AE70009847224B019300230093802220492148C8
:10AE80001B4CA047012802D01F481B4B98470023AA
:10AE90000193009380221D491D48154CA0470128AD
:10AEA00002D01C48144B98471B4B0193002300937E
:10AEB00080221A491A480E4CA047012802D019488E
:10AEC0000D4B9847184B019300230093802217499C
:10AED0001748074CA047012802D01648064B984750
:10AEE00002B010BD640D00201C4D410025AD400096
:10AEF00001EF4000204D4100551341006C0D002032
:10AF00003C4D41000DAA4000484D4100704D4100AC
:10AF1000EDA94000744D4100680D0020904D4100A6
:10AF2000F1A84000944D4100600D0020B04D41005B
:10AF300075A84000B44D410010B584B0104B187096
:10AF40000022039204AB43F8082D0E4A106803AAAE
:10AF50000092042201210C4CA047029B5BB9039B89
:10AF600063B14FF08052094B1A60BFF34F8FBFF3AC
:10AF70006F8F012000E0002004B010BD0120FBE72E
:10AF80007B220020640D0020B5F8400004ED00E0B5
:10AF9000014B1868704700BF600D0020014B186816
:10AFA000704700BF680D00200023044A1370044A54
:10AFB00013700120034B1870704700BF780D0020FC
:10AFC000740D0020710D00207047002070470000B4
:10AFD0000D4B5B881A0A032A01D00020704713F03A
:10AFE000FF0F0ED1084BDB88402B01D000207047AB
:10AFF000054B064A9A60064A1A6140229A8101204E
:10B0000070470020704700BF102300207C0D0020F7
:10B0100045B040000122014B1A707047710D0020AD
:10B0200010B5034B034A04490448054CA04710BD22
:10B03000D1AF4000CC020020740D0020780D00201C
:10B0400089B1400008B5084B9B89402B00D008BD52
:10B05000064B1B781BB90648064B9847F7E7044890
:10B06000054B984708BD00BF10230020700D00203D
:10B070007C0D00204198400021504000014B187089
:10B08000704700BF700D0020224B1B780BB918468B
:10B0900070472DE9F04184B00746EFF31083B3FA0F
:10B0A00083F35B09039372B6BFF35F8F00211A4BE2
:10B0B0001970DDF80C80194D40222846184B98472E
:10B0C0003C4640372E4620686168A268E3680FC698
:10B0D00010343546BC42F5D1124B009340230F4A41
:10B0E00000218120104CA04780F00100094B18700E
:10B0F000B8F1000F05D00122074B1A70BFF35F8F24
:10B1000062B6044B1B7883F00103184604B0BDE817
:10B11000F08100BF710D00202F030020BC0D002026
:10B12000FD1B410015B0400065D3400010B504463A
:10B13000134B9847837A212B01D0002010BD00F1DA
:10B140000902104B5B881B0A212B04D0C27B93425F
:10B150000BD0002010BD0B4B9A60427AD9888A42EE
:10B1600028BF0A469A81012010BD064B9C60028AC6
:10B17000D9888A4228BF0A469A81012010BD00BFA3
:10B1800061B7400010230020F8B5264C247865B242
:10B19000002D07DB002D40DB04F06004202C22D0C2
:10B1A0000020F8BD14F0600603D11E4F7F78062FF3
:10B1B0000BD0202EEED11B4A5278022A09D0032A46
:10B1C0000CD0012AE6D19847F8BD1046164B984797
:10B1D000F8BD144B986001209881F8BD114B99601F
:10B1E00001209881F8BD0F4A52780A2A07D00B2A0D
:10B1F0000BD0092A01D00020F8BD9847F8BD094BB3
:10B200005B881B0A03700120F8BD064BDB8833B94D
:10B21000044B5B880B700120F8BD0020F8BD0020B6
:10B22000F8BD00BF102300202DB14000014B18686D
:10B23000704700BF7C220020024B1B681B685888A7
:10B2400018447047080E002038B504460D46094BD7
:10B250009847024620782044904207D24378042B36
:10B2600006D0AB4205D003781844F5E7002038BD7E
:10B27000002038BD39B2400038B5144B1B780BB3F1
:10B28000134B1B681B681A7982421DD90D46044670
:10B29000104A1360104B984703E01A7813440D4A84
:10B2A00013600C4B1B6898420AD95A78042AF4D1CF
:10B2B0009A789442F1D1DA78AA42EED1012038BDD1
:10B2C000002038BD002038BD002038BD040E00200D
:10B2D000080E00200C0E002039B24000084BDB881D
:10B2E00063B9074B5B88012B01D000207047054AEA
:10B2F000138823F002031380012070470020704759
:10B3000010230020FC0D002000207047044BDB8838
:10B3100023B9044A024B1A6101207047002070478C
:10B320001023002051B6400038B5134B1B7803B3EF
:10B33000124B1C79124B1B681B681B799C4201D372
:10B34000002317E0002120460E4B9847034688B1A2
:10B350000B4B1B685B6853F82450EB689847014619
:10B360002046084B9847034620B1AB6898470346F0
:10B3700000E00023184638BD040E002010230020F2
:10B38000080E002079B2400038B5104B1B78D3B1BD
:10B3900000240F4B1B681A681279944211D25B6823
:10B3A00053F82450EB68984701462046094B9847CC
:10B3B000034648B1AB689847034628B90134E4B264
:10B3C000E7E7002300E00023184638BD040E002004
:10B3D000080E002079B2400070B504460021114BE0
:10B3E0009847054608B9284670BD0F4B1B685B6837
:10B3F00053F82460F368984701462046094B984764
:10B4000005460028EFD0094B1C6805212046084B53
:10B410009847044618B18078064B9847F5E773685B
:10B420009847E0E779B24000080E00200C0E00209B
:10B4300049B24000E5D0400008B5064BDB88022B3E
:10B4400001D0002008BD02210348044B9847012089
:10B4500008BD00BF10230020FC0D0020C9CF400014
:10B4600010B5184B9B78032B2AD8DFE803F00502B0
:10B47000100B0920144C0CE004211448144B98477D
:10B48000002006E0134B98470446102001E00620F8
:10B49000114C08B1002308E0012010BDE15C0F4A07
:10B4A00002EB430251800133DBB28342F6D3411CED
:10B4B0004900C9B209480170054B9847012010BDE9
:10B4C000002010BD102300201C03002018030020C2
:10B4D000C9CF40002DB2400028030020F402002014
:10B4E00008B5234B5B88DAB21B0A013B0E2B38D818
:10B4F000DFE803F008173137373737373737373753
:10B5000037372A001B4B186801781B4B9847184B9C
:10B51000DA889B899A4228D2154B9A8101231846D2
:10B5200008BD144B1B685B7C9A4201D30023F6E7ED
:10B53000104B5B6853F8320041880F4B98470C4B17
:10B540009B6802225A70E2E70A4B986858B141881A
:10B55000094B9847DBE7094B984703460028D6D1AB
:10B56000DDE70023DBE70023D9E70123D7E700BFAE
:10B5700010230020FC010020C9CF400061B440002E
:10B5800008B5064BDB88012B01D0002008BD012146
:10B590000348044B9847012008BD00BF102300203A
:10B5A000040E0020C9CF400038B5154BDB88012BB5
:10B5B00002D00024204638BD124B1B78F3B1104B4B
:10B5C0001D79114B1B681B681B799D4201D3002418
:10B5D000F0E7002128460D4B984704460028E9D0A3
:10B5E000094B1B685B6853F82530DB689847084BAC
:10B5F000187001211846074B9847DBE70024D9E76C
:10B6000010230020040E0020080E002079B2400014
:10B61000000E0020C9CF400008B5094BDB88022B83
:10B6200001D0002008BD064B1879064B9847064B01
:10B63000188002211846054B9847012008BD00BF1D
:10B640001023002035D14000FE0D0020C9CF40005E
:10B6500008B5034B588800F07F00024B984708BD9F
:10B660001023002071CF400038B505460F4B984796
:10B670000346C0B10E4B1C68052120460D4B984770
:10B68000044640B18288C17880780B4B98470346C6
:10B690000028F1D107E0094B1B685B6853F825309F
:10B6A0001B6898470346184638BD00BF79B2400072
:10B6B0000C0E002049B24000D5CF4000080E0020FB
:10B6C00038B50C4BDB8893B90B4B1B780BB90023B7
:10B6D0000EE0084B1C799D782046084B984703469E
:10B6E00030B129462046064B9847034600E0002328
:10B6F000184638BD10230020040E0020D9B34000A6
:10B7000069B6400008B5074BDB884BB9054B5B8831
:10B710000BB1002008BD034B1879034B984708BDB7
:10B72000002008BD1023002071D24000094BDB88A7
:10B730006BB9084B5B880BB10020704710B5054C06
:10B740002079054B98472079044B984710BD00207D
:10B75000704700BF10230020E1D4400079D14000A1
:10B76000014B1868704700BF0C0E002008B5014B54
:10B77000984708BD11CE400010B50B4B1B7863B144
:10B78000002404E02046094B98470134E4B2084BFA
:10B790001B681B681B799C42F4D30022024B1A7071
:10B7A0000122044B1A8010BD040E0020D9B34000C2
:10B7B000080E0020FC0D002008B5024B9847024BF4
:10B7C000984708BDF9CE400079B740001C4BDB8894
:10B7D00013B100231846704710B51A4B984750B361
:10B7E000174B9A78184B1B685B7C9A4201DD00234B
:10B7F00022E0164B9847124B9B78154A1370EBB119
:10B80000114A526803F10053013B02EBC303114A92
:10B81000136000240F4B1B681B681B799C4208D2E5
:10B82000002120460C4B9847034628B10134E4B26E
:10B83000F0E7012300E00023184610BD0123FBE7D9
:10B8400010230020ADCF4000FC01002079B740005C
:10B85000040E0020080E002069B6400008B5344BE5
:10B860001B7813F0800F0ED113F01F0343D1304A21
:10B870005278013A082A3ED8DFE802F0343D373DDD
:10B88000313D3D3D3A002A4AD288002A4ED013F07D
:10B890001F0306D1264A5278062A0BD0082A0CD05C
:10B8A0002AB1012B0CD0022B11D0002008BD214B56
:10B8B000984708BD204B984708BD204B984708BDC6
:10B8C0001B4A52780A2AEED11D4B984708BD184BE7
:10B8D0005B780BB1002008BD1A4B984708BD1A4B86
:10B8E000984708BD194B984708BD194B984708BDA4
:10B8F000184B984708BD012B03D0022B08D000201D
:10B9000008BD0B4A52780B2AF7D1134B984708BD54
:10B91000074B5B78012B03D0032B04D0002008BD1C
:10B920000E4B984708BD0E4B984708BD002008BD38
:10B930001023002039B44000E1B4400081B540003C
:10B94000A9B5400019B640000DB34000DDB240007B
:10B9500009B34000CDB74000C1B6400005B7400074
:10B960002DB740000B4B1B7813B110B5002402E03B
:10B9700070470134E4B2084B1B681A68127994428C
:10B9800007D25B6853F824301B69002BF1D098472D
:10B99000EFE710BD040E0020080E002008B5184B7C
:10B9A00000229A811A615A611B7813F0800F11D11D
:10B9B00013F0600F14D0124B1B7803F01F03012B00
:10B9C00014D00F4B1B7803F01F03022B14D000235D
:10B9D000184608BD0A4AD288002AE9D10023F7E7B1
:10B9E000084B984703460028E5D0F1E7064B9847F7
:10B9F00003460028E5D0EBE7044B98470346E7E70A
:10BA0000102300205DB8400029B3400089B34000F6
:10BA1000F8B504460E46114B984705462046104B94
:10BA20009847054001D0002403E0F8BD0134062CFE
:10BA300011D88DB123010B4AD058B042F6D102EB98
:10BA4000041359680D42F1D01F46DB6898477B68A4
:10BA500025EA0305EAE7F8BDF8BD00BF57D8400066
:10BA60005BD84000100E0020F8B5164C2768062F52
:10BA700026D8002401E00134E4B2A446A7420AD348
:10BA8000114E250106EB050E75598D42F3D1DEF8F6
:10BA900004509542EFD1CEF80010CEF80420CEF835
:10BAA00008300699CEF80C100137BC4505D0114678
:10BAB0001A46064B98470020F8BD02490F60F6E78A
:10BAC0000120F8BD800E0020100E00201DD840007F
:10BAD0002DE9F04182B004460F4690460A4B984744
:10BAE00005462046094B984706462046084B98478E
:10BAF000CDF800803B46024631462846054CA0471B
:10BB000002B0BDE8F08100BF5FD840006DD84000B2
:10BB100073D8400069BA400008B50B210148024BB8
:10BB2000984708BD000E0E4011BA400008B50C2120
:10BB30000148024B984708BD00100E4011BA400062
:10BB4000F8B506460C461546224B984707464FF077
:10BB5000FF313046204B98473046204B9847002C09
:10BB60000CDB630904F01F0101228A4020331C49C9
:10BB700041F82320BFF34F8FBFF36F8F002C08DBFA
:10BB8000630904F01F0101228A406033144941F81F
:10BB90002320002C17DB2D01EDB204F1604303F5E7
:10BBA000614383F80053002C08DB620904F01F0492
:10BBB000012303FA04F40A4B43F822403946304685
:10BBC000084B9847F8BD04F00F022D01EDB2064B6B
:10BBD0009D54E8E75BD8400053D8400057D8400058
:10BBE00000E100E04FD8400014ED00E082B00246D2
:10BBF00010B9244B1B783BB912B1224B1B780BB305
:10BC0000204B1A7002B070471F4B1B7803B9FEE738
:10BC1000EFF31083B3FA83F35B09009372B6BFF3BB
:10BC20005F8F0021194B1970009817490B78013B61
:10BC30000B700028E0D00121144B1970BFF35F8F07
:10BC400062B6D9E7104B1B78FF2B19D0EFF31083A6
:10BC5000B3FA83F35B09019372B6BFF35F8F0021E0
:10BC60000A4B1970019808490B7801330B700028B2
:10BC7000C6D00121054B1970BFF35F8F62B6BFE7D5
:10BC8000FEE700BF850E0020282300202F030020A0
:10BC900084B02A4B9A6842F480729A609A6822F0C3
:10BCA0007F029A601A6B0192019A42F04F02019250
:10BCB000019A22F4074222F080020192019A42F492
:10BCC00000420192019A1A631C4B1B6B13F4004F44
:10BCD000FAD01A4A136B0293029B43F04F0302936C
:10BCE000029B43F400430293029B136300238DF8ED
:10BCF000033006E000BF9DF803300133DBB28DF85E
:10BD000003309DF80330DBB2132BF3D9EFF310832C
:10BD1000B3FA83F35B09039372B6BFF35F8F00221C
:10BD2000074B1A70039B0121044A116123B1044B94
:10BD30001970BFF35F8F62B604B0704700400440D3
:10BD40002F030020034A0023136153619381024AA9
:10BD500013707047102300208A0E002082B0052245
:10BD6000104B1A70104A136B0193019B43F04F0361
:10BD70000193019B43F020030193019B1363002374
:10BD80008DF8033006E000BF9DF803300133DBB2CD
:10BD90008DF803309DF80330DBB2132BF3D902B0DA
:10BDA000704700BF8A0E00200040044082B003228A
:10BDB000104B1A70104A136B0193019B43F04F0311
:10BDC0000193019B43F010030193019B1363002334
:10BDD0008DF8033006E000BF9DF803300133DBB27D
:10BDE0008DF803309DF80330DBB2132BF3D902B08A
:10BDF000704700BF8A0E0020004004400422014B1F
:10BE00001A7070478A0E002008B5024B1B6903B1F7
:10BE1000984708BD1023002030B589B06A4B1B78C5
:10BE2000032B29D0694B9C89694B1B88E41AA4B267
:10BE3000002C43D1674A11880B449BB21380634A9C
:10BE4000D288934203D0644B1B78002B2CD0634BD9
:10BE50009847634A136B0393039B43F04F03039389
:10BE6000039B23F001030393039B13635C4B1B6B46
:10BE700013F0010FFAD115E0594A136B0293029B9C
:10BE800043F04F030293029B23F001030293029BB2
:10BE90001363534B1B6B13F0010FFAD1514B9847AF
:10BEA000514B984709B030BD484B5B6933B1984757
:10BEB00020B10022464B1A80444B9C893F2C37D935
:10BEC0000022454B1A704024404B9A68404B1B8817
:10BED0001A44EFF31083B3FA83F35B09079372B646
:10BEE000BFF35F8F0021414B197007983C4B1B6BD0
:10BEF00013F0020F3ED028B101223C4B1A70BFF361
:10BF00005F8F62B60422304B1A70354A136B04936C
:10BF1000049B43F04F030493049B23F00103049319
:10BF2000049B13632E4B1B6B13F0010FFAD1B9E77F
:10BF30000122294B1A70C7E7157829490D6501338D
:10BF4000DBB2013299B28C42F6D8214B1A881444E4
:10BF50001C80234A136B0593059B43F04F03059305
:10BF6000059B43F010030593059B136300238DF895
:10BF7000073008E00023E5E700BF9DF807300133F4
:10BF8000DBB28DF807309DF80730DBB2132BF3D905
:10BF9000134A136B0693069B43F04F030693069BCD
:10BFA00023F001030693069B13630D4B1B6B13F0E9
:10BFB000010FFAD100283FF475AF01220B4B1A7024
:10BFC000BFF35F8F62B66DE78A0E0020102300205A
:10BFD000860E0020880E0020840E0020FDBD40004B
:10BFE0000040044009BE400045BD40002F03002032
:10BFF00010B586B0654B1B78012B1ED0022B04D0E8
:10C00000042B02D0624B984701E0624B9847624A8A
:10C01000136B0093009B43F04F030093009B23F0AE
:10C0200002030093009B13635B4B1B6B13F0020F27
:10C03000FAD15A4B984706B010BD574B186BC0F356
:10C040000A40574B9B89574A14882218934201DAB9
:10C05000181B80B2524B9A682244002305E04E49D7
:10C06000096D11700133DBB2013299B28842F6D802
:10C070000444A4B24B4B1C8040281BD0484B9C81ED
:10C080005B6913B19847002832D0434A136B02937F
:10C09000029B43F04F030293029B23F0020302939F
:10C0A000029B13633C4B1B6B13F0020FFAD13E4B08
:10C0B0009847C0E73A4BDA883C4B1B8823449A42A6
:10C0C000DCDD374B9B899C4227D0334A136B0593A9
:10C0D000059B43F04F030593059B23F00203059353
:10C0E000059B13632C4B1B6B13F0020FFAD1A2E7D5
:10C0F000274B9847284A136B0193019B43F04F034A
:10C100000193019B23F002030193019B1363224BD4
:10C110001B6B13F0020FFAD18DE7214B5B6953B112
:10C120009847E8B121491F4A0B88108803440B80C7
:10C1300000231380C9E7164B9847174A136B0393E4
:10C14000039B43F04F030393039B23F002030393EA
:10C15000039B1363104B1B6B13F0020FFAD16AE7BA
:10C160000B4B98470C4A136B0493049B43F04F030B
:10C170000493049B23F002030493049B1363064B74
:10C180001B6B13F0020FFAD155E700BF8A0E002097
:10C190005DBD400009BE40000040044045BD400078
:10C1A00010230020860E0020ADBD4000880E002028
:10C1B0000023042B14D810B40A499A00D418A00004
:10C1C00004460844407C214400F083026FF3C71208
:10C1D0004A740133DBB2042BEED95DF8044B70478F
:10C1E000704700BF8C0E002038B5437C13F0100F51
:10C1F00016D00D46437C6FF30413437404687CB17E
:10C2000002F10C03074951F8233013F4806F01D079
:10C2100042F080028168012D14BF00200120A04758
:10C2200038BD00BF0040044010B500240BE0234699
:10C230000134E4B203EB8303980022460121034B4F
:10C240001844034B9847042CF1D910BD8C0E0020E4
:10C25000E9C1400010B500F00F02531E03EB830349
:10C260009C00012102482044024B984710BD00BFAA
:10C270008C0E0020E9C1400030B482B00246441E5A
:10C280003B4900F10C0551F8253051F8251013F009
:10C29000020302D001F0400151B9002B39D004EB68
:10C2A00084039900334B0B44597C6FF38301597419
:10C2B00004EB840399002F4B0B445B7C13F00C0FB1
:10C2C00032D12B4900F10C0551F825300093009B29
:10C2D00043F04F030093009B23F002030093009B65
:10C2E00041F8253002F10C03214951F8233013F0B5
:10C2F000020FF7D1002838D0032836D004EB84048D
:10C30000A2001C4B13445A7C012161F383025A742E
:10C310002BE004EB84039900164B0B44597C012558
:10C3200065F383015974C3E711490C3051F820308B
:10C330000193019B43F04F030193019B23F04003C2
:10C340000193019B41F8203002F10C03084951F898
:10C35000233013F0400FF7D104EB8404A200054B07
:10C3600013445A7C6FF383025A7402B030BC704796
:10C37000004004408C0E0020F0B4461EB30033444D
:10C3800099002A4A0A445368D1680B449468641A95
:10C39000128AC2F30902944209D31446002706EB1D
:10C3A00086029500214A2A442144D1601EE00127DB
:10C3B000F5E71D781E4A00F1140142F821505D781E
:10C3C00042F821509D7842F82150DD7842F8215002
:10C3D0001D7942F821505D7942F821509D7942F84B
:10C3E0002150DD7942F82150083C0833072CE0D871
:10C3F00007E01D7800F114020D4941F82250013C7C
:10C400000133002CF5D1094BB10088198200104688
:10C410001A44527CC2F3810203440132597C62F314
:10C42000830159743846F0BC704700BF8C0E002061
:10C430000040044070B582B0441E04EB84039A00AF
:10C44000364B13445B7CC3F3810328B1032801D02E
:10C45000022202E0012200E001229A4254DDA20001
:10C46000224495002D4B2B44DA689B689A4205D3F1
:10C470002A4B2B445B7C13F0400F48D00E460546F8
:10C48000274B9847FEB1274A0C3552F825300193C7
:10C49000019B43F04F030193019B43F01003019371
:10C4A000019B42F8253000238DF8033006E000BFE1
:10C4B0009DF803300133DBB28DF803309DF8033073
:10C4C000DBB2132BF3D940B104EB84039A00134B76
:10C4D00013445A7C6FF386125A74A20022449100CE
:10C4E0000E4B0B44DA689B689A4212D30B4B0B44F9
:10C4F0005B7C13F0400F0ED1084B0B445A7C42F08A
:10C5000080025A74002000E0012002B070BD0020BB
:10C51000FBE70120F9E70120F7E700BF8C0E0020C0
:10C5200079C34000004004402DE9F84305468446A5
:10C53000471EBB003B449A002A4C1444A268E3689F
:10C54000A2EB030EB4F81080C8F3090862681A441D
:10C550000C30254951F82060C6F30A4666B3B6454B
:10C560000BD9B6464FF0000907EB870188001D493B
:10C5700001447344CB6000210AE04FF00109F3E766
:10C580000CF11403184850F82330137001310132B4
:10C590008E45F5D82846154B9847B9F1000F01D1C3
:10C5A000B04507D905F10C030F4A52F8233013F0B8
:10C5B000200F04D0BDE8F8834FF00009EAE701231B
:10C5C000AB405361074ABB00D819810008461144AB
:10C5D000C968024491602A4600212046044B9847CE
:10C5E000E8E700BF8C0E00200040044079C2400004
:10C5F000E9C140002DE9F0418CB00124ADE12046B5
:10C60000B34B98470120FAE1BB003B449900B14A83
:10C610000A44537CC3F38101033161F383035374F0
:10C62000537C13F0200F00F0848013F00C0F3BD0EC
:10C63000A94A04F10C0152F821300193019B43F007
:10C640004F030193019B43F010030193019B42F8B8
:10C65000213000238DF8013006E000BF9DF8013045
:10C660000133DBB28DF801309DF80130DBB2132BC2
:10C67000F3D9994A06F10C0152F821300293029B3A
:10C6800043F04F030293029B23F001030293029BAA
:10C6900042F8213006F10C038F4A52F8233013F090
:10C6A000010FF7D10120AAE18B4A04F10C0152F8E5
:10C6B00021300393039B43F04F030393039B23F029
:10C6C00001030393039B42F8213006F10C03824AD5
:10C6D00052F8233013F0010FF7D1114606F10C0385
:10C6E00052F823200492049A42F04F020492049AD2
:10C6F00042F020020492049A41F8232000238DF88E
:10C70000023006E000BF9DF802300133DBB28DF845
:10C7100002309DF80230DBB2132BF3D907EB870709
:10C72000BA006C4B13445A7C6FF345125A740120C3
:10C7300065E113F0800F42D1BB003B449A00654B8A
:10C740001344DA689B689A424CD307EB87039A003C
:10C75000604B13445B7C13F04C0F43D1EFF3108319
:10C76000B3FA83F35B090B9372B6BFF35F8F0022BA
:10C770005A4B1A700B9B584A55612BB10122574BEB
:10C780001A70BFF35F8F62B6534A06F10C0152F87C
:10C7900021300593059B43F04F030593059B23F040
:10C7A00001030593059B42F8213006F10C034A4A28
:10C7B00052F8233013F0010FF7D101201FE1BB0025
:10C7C0003B449A00434B1344597C6FF3C71159748F
:10C7D000DA689A60404B5D61224600214046404B3A
:10C7E0009847A9E7002C4AD0032C48D007EB8703D1
:10C7F0009A00384B13445B7C13F00C0F3FD0364A41
:10C8000006F10C0152F821300693069B43F04F03CA
:10C810000693069B43F010030693069B42F82130D3
:10C8200000238DF8033006E000BF9DF8033001338C
:10C83000DBB28DF803309DF80330DBB2132BF3D954
:10C84000254A06F10C0152F821300793079B43F06B
:10C850004F030793079B23F001030793079B42F8BD
:10C86000213006F10C031C4A52F8233013F0010F5B
:10C87000F7D1002120461B4B98470120BFE0002C38
:10C880004AD0032C48D001212046164B984758B374
:10C89000114A06F10C0152F821300893089B43F02D
:10C8A0004F030893089B23F001030893089B42F869
:10C8B000213006F10C03084A52F8233013F0010F1F
:10C8C000F7D100212046074B9847012097E000BF91
:10C8D00029C540008C0E0020004004402F0300209A
:10C8E000E9C1400035C440004749BB00D819820067
:10C8F0000A4492F811E06FF3C71E82F811E0D26883
:10C900001F44BB0019448A60404B5D6122460021F0
:10C9100040463F4B9847BBE7012120463D4B984797
:10C920003A4A06F10C0152F821300993099B43F071
:10C930004F030993099B23F001030993099B42F8D4
:10C94000213006F10C03314A52F8233013F0010F65
:10C95000F7D1012053E00134E4B2052C4ED82B4B23
:10C960009B6926460125A5402B42F4D0671E07EBA4
:10C9700087029300244A02EB030804F10C03234AC4
:10C9800052F8233013F0420F7FF439AE04F10C0358
:10C990001E4A52F8233013F0010F7FF435AE04F134
:10C9A0000C031A4A52F8233013F0080FD3D004F1C5
:10C9B0000C0152F821300A930A9B43F04F030A936B
:10C9C0000A9B23F008030A930A9B42F8213006F1E0
:10C9D0000C030E4A52F8233013F0080FF7D106F17A
:10C9E0000C0352F8233003F4E063B3F5807F09D0E1
:10C9F00006F10C0352F82330012000E000200CB0B7
:10CA0000BDE8F0810120FAE78C0E002000400440D0
:10CA1000E9C1400035C4400000B587B0534B1B78D6
:10CA2000E3B9534B1B6BC3F30A43082B3BD0504A6B
:10CA3000136B0193019B43F04F030193019B23F080
:10CA400004030193019B1363494B1B6B13F0040F09
:10CA5000FAD1484B984707B05DF804FB464B98471E
:10CA6000464B9847DDE7424A116D454A99540133D8
:10CA7000DBB2072BF7D9434B9847B0B93C4A136B4D
:10CA80000293029B43F04F030293029B23F00403A3
:10CA90000293029B1363364B1B6B13F0040FFAD106
:10CAA000344B9847D7E70023E3E7354B93F9003041
:10CAB000002B1EDB2E4A136B0593059B43F04F039F
:10CAC0000593059B23F004030593059B1363284BF3
:10CAD0001B6B13F0040FFAD1294BDB88002B42D0DB
:10CAE0000023294A1380294A138001221F4B1A7000
:10CAF000B1E71F4A136B0393039B43F04F03039368
:10CB0000039B43F080030393039B136300238DF87F
:10CB1000033006E000BF9DF803300133DBB28DF82F
:10CB200003309DF80330DBB2132BF3D9104A136B9B
:10CB30000493049B43F04F030493049B23F00403EA
:10CB40000493049B13630A4B1B6B13F0040FFAD17D
:10CB500000230D4A13800D4A13800222034B1A70E2
:10CB60000B4B984777E70B4B984774E78A0E0020EA
:10CB7000004004405DBD400009BE400045BD40008E
:10CB8000102300209DB94000880E0020860E002052
:10CB900019BE4000ADBD4000204BDB6913F0010F12
:10CBA00037D000B583B01D4B1B6B13F0040F24D19D
:10CBB0001A4B1B6B13F0010F23D1184B1B6B13F097
:10CBC000020F22D1154B1B6B13F0080F23D0134A11
:10CBD000136B0193019B43F04F030193019B23F0DF
:10CBE00008030193019B13630C4B1B6B13F0080F9D
:10CBF000FAD1012003B05DF804FB094B98470120EE
:10CC0000F8E7084B98470120F4E7074B98470120C5
:10CC1000F0E7002070470020ECE700BF0040044030
:10CC200019CA400019BE4000F1BF400010B54C4B7E
:10CC3000984720B94B4BDB6913F4807F10D030202C
:10CC4000494B9847474B9B6913F4006F04D0454B01
:10CC5000DB6913F4006F0AD1444B984770B110BDE3
:10CC600072B6BFF35F8F0022414B1A7010BD4FF4B4
:10CC700000623C4B1A623F4B984710BD3E4B9847B1
:10CC80000028ECD1374B9B6913F4005F04D0354B7F
:10CC9000DB6913F4005F3DD1324B9B6913F4007FD5
:10CCA00004D0304BDB6913F4007F33D12D4B9B69EB
:10CCB00013F4806F04D02B4BDB6913F4806F29D100
:10CCC000284B9B6913F4807F04D0264BDB6913F457
:10CCD000807F2FD1234BDB6913F4805FBFD0214CC1
:10CCE0004FF480532362254B9847254B9847636840
:10CCF00023F001036360636823F002036360214B48
:10CD00009847214B98474FF4807323614FF4006399
:10CD10002361A4E7134C4FF418532362636101208D
:10CD20001A4B98474FF48073236223614FF40063DA
:10CD3000236110BD0B4B4FF480721A625A614FF49D
:10CD400000521A614FF400721A614FF480621A6146
:10CD500030200F4B984700200C4B984710BD00BF68
:10CD6000CDDD40000040044095DC400099CB400000
:10CD70002F03002065B94000F5C5400029C24000DE
:10CD800079B7400091BC400045BD4000EDBB40007C
:10CD9000E9DC400010B582B0EFF31083B3FA83F3FF
:10CDA0005B09019372B6BFF35F8F0022144B1A70B8
:10CDB000019C0120134B98473020134B9847134B8D
:10CDC0005A6F22F480725A675A6F42F400725A679F
:10CDD0004FF480721A614FF400521A614FF40072DE
:10CDE0001A614FF480621A614FF400621A612CB12B
:10CDF0000122034B1A70BFF35F8F62B602B010BD01
:10CE00002F030020EDBB400095DC400000400440B3
:10CE100030B583B0EFF31083B3FA83F35B0900936B
:10CE200072B6BFF35F8F0024204B1C70009D204B17
:10CE3000984730201F4B98471F4B98471F4B502255
:10CE400083F830234FF480325A601D4B98474FF4DB
:10CE500080201C4B98471C4B1C701C4B1B78FF2BD5
:10CE600022D0EFF31083B3FA83F35B09019372B618
:10CE7000BFF35F8F00220D4B1A700199134A13788C
:10CE80000133137029B10122084B1A70BFF35F8F71
:10CE900062B60F4B98472DB10122044B1A70BFF3B5
:10CEA0005F8F62B603B030BDFEE700BF2F030020E6
:10CEB00099D6400095DC400081D8400000E100E0B8
:10CEC000B1C14000B9DD4000850E002028230020BC
:10CED00095CD400008B5064B5A6F42F480725A67F0
:10CEE0005A6F22F400725A670020024B984708BD1F
:10CEF00000400440EDBB400010B582B0EFF310835A
:10CF0000B3FA83F35B09009372B6BFF35F8F00221D
:10CF1000144B1A70009C144B9847144B1B7803B9A0
:10CF2000FEE7EFF31083B3FA83F35B09019372B664
:10CF3000BFF35F8F00220B4B1A7001990B4A1378D5
:10CF4000013B137029B10122064B1A70BFF35F8FAA
:10CF500062B62CB10122034B1A70BFF35F8F62B629
:10CF600002B010BD2F030020D5CE400028230020A2
:10CF70000D4B5A6822F001025A609A6822F48072BE
:10CF80009A60024670B1986820F07F0002F07F023C
:10CF9000104398609A6842F480729A605A6842F02E
:10CFA00001025A60704700BF00400440054B5B68B7
:10CFB00013F0010F04D0034B986800F07F00704716
:10CFC0000020704700400440014B986099817047F1
:10CFD00010230020F0B583B045B200F00F00052803
:10CFE00073D801F00306044600F10C033B4F57F8D9
:10CFF000233013F4004F6BD1012E53D0031FDBB24B
:10D00000012B54D94023934266DB461E06EB86076C
:10D01000334B03EB870303F11007B3F810E062F31F
:10D02000090EA3F810E05B7C03F07F036FF3451358
:10D030007B70002D3EDB294EB36A012282401343F0
:10D04000B362264B9B6A1A42FBD0244B9E6A26EAA7
:10D0500002029A6200F10C0253F822300193019B04
:10D0600043F04F030193019B23F4074323F0800314
:10D070000193002D23DB0A0202F4407242F40042C5
:10D08000019B1343019301990C30144B43F820107A
:10D0900004F10C03114951F8233032EA0303F7D1AC
:10D0A000012013E0B0B10328A8D100200EE04FF416
:10D0B0000073A8E77B786FF383037B70BBE70A02FA
:10D0C00002F4407242F40442DAE7002003B0F0BDFB
:10D0D0000020FBE70020F9E70020F7E700400440CC
:10D0E0008C0E002000F00F03052B1ED810B582B067
:10D0F00019460E4C0C3354F823200192019A42F049
:10D100004F020192019A22F400420192019A44F8DE
:10D11000232001F10C03054A52F8233013F4004F89
:10D12000F7D1034B984702B010BD70470040044050
:10D1300055C2400000F00F00431E052815D803EB30
:10D1400083039A000A4B13445B7C13F0200F08D131
:10D150000C30084B53F8203013F0280F03D0012077
:10D16000704701207047002070470020704700BFC3
:10D170008C0E00200040044010B485B044B200F092
:10D180000F00052865D8421EEFF31083B3FA83F32E
:10D190005B09039372B6BFF35F8F0021314B1970A7
:10D1A0000399002C14DB304A00F10C0452F82430AF
:10D1B0000293029B43F04F030293029B43F0200330
:10D1C0000293029B42F8243000238DF807302EE0B2
:10D1D00000F10C03244C54F8233013F0100F09D144
:10D1E00002EB82039C00214B23445B7CC3F381034D
:10D1F000012BD8DD02EB820294001C4B23445A7CA5
:10D2000042F020025A74012303FA00F0164B186111
:10D2100021B30120134B1870BFF35F8F62B619E082
:10D2200000BF9DF807300133DBB28DF807309DF861
:10D230000730DBB2132BF3D9012303FA00F00A4BBA
:10D24000186169B10120074B1870BFF35F8F62B698
:10D2500000E0002005B05DF8044B70470120F9E7BD
:10D260000120F7E72F030020004004408C0E00202F
:10D2700000F00F0005286CD830B583B00246441E7C
:10D2800004EB84039900354B0B44597C6FF3451133
:10D29000597400F10C03324951F8233013F0200F78
:10D2A00059D000F10C0551F825300093009B43F054
:10D2B0004F030093009B23F020030093009B41F851
:10D2C000253002F10C03264951F8233013F0200FCA
:10D2D000F7D10D468B6A012181400B43AB62204B95
:10D2E0009B6A1942FBD01E4B9D6A25EA0101996297
:10D2F0000C3053F820100191019941F04F01019138
:10D30000019921F008010191019943F8201002F1DF
:10D310000C03134951F8233013F0080FF7D104EB35
:10D3200084039A000D4B13445B7C13F0100F01D162
:10D33000012011E00949A200101983000B44587C18
:10D340006FF3041058741444A300CB58984701207D
:10D3500002E000207047012003B030BD8C0E002099
:10D3600000400440F0B583B000F00F04052C00F23B
:10D37000A28047B2651E04F10C00554E56F82000FD
:10D3800010F4004F00F09A8005EB8500514E06EB3B
:10D390008000407C10F0200F40F0928004F10C00DF
:10D3A0004B4E56F8200010F0200F40F08B80EFF32A
:10D3B0001080B0FA80F04009009072B6BFF35F8F22
:10D3C000002645480670DDF800E005EB8500414E7B
:10D3D00006EB8000407C10F0100F0AD0BEF1000F69
:10D3E00072D001223C4B1A70BFF35F8F62B60020EF
:10D3F00062E005EB8500374E06EB8000467C46F088
:10D4000010064674BEF1000F05D0012632480670A2
:10D41000BFF35F8F62B6DFF8BCE005EB85008000EC
:10D420000EEB00067260B3600022F260089A4EF8BC
:10D43000002011B95BBB012000E00120254AA900B2
:10D440004B1902EB83035B7C60F386130D4402EB04
:10D4500085026FF3C7135374EFF31083B3FA83F3AA
:10D460005B09019372B6BFF35F8F00221A4B1A70EB
:10D47000019D0123A340164A1361002F09DB2DB340
:10D480000120154B1870BFF35F8F62B614E00020C7
:10D49000D4E704F10C0352F8233013F0110FEED14E
:10D4A000012120460D4B98470028E8D00021204656
:10D4B0000A4B9847E3E7002003B0F0BD0020FBE7EC
:10D4C0000020F9E70020F7E70020F5E70120F3E767
:10D4D000004004408C0E00202F03002035C4400083
:10D4E00070B586B000F00F04052C00F2C98042B27E
:10D4F000EFF31083B3FA83F35B09059372B6BFF3BE
:10D500005F8F00215F4B1970059B26460125A540C2
:10D510005D494D612BB101215A4B1970BFF35F8FEB
:10D5200062B6002A80F2948004F10C03564A52F845
:10D53000233013F0100F64D0002C49D0032C47D0B7
:10D5400004F10C0152F821300193019B43F04F0389
:10D550000193019B23F010030193019B42F82130BA
:10D5600006F10C03484A52F8233013F0100FF7D19C
:10D5700006F10C03444A52F8233013F0100FF7D190
:10D5800004F10C0152F821300293029B43F04F0347
:10D590000293029B43F010030293029B42F8213056
:10D5A00000238DF8033006E000BF9DF803300133FF
:10D5B000DBB28DF803309DF80330DBB2132BF3D9C7
:10D5C00006F10C03304A52F8233013F0100FF7D055
:10D5D0002D4A04F10C0152F821300393039B43F0D0
:10D5E0004F030393039B23F010030393039B42F821
:10D5F000213006F10C03244A52F8233013F0100FA7
:10D60000F7D1214A04F10C0152F821300493049B14
:10D6100043F04F030493049B23F001030493049B02
:10D6200042F8213006F10C03174A52F8233013F068
:10D63000010FF7D1621E02EB82029100134B0B44E3
:10D640005A7C6FF383025A740AE02046104B9847C5
:10D6500006F10C030C4A52F8233013F0420FF4D1B8
:10D66000094A936A2B439362074B9B6A1D42FBD086
:10D67000054A936A23EA050595622046054B9847BB
:10D6800006B070BD2F030020004004408C0E002027
:10D6900079C2400055C24000064BD3F8142122F451
:10D6A0004062C3F81421D3F8202142F00102C3F8EC
:10D6B0002021704700020E400B4619B10968016035
:10D6C0005B6843601AB11368036153684361704734
:10D6D00021F0FE01C905C90D0162704710B51E4B4E
:10D6E00053F820402268536A13F0805F11D0022360
:10D6F000C2F8203123684FF0FF32DA61002323752E
:10D70000236913F0010F26D0636823B3204698479E
:10D7100010BD13F0006F13D00223C2F8203123682C
:10D720004FF00062DA61236913F0020F03D0A3689F
:10D730000BB12046984723680122C3F8202110BD71
:10D7400013F0007F07D0236913F0040F03D0E368C0
:10D750000BB12046984710BDF00E002008B5002000
:10D76000014B984708BD00BFDDD6400008B5012039
:10D77000014B984708BD00BFDDD6400070B5054697
:10D780000E461446016001230B60214B99422BD0B9
:10D790000D20204B9847204B1D6023781B0203F47B
:10D7A000FE43736063782BBB0022A3780BB142F079
:10D7B0000402E3780BB142F0080223790BB142F086
:10D7C000100263791B0203F47063A179090389B223
:10D7D0000B431343B3652389C3F30E03628943EA02
:10D7E0000243F36500230CE012200A4B98470A4BD2
:10D7F0005D60D2E70222D8E705EB83020021516089
:10D800000133022BF8D900202861287570BD00BFB4
:10D810000000034095DC4000F00E002012F0100FD5
:10D8200012D0C0F8B01012F0200F07D0C0F8D410FA
:10D8300012F0400F05D0C0F8C0107047C0F8D010EB
:10D84000F6E7C0F8C4107047C0F8B4107047016420
:10D85000704741647047C06C7047806C70474009E6
:10D8600000F5001000F207704002704740090B30CD
:10D87000704700F01F00012303FA00F0704700001A
:10D8800008B500200A4B98470A4B98470028FBD060
:10D89000094B9847094A0A4BDA620A4B9847002815
:10D8A000FBD00020084B9847084B984708BD00BFA5
:10D8B00011DC400035DC400079DC4000013FB80558
:10D8C00000040E4085DC400099DD4000ADDD4000E5
:10D8D00010B5A2B01848194B98470020184B98472C
:10D8E000184B98470028FBD0174B9847174A184BFE
:10D8F0009A62184B98470028FBD00020164B984797
:10D90000164B984716480D4B9847164B1A68164BFE
:10D910001344164A934201D922B010BD202300932C
:10D9200002AB0F220E211248124CA047BDF848103E
:10D930001148124B9847EFE7000E27071DE1400002
:10D9400011DC400035DC40005DDC4000013FB70BDE
:10D9500000040E4069DC4000BDDB400029E04000CF
:10D960000000DC0530030020C0D3BDF980C3C9012D
:10D97000000A0E401100002010140E40DDDD4000B2
:10D9800070B50D461446064658B14FF0FF360AE012
:10D99000064B1868064B1B68294698470135013627
:10D9A000013C002CF4DC304670BD00BF3823002061
:10D9B0003023002070B5013802280FD81446002506
:10D9C0008CB10A4B18684E1C094B1B6809789847A4
:10D9D000002806DB0135013C3146F1E74FF0FF3509
:10D9E00001E04FF0FF35284670BD00BF382300200E
:10D9F00034230020A1F10E03012B02D84FF0FF3099
:10DA0000704710B582B0EFF31083B3FA83F35B096C
:10DA1000019372B6BFF35F8F00240B4B1C70019C07
:10DA2000120222F07F4222F0FF02C9B2114341F0FC
:10DA3000B441064B98472CB10122034B1A70BFF337
:10DA40005F8F62B602B010BD2F0300207900002066
:10DA50004C4B1B78FF2B31D000B583B0EFF3108314
:10DA6000B3FA83F35B09019372B6BFF35F8F0022B1
:10DA7000454B1A700199434A13780133137029B149
:10DA80000122414B1A70BFF35F8F62B63F4A90424A
:10DA900015D03F4A904220D03E4A90422BD03E4A79
:10DAA000904236D03D4A904241D03D4A90424CD0BF
:10DAB0003C4A904257D003B05DF804FBFEE71620C5
:10DAC000394B98470720394B984700210720384B9E
:10DAD00098470720374B9847EDE71520324B98477A
:10DAE0000720324B984700210720314B98470720E9
:10DAF000304B9847DFE714202B4B984707202B4BE0
:10DB00009847002107202A4B98470720294B984720
:10DB1000D1E71320244B98470620244B9847002137
:10DB20000620234B98470620224B9847C3E70E2038
:10DB30001D4B984706201D4B9847002106201C4B83
:10DB4000984706201B4B9847B5E70920164B984786
:10DB50000620164B984700210620154B98470620B3
:10DB6000144B9847A7E708200F4B984706200F4B08
:10DB70009847002106200E4B984706200D4B9847EA
:10DB800099E700BF282300202F0300200000044055
:10DB90000080004000C00140008001400040024081
:10DBA0000000024000C0004095DC400085DD4000E0
:10DBB0003DDD400071DD400001607047134A136B8A
:10DBC00023F07003184310634FF400630F4A926E02
:10DBD00012F0080F02D1A3B1013BF7E70B4A136B18
:10DBE00023F0030343F0020313634FF40063074A77
:10DBF000926E12F0080F02D12BB1013BF7E7002023
:10DC00007047012070470120704700BF00040E409C
:10DC1000012803D0054A064B1A607047044A9368EE
:10DC200043F0254343F480139360F3E7080000A515
:10DC300010140E40074B5B6913F0800F06D0064BA3
:10DC40009B6E13F0800F03D10020704700207047B7
:10DC50000120704710140E4000040E400022014BBA
:10DC60009A62704700040E40024B986E00F002006A
:10DC7000704700BF00040E400022014BDA6270477B
:10DC800000040E40024B986E00F00400704700BF85
:10DC900000040E4032281ED81F280CD8114B9A6958
:10DCA00001238340934318D0012303FA00F00D4B66
:10DCB00018610020704720380A4BD3F8082101234F
:10DCC000834093430BD0012303FA00F0054BC3F8C4
:10DCD000000100207047012070470020704700209D
:10DCE000704700BF00040E40322822D81F280ED8EB
:10DCF000114B9A6901238340934301D00020704760
:10DD0000012303FA00F00C4B5861002070472038C3
:10DD1000094BD3F8082101238340934301D000200D
:10DD20007047012303FA00F0034BC3F804010020FD
:10DD300070470120704700BF00040E4041F004010D
:10DD400000F11002094B43F822104FF40062074B18
:10DD5000996E4FF480738340194202D11AB1013A8F
:10DD6000F5E7002070470120704700BF00040E4017
:10DD70004FF4807303FA00F0014B1860704700BF46
:10DD800000040E404FF4807303FA00F0014B58601A
:10DD9000704700BF00040E40000200F4706040F0C5
:10DDA0000100014B9863704700040E408022014B34
:10DDB0001A60704700040E40C0F31200024B1A6F45
:10DDC00010431867704700BF00040E40024B1878DC
:10DDD00080F00100704700BFF80E0020C36923F4F3
:10DDE000F053490201F4F051194341F0B44141F4B8
:10DDF0008071C161704730B4B2EB011F17D310249A
:10DE000001FB04F14B0803EBC202B2FBF1F2D308B1
:10DE10005D1E4FF6FE718D4210D8082C09D01204F9
:10DE200002F4E0221A430262002030BC704708244A
:10DE3000E6E7416841F400214160F0E70120F4E7A2
:10DE400040230360704788230360704710230360FA
:10DE500070472423036070474FF48073036070475A
:10DE60004FF4002303607047436913F0020F04D09E
:10DE7000C1F30801C1610020704701207047436968
:10DE800013F0020FFBD0C1F30801C16100207047FD
:10DE9000436913F0010F05D08369C3F308030B60D6
:10DEA0000020704701207047014BC0F8E4307047F4
:10DEB0000041535510B50446094B98470023636051
:10DEC0006362A3622046074B98472046064B98475B
:10DED0002046064B98472046054B984710BD00BF8B
:10DEE000A9DE400047DE400053DE400059DE40001E
:10DEF00061DE400070B505460C461646104B98474B
:10DF00000022104B1A60B4B13246216828460E4BED
:10DF10009847024688B96368A1680B4321690B439F
:10DF2000E1680B430749086803430B6069680B43CA
:10DF30006B60104670BD0122FBE70122F9E700BFCC
:10DF4000B5DE4000FC0E0020F7DD400000B583B0D8
:10DF5000234B244A9A4209D0214B224A03E01168FC
:10DF600019600433043220498B42F8D31F4B02E07E
:10DF700000221A6004331E4A9342F9D31D4A22F04C
:10DF80007F011D4B9960EFF31083B3FA83F35B09B4
:10DF9000019372B6BFF35F8F0021184B197001987F
:10DFA00017490B6843F470030B60BFF34F8FBFF347
:10DFB0006F8F28B10121114B1970BFF35F8F62B6CB
:10DFC00002F16042B2F5203F04D20B4A936843F05D
:10DFD000005393600B4B98470B4B9847FEE700BFED
:10DFE0001000002074504100E80C0020E80C0020D4
:10DFF0001C2400200040400000ED00E02F03002022
:10E0000088ED00E005134100AD02410008B5012094
:10E01000034B9847EFF30580024B9847FFDE00BFA4
:10E02000854D4000914D4000344B1B6B03F00303C2
:10E03000012B20D083B1022B39D0304B1B6B03F066
:10E040007003702B51D02D4B1A6BC2F302122C4966
:10E050000B68D3400B6070472A4B5B6913F0800F4D
:10E0600004D04FF40042264B1A60E6E74FF4FA4220
:10E07000234B1A60E1E7214B1B6A13F0807F03D02A
:10E08000214A1F4B1A60D8E7204A1D4B1A601B4BD0
:10E090001B6A03F07003102B05D0202BCDD11C4A36
:10E0A000174B1A60C9E71B4A154B1A60C5E7154B99
:10E0B0005B6913F0800F13D04FF40042104B1A60CD
:10E0C0000E4B1B6B03F00303022BB6D10B4B9A6A6A
:10E0D000C2F30C420A490B6802FB03330B60ACE746
:10E0E0004FF4FA42064B1A60EAE7054A13680A49F8
:10E0F000A1FB03135B081360704700BF00040E40D0
:10E100003003002010140E40001BB70000127A00EC
:10E1100000366E010024F400ABAAAAAA144B984260
:10E120000FD9144B984211D9134B984212D9134B63
:10E13000984213D9124B984214D9124A124B1A60C2
:10E1400070474FF08062104B1A6070470F4A0E4BB9
:10E150001A6070470E4A0C4B1A6070470D4A0A4B02
:10E160001A6070474FF00422074B1A60704700BFD7
:10E17000FF2C3101FF596202FF869303FFB3C404F1
:10E18000FFE0F50500050004000A0E400001000450
:10E1900000020004000300040A4B1B6853B1094B42
:10E1A0001B681A180849914208DB1046054A10609E
:10E1B00018467047054A034B1A60F0E74FF0FF30EE
:10E1C000704700BF000F0020FC7F02202054002079
:10E1D0004FF0FF3070474FF400534B600020704702
:10E1E000012070470020704700F1080343604FF0A2
:10E1F000FF328260C3600361002303607047002325
:10E200000361704743684B609A688A609A685160FE
:10E2100099600861036801330360704730B40D688A
:10E22000B5F1FF3F02D000F1080202E0026904E00C
:10E230001A4653681C68A542FAD253684B6099602D
:10E240008A605160086103680133036030BC704725
:10E2500003694268816891608268416851605A68C8
:10E26000904206D0002202611A68013A1A601868CA
:10E27000704782685A60F5E782B0002301934FF03F
:10E28000500383F31188BFF36F8FBFF34F8F019B50
:10E29000002BFCD002B0704708480068006880F38B
:10E2A00008884FF0000080F3148862B661B6BFF3AF
:10E2B0004F8FBFF36F8F00DF00BF000008ED00E05D
:10E2C000DFF80C00016841F4700101607047000044
:10E2D00088ED00E04FF0807340F8043C21F001012C
:10E2E00040F8081C054B40F80C3C40F8202C6FF01F
:10E2F000020340F8243C4438704700BF79E24000F4
:10E30000074B19680868B0E8F04F80F30988BFF33D
:10E310006F8F4FF0000080F311887047AFF30080DB
:10E32000040F00204FF0500383F31188BFF36F8F69
:10E33000BFF34F8F024A136801331360704700BF69
:10E3400034030020034A1368013B13600BB983F3C5
:10E350001188704734030020000000000000000016
:10E36000EFF30980BFF36F8F154B1A681EF0100F83
:10E3700008BF20ED108A20E9F04F10602DE9090058
:10E380004FF0500080F31188BFF34F8FBFF36F8FB2
:10E3900000F07CFF4FF0000080F3118809BC196881
:10E3A0000868B0E8F04F1EF0100F08BFB0EC108AFC
:10E3B00080F30988BFF36F8F704700BFAFF3008011
:10E3C000040F002008B54FF0500383F31188BFF30A
:10E3D0006F8FBFF34F8F054B984718B14FF08052A6
:10E3E000034B1A60002383F3118808BD09F0400035
:10E3F00004ED00E0054B00221A6005490A6005495A
:10E40000054A116007221A60704700BF10E000E063
:10E4100018E000E0FF7F010014E000E010B50E4BB3
:10E420001A6842F470021A601A6842F070421A6068
:10E430000A4B984700240A4B1C600A4B98470A4A2B
:10E44000136843F040431360084B9847084B9847C4
:10E45000084B9847204610BD20ED00E0F5E3400052
:10E4600034030020C1E2400034EF00E099E24000B4
:10E470008DF2400079E2400010B50446044B984705
:10E480002046044B98470446034B9847204610BD4E
:10E49000EDEF40007D134100FDF0400048B110B5A4
:10E4A0000446044B98472046034B9847034B984734
:10E4B00010BD7047EDEF40008D134100FDF04000AE
:10E4C000436A23B1036B1868C0F105007047002050
:10E4D0007047000010B50446064B9847A26BE36BEB
:10E4E0009A4204D00024044B9847204610BD0124D2
:10E4F000F9E700BF25E3400045E3400010B50446BE
:10E50000054B9847A36B23B10024044B9847204642
:10E5100010BD0124F9E700BF25E3400045E34000BA
:10E5200070B504461646856B026C5AB903681BB178
:10E5300000200135A56370BD4068174B9847002344
:10E540006360F6E76EB98068144B9847226CA36845
:10E550001344A3606268934219D32368A360002028
:10E56000E7E7C0680D4B9847226C5242E3681344BA
:10E57000E36021688B4202D263681A44E260022E93
:10E5800001D00020D5E725B1013D0020D1E70020D2
:10E59000CFE70020CDE700BF9DF54000011A410004
:10E5A000026C72B110B5C3681344C3604468A342DF
:10E5B00001D30368C3600C46C1682046014B9847ED
:10E5C00010BD7047011A410038B505461A4B9847EF
:10E5D00095F8454064B201E0013C64B2002C0ADDCC
:10E5E0006B6A43B105F12400144B98470028F3D01F
:10E5F000134B9847F0E7FF2385F84530114B9847B8
:10E600000D4B984795F8444064B201E0013C64B278
:10E61000002C0ADD2B6943B105F11000074B984728
:10E620000028F3D0064B9847F0E7FF2385F84430E5
:10E63000044B984738BD00BF25E3400091F34000EC
:10E640008DF4400045E3400038B504460D46144BB8
:10E6500098472168E26B236C03FB02106060002086
:10E66000A063A160013A02FB0313E360FF2384F877
:10E67000443084F8453055B923691BB9094B984794
:10E68000012038BD04F11000074B9847F6E704F16C
:10E690001000064DA84704F12400A847EEE700BF8C
:10E6A00025E3400045E3400091F34000E9E14000EC
:10E6B00038B51D46049C0B4649B12260E0632364D3
:10E6C00001212046034B984784F84C5038BD246004
:10E6D000F4E700BF49E64000F0B583B005461746B1
:10E6E0000E4689B100FB01F05030084B98470446B4
:10E6F00038B100903B4600F1500231462846044DA7
:10E70000A847204603B0F0BD0020EDE779E44000C3
:10E71000B1E64000F0B585B004460F4601921E46B2
:10E72000002526E0324639462046354B9847636A35
:10E7300023B9344B9847012005B0F0BD04F1240003
:10E74000314B9847F5E72F4B98470020F4E702A894
:10E750002E4B9847012519E0002384F8443021E02E
:10E76000002384F8453023E02046294B9847294B65
:10E770009847294B9847A26BE36B9A42D2D3022E5B
:10E78000D0D0019B002BDED0002DE0D01D4B984750
:10E79000224B9847204B984794F844305BB2B3F132
:10E7A000FF3FD9D094F845305BB2B3F1FF3FD7D0EB
:10E7B000144B984701A902A8194B9847C8B920469D
:10E7C000184B98470028CFD0019904F11000164B40
:10E7D000984720460E4B98470E4B98470028C8D1C3
:10E7E0004FF08052114B1A60BFF34F8FBFF36F8F02
:10E7F000BFE72046064B9847064B984700209BE70B
:10E8000021E5400045E3400091F3400011F4400051
:10E81000C9E54000FDF0400025E34000EDEF400079
:10E8200029F44000D5E4400041F3400004ED00E04D
:10E8300048B110B5002141600160C1600B460A4635
:10E84000014CA04710BD704715E7400010B50246C7
:10E8500000210120034B98470446034B984720466C
:10E8600010BD00BFD9E6400031E84000F8B5EFF335
:10E8700011864FF0500484F31188BFF36F8FBFF3FC
:10E880004F8F856BC46BA54205D3022B03D00020AC
:10E8900086F31188F8BD1746054690F8454064B2E6
:10E8A0001A460E4B9847B4F1FF3F05D0013464B2CD
:10E8B00085F845400120EBE76B6A0BB90120E7E7DB
:10E8C00005F12400064B984718B127B101203860A4
:10E8D000DEE70120DCE70120DAE700BF21E54000A8
:10E8E00091F34000F0B585B004460F460192002632
:10E8F00032E039462046384B9847013DA5632369ED
:10E9000023B9364B9847012005B0F0BD04F1100043
:10E91000334B9847F5E7314B98470020F4E702A8BE
:10E92000304B9847012621E0002384F8443029E049
:10E93000002384F845302BE020462B4B98472B4B87
:10E94000984709E02046284B9847284B984720468F
:10E95000274B984700283DD1264B9847A56B002DA3
:10E96000C7D1019B002BD6D0002ED8D01B4B984787
:10E97000214B98471F4B984794F844305BB2B3F152
:10E98000FF3FD1D094F845305BB2B3F1FF3FCFD019
:10E99000124B984701A902A8184B98470028D1D1DB
:10E9A0002046134B98470028C6D0019904F1240053
:10E9B000134B984720460C4B98470C4B9847002820
:10E9C000CAD14FF080520F4B1A60BFF34F8FBFF385
:10E9D0006F8FC1E7002097E7A1E5400045E34000C5
:10E9E00091F3400011F44000C9E54000FDF0400003
:10E9F000FDE4400025E34000EDEF400029F4400035
:10EA000041F3400004ED00E070B584B0044601918C
:10EA1000002635463EE0013BA36323683BB12369F2
:10EA20004BB9444B98470126304604B070BD424B69
:10EA300098476060F3E704F11000404B9847F0E717
:10EA40003C4B98470026EFE702A83D4B984701252D
:10EA50002AE0002384F8443032E0002384F8453073
:10EA600034E0384B98476068374B98470646314B3F
:10EA700098473BE02046354B9847354B984709E08F
:10EA80002046324B9847324B98472046314B9847A7
:10EA9000002840D12B4B9847A36B002BBBD1019B87
:10EAA000002BCDD0002DCFD0224B98472A4B984732
:10EAB000244B984794F844305BB2B3F1FF3FC8D081
:10EAC00094F845305BB2B3F1FF3FC6D0194B98477D
:10EAD00001A902A8214B98470028D1D120461D4BFF
:10EAE00098470028C6D02368002BBAD0019904F1BA
:10EAF00024001B4B98472046144B9847144B9847CB
:10EB00000028C7D14FF08052164B1A60BFF34F8FC9
:10EB1000BFF36F8FBEE7002E86D00A4B9847204682
:10EB2000114B984701466068104B9847014B984736
:10EB3000002679E745E34000C5F6400091F3400028
:10EB400011F4400025E34000D5F44000C9E5400041
:10EB5000FDF04000FDE44000EDEF400029F44000EE
:10EB600041F3400004ED00E0C1E4400025F6400020
:10EB70000023092B0CD8074A52F833200AB101337D
:10EB8000F7E7044A42F8331002EBC30358607047BA
:10EB9000704700BF3C23002070B504460D46164662
:10EBA000124B984794F844305BB2B3F1FF3F0DD05D
:10EBB00094F845305BB2B3F1FF3F0BD00C4B984754
:10EBC000A36B5BB120460B4B984770BD002384F8C4
:10EBD0004430EDE7002384F84530EFE7324629461C
:10EBE00004F12400044B9847ECE700BF25E3400004
:10EBF00045E34000C9E5400065F34000F0B5036817
:10EC00004BB343685B68436000F10807BB4204D024
:10EC10004368D3F80CE0002609E05B684360F7E73F
:10EC20005B68436008E02E46B6B9AE4514D0436831
:10EC30005B6843609F42F3D04368DD6800230F2B7D
:10EC4000F2D8EA1892F83420CC5CA242ECD1002A27
:10EC5000E9D00133F3E700263046F0BD002301E0A0
:10EC6000013001330278A52AFAD0C3F38F00704730
:10EC70000A4B1B681B684BB901234BB9074B1B6838
:10EC8000DB68DB685A68064B1A6070470023F4E7BC
:10EC90004FF0FF32024B1A60704700BF080F002090
:10ECA000B40F00202DE9F84F81460D4617469A46CD
:10ECB0000A9EDDF82C800C9C9200A521206B1D4B38
:10ECC0009847236B07F18042013A03EB820727F054
:10ECD000070700230F2B07D8E95CE21882F83410ED
:10ECE000EA5C0AB10133F5E7002384F84330042ECF
:10ECF00000D90426E662E66400252565201DDFF8BC
:10ED00003CB0D84704F11800D8472461C6F1050685
:10ED1000A6616462656584F8585052464946384693
:10ED2000054B98472060B8F1000F01D0C8F80040AB
:10ED3000BDE8F88FFD1B4100D5E24000FFE1400037
:10ED400070B5002407E004EB840293000B481844DC
:10ED50000B4B98470134042CF5D90A4E3046084C29
:10ED6000A047094D2846A0470848A0470848A047A3
:10ED7000084B1E60084B1D6070BD00BF100F0020C7
:10ED8000E9E14000880F00209C0F0020BC0F00200C
:10ED9000D40F0020080F00200C0F002010B50446EF
:10EDA0001C4B98471C4A1368013313601B4B1B68AC
:10EDB000002B26D01A4B1B683BB9184B1B68DA6A2C
:10EDC000E36A9A4201D8154B1C60164A1368013356
:10EDD00013606364E36A01229A401349086802439E
:10EDE0000A6003EB83039A00211D10481044104B66
:10EDF0009847104B98470A4B1B680BB1074B1B6891
:10EE000010BD064B1C601368012BDED10A4B9847DE
:10EE1000DBE700BF25E34000740F0020040F002053
:10EE2000D00F0020800F0020840F0020100F002042
:10EE300005E2400045E3400041ED400070B5044666
:10EE40000E461D4B1D681D4B186804301C4B98471F
:10EE500050B91A4B1B68DA6A012303FA02F2194906
:10EE60000B6823EA02030B60B4F1FF3F13D02C447C
:10EE7000124B1B685C60A54216D8134B18680F4BE9
:10EE800019680431114B9847114B1B689C4201D201
:10EE90000F4B1C6070BD002EE9D0084B196804317F
:10EEA0000C480D4B984770BD0C4B1868034B196804
:10EEB0000431064B984770BDE80F0020040F002076
:10EEC00051E24000840F0020080F00201DE24000A6
:10EED000B40F0020D40F002005E240000C0F0020EA
:10EEE00008B54FF08052044B1A60BFF34F8FBFF349
:10EEF0006F8F024B9847F4E704ED00E0E501410015
:10EF00002DE9F04385B006460F4615469846900019
:10EF1000144B984700B381465C20124B9847044637
:10EF2000B0B1C0F83090CCB10023039302940D9B94
:10EF300001930C9B009343462A46394630460A4DBE
:10EF4000A8472046094B9847012005B0BDE8F0834B
:10EF50004846074B9847E6E70024E4E74FF0FF30C8
:10EF6000F3E700BF79E44000A5EC40009DED4000D0
:10EF70009DE4400010B582B0134B01930023009331
:10EF8000462212491248134CA047012803D00128F9
:10EF900004D002B010BD104B9847F8E74FF0500373
:10EFA00083F31188BFF36F8FBFF34F8F4FF0FF32A2
:10EFB0000A4B1A6001220A4B1A600022094B1A60A0
:10EFC000094B9847E5E700BFB00F0020E44D410032
:10EFD000E1EE400001EF400059FB4000B40F00207B
:10EFE000D00F0020E80F00201DE44000024A136803
:10EFF00001331360704700BF7C0F0020014B18687D
:10F00000704700BFE80F002070B52F4B1B68002B26
:10F0100052D12E4B1E6801361E604EB12C4B1B6820
:10F020009E422FD22B4B1B68002B42D0002070BD7C
:10F03000294A1168294B186810601960284A13681A
:10F0400001331360274B9847E8E7012320E04FF096
:10F05000FF321F4B1A60E5E71D4A1360E2E704F137
:10F060001800214B9847E36A01229A401F4908681B
:10F0700002430A6003EB83039A0029461C481044AC
:10F080001C4B9847144B1B681B68002BDDD00023DA
:10F09000002BDCD1104B1B68DB68DC6863689E4288
:10F0A000DAD3251D2846104B9847A36A002BD6D1EA
:10F0B000D9E7114B9847B9E7064A13680133136043
:10F0C0000D4B9847B2E700BF7C0F0020E80F0020EF
:10F0D000B40F0020780F0020080F00200C0F002034
:10F0E000B80F002071EC400051E24000840F002076
:10F0F000100F002005E24000A902410070B5274B27
:10F100009847274B1A68013A1A601B68002B32D1C6
:10F11000244B1B68002B2ED00024234B1B6813B3F9
:10F12000214BDB68DC6804F11800204EB047251D38
:10F130002846B047E36A01229A401D490868024305
:10F140000A6003EB83039A0029461A4810441A4BBD
:10F150009847E26A194B1B68DB6A9A42DDD30122A9
:10F16000174B1A60D9E70CB1164B9847164B1C6821
:10F170003CB9134B1B68154B9847002070BD013CF0
:10F1800007D0134B98470028F9D001220C4B1A6086
:10F19000F5E700220C4B1A60EBE700BF25E34000C7
:10F1A0007C0F0020740F0020BC0F002051E24000B3
:10F1B000840F0020100F002005E24000040F002003
:10F1C000EC0F002071EC4000780F002045E3400078
:10F1D00009F0400010B550B9002038B94FF0805206
:10F1E000084B1A60BFF34F8FBFF36F8F10BD0446FB
:10F1F000054B984700212046044B9847044B9847FD
:10F20000EBE700BF04ED00E0EDEF40003DEE400015
:10F21000FDF0400070B50646154B98470524013CAB
:10F2200004EB84029300314612481844124B98476D
:10F23000054608B9002CF2D12DB15DB18DB10F4B4F
:10F240009847284670BD0E4B186831460A4B9847C0
:10F250000546F2E70B4B18683146074B98470546C1
:10F26000ECE731460848044B98470546E7E700BFFE
:10F27000EDEF4000100F0020FDEB4000FDF04000DE
:10F28000080F00200C0F0020D40F0020264B1B6815
:10F29000002B2FD110B50022244B1A60244B1B6881
:10F2A0001B6B1A68B2F1A53F28D0214B186819686A
:10F2B0003431204B9847204B1B68B3FA83F3DBB201
:10F2C000C3F11F031D489A00D418A10001444C68E3
:10F2D00064684C601A4491000831084484421AD092
:10F2E00003EB83039A00154B13445B68DA68104BF9
:10F2F0001A6010BD01220D4B1A6070475A68B2F1B6
:10F30000A53FD2D19A68B2F1A53FCED1DB68B3F167
:10F31000A53FCAD1CFE7606803EB83029100074A9B
:10F320000A445060DCE700BF7C0F0020EC0F002097
:10F33000040F0020A9014100840F0020100F0020BD
:10F3400010B50C46044B19681831044B984701213D
:10F350002046034B984710BD040F00201DE24000DB
:10F360003DEE400038B50D461446064B196818317D
:10F37000054B98470CB14FF0FF3521462846034B0B
:10F38000984738BD040F002005E240003DEE4000E4
:10F3900038B5C368DC6804F118052846144B984753
:10F3A000144B1B68E3B9251D2846114B9847E36AA7
:10F3B00001229A401049086802430A6003EB830364
:10F3C0009A0029460D4810440D4B9847E26A0D4BB0
:10F3D0001B68DB6A9A4208D901200B4B186038BDC4
:10F3E00029460A48064B9847F0E7002038BD00BF81
:10F3F00051E240007C0F0020840F0020100F0020FD
:10F4000005E24000040F0020EC0F0020BC0F00209C
:10F41000034B1B680360034B1B684360704700BFCE
:10F42000B80F0020E80F0020F8B504460D46124B37
:10F430009847124B19686268881A2B68B3F1FF3F2E
:10F4400016D027680E4E3668B74201D0914211D2CD
:10F45000984206D300232B6001240A4B984720468C
:10F46000F8BD1B1A2B602046074B98470024F4E791
:10F470000024F2E70124F0E725E34000E80F002034
:10F48000B80F002045E3400011F440000122014B79
:10F490001A607047EC0F002008B5034618B1186BCE
:10F4A000024B984708BD024B1B68F8E75DEC400033
:10F4B000040F0020054B1B6823B1054B1B681BB9CB
:10F4C000022070470120704700207047D00F0020B5
:10F4D0007C0F0020002854D038B50446C26A2A495F
:10F4E0000968C96A8A4242D28169002905DB264936
:10F4F0000968C96AC1F105018161606902EB820294
:10F500009100224A0A44904207D000223AB91E4A8A
:10F510001268D26AE262012038BD0122F6E7251D99
:10F5200028461B4B984768B9E36A03EB83018A00BE
:10F5300016498A5832B901229A4016490B6823EAC3
:10F5400002030B60104B1B68DB6AE362012404FAC0
:10F5500003F21049086802430A6003EB83039A0030
:10F5600029460A4810440C4B9847204638BDC26CC7
:10F57000054B1B68DB6A9A4201D2012038BD00208E
:10F5800038BD0020704700BF040F0020100F00207E
:10F5900051E24000840F002005E24000002834D0F2
:10F5A00038B50446026D013A0265C06AE16C8842D2
:10F5B0002DD00AB1002038BD251D2846154B98478F
:10F5C00068B9E36A03EB83018A0013498A5832B9A8
:10F5D00001229A4011490B6823EA02030B60E36C95
:10F5E000E362C3F10502A261012404FA03F20B49AC
:10F5F000086802430A6003EB83039A002946064821
:10F600001044074B9847204638BD00207047002023
:10F6100038BD00BF51E24000100F0020840F0020D1
:10F6200005E24000002843D038B50446C26C8A4247
:10F6300000D20A46E16A8A4202D0206D012800D039
:10F6400038BDE262A069002802DBC2F10502A261B6
:10F65000636901EB81018800164A0244934225D078
:10F660000022002AECD0251D2846134B984768B984
:10F67000E36A03EB83018A000E498A5832B90122FA
:10F680009A400E490B6823EA02030B60E36A0122E9
:10F690009A400A49086802430A6003EB83039A0010
:10F6A000294604481044064B9847C9E70122D8E789
:10F6B000704700BF100F002051E24000840F00206F
:10F6C00005E24000054B1B6823B1044B1A68136D1B
:10F6D00001331365014B1868704700BF040F002009
:10F6E00038B505460C461A4B98471A4B1B685B6D9C
:10F6F0002BB9184B1B68012283F85820ACB9164B64
:10F700009847134B9847134B1B685C6D24B1CDB9D8
:10F71000104B1B68621E5A650E4B1B68002283F853
:10F7200058200D4B9847204638BD114620460B4BBC
:10F7300098474FF080520A4B1A60BFF34F8FBFF3C8
:10F740006F8FDCE7034B1B6800225A65E4E700BFBC
:10F7500025E34000040F002045E340003DEE40005B
:10F7600004ED00E0F8B507460D4614461E46214B51
:10F770009847214B1B6893F85830DBB2022B0AD014
:10F780001D4B1A68506D20EA070050651B68012266
:10F7900083F85820CEB9194B9847164B98471CB19F
:10F7A000154B1B685B6D2360134B1B6893F8583037
:10F7B000DBB2022B16D000240F4B1B68002283F80B
:10F7C00058200E4B98472046F8BD114630460C4B4A
:10F7D00098474FF080520B4B1A60BFF34F8FBFF327
:10F7E0006F8FD8E7044B1A68536D23EA05055565FA
:10F7F0000124E1E725E34000040F002045E3400039
:10F800003DEE400004ED00E0F8B504460F46154615
:10F810001E46214B98470EB1636D336094F8583003
:10F82000DBB2022284F858206A1E032A1AD8DFE8C5
:10F8300002F0020C1114626D174367650125012B5C
:10F8400014D0164B98472846F8BD626D01326265A8
:10F850000125F4E767650125F1E7022B04D0676510
:10F860000125ECE70125EAE70025E8E7261D3046FB
:10F870000B4B9847E36A01229A400A490868024301
:10F880000A6003EB83039A00314607481044074B94
:10F890009847074B1B68D4E725E3400045E3400049
:10F8A00051E24000840F0020100F002005E24000CC
:10F8B000040F0020F8B5EFF311854FF0500484F3E6
:10F8C0001188BFF36F8FBFF34F8F0BB1446D1C6076
:10F8D00090F85830DBB2022480F85840013A032AED
:10F8E0001AD8DFE802F0020C1114426D1143416591
:10F8F0000126012B14D085F311883046F8BD426DE6
:10F90000013242650126F4E741650126F1E7022B49
:10F9100004D041650126ECE70126EAE70026E8E786
:10F920000446164B1B68F3B9071D3846144B98471D
:10F93000E36A01229A401349086802430A6003EB14
:10F9400083039A00394610481044104B9847E26AE6
:10F950000F4B1B68DB6A9A42CDD9069B4BB1012342
:10F96000069A1360C7E700F118010A48074B984749
:10F97000EDE70122084B1A60BDE700BF7C0F0020B5
:10F9800051E24000840F0020100F002005E24000EB
:10F99000040F0020BC0F0020EC0F0020F8B5EFF39F
:10F9A00011854FF0500383F31188BFF36F8FBFF3BE
:10F9B0004F8F90F85830DBB2022280F85820426D09
:10F9C00001324265012B02D085F31188F8BD0E4645
:10F9D0000446154B1B68E3B9071D3846134B98477F
:10F9E000E36A01229A401249086802430A6003EB65
:10F9F00083039A0039460F4810440F4B9847E26A38
:10FA00000E4B1B68DB6A9A42DED946B10123336094
:10FA1000DAE700F118010A48074B9847EFE701229F
:10FA2000084B1A60D0E700BF7C0F002051E2400075
:10FA3000840F0020100F002005E24000040F00207A
:10FA4000BC0F0020EC0F0020064B1A681368B3FAB5
:10FA500083F35B09036013B9D3681868704700200B
:10FA6000704700BFF00F002008B54160006191426F
:10FA70000CD8D21A83699A4201D3012008BD011D16
:10FA8000094B1868094B9847002008BD9A4201D2DB
:10FA9000994206D2011D064B1868044B9847002076
:10FAA00008BD012008BD00BFF40F00201DE240008A
:10FAB000F00F002070B5104B9847104B1B6813B126
:10FAC0000F4B984770BD0F4D28460F4EB0470F4C57
:10FAD0002046B0470E4B1D600E4B1C6000220C21CF
:10FAE0000A200D4B9847054B18600028E8D00B49B9
:10FAF0000B4B9847E4E700BF25E3400024100020AB
:10FB000045E34000F80F0020E9E140000C10002020
:10FB1000F00F0020F40F0020D9E64000EC4D41002A
:10FB200071EB40002DE9F041079C7CB198461546E9
:10FB30000E460746064B98472760A661E561C4F864
:10FB40002080069B6362201D024B9847BDE8F08130
:10FB5000B5FA4000FFE1400010B582B0094B98476C
:10FB6000094B1B6863B1094B0193032300930023E6
:10FB70004FF42F7206490748074CA04702B010BD4A
:10FB80000020FBE7B5FA40002410002028100020D8
:10FB9000F44D410091FE400001EF40002DE9F0419D
:10FBA00082B005460E46174698462C20084B9847CB
:10FBB000044640B10190089B009343463A463146C3
:10FBC0002846044DA847204602B0BDE8F08100BF9A
:10FBD00079E4400025FB400030B585B0134C256822
:10FBE0000DB31C46019102920390052913DC104BC2
:10FBF0009847022807D000231A4601A90B4800683D
:10FC00000C4CA0470DE00023089A01A907480068A2
:10FC1000084CA04705E00023224601A92846064CCF
:10FC2000A04705B030BD0020FBE700BF2410002036
:10FC3000B5F4400015E740006DE8400070B582B0B3
:10FC4000154B1B681A6802B3DB681E68DC68251D4B
:10FC50002846124B9847636A20469847E369012B70
:10FC6000EED1A36933449E4207D2636024612946E2
:10FC7000094B18680A4B9847E2E7002100910B46B0
:10FC800032462046074CA047DAE7074A1068024987
:10FC90000860136002B070BDF00F002051E2400018
:10FCA0001DE24000D9FB4000F40F002038B50546A6
:10FCB000084B98470446084B1B68984205D300231D
:10FCC0002B60054B1C60204638BD044B9847012330
:10FCD0002B60F6E7FDEF4000201000203DFC4000C7
:10FCE00070B582B005460E460F4B1B68DB68DC68BA
:10FCF000201D0E4B9847E369012B04D0636A204610
:10FD0000984702B070BDA1692B463246294420466F
:10FD1000074EB0470028F1D0002100910B462A463B
:10FD20002046044DA847E9E7F00F002051E24000CB
:10FD300069FA4000D9FB400070B582B006460C4617
:10FD4000174B984701A8174B9847019B23BB0546C3
:10FD50000CB9B04219D22CB1134B1B681C68B4FA11
:10FD600084F464092246711B104B1868104B9847A5
:10FD7000104B984738B94FF080520F4B1A60BFF3C1
:10FD80004F8FBFF36F8F02B070BD0A4B9847294663
:10FD900030460A4B9847F6E7064B9847F3E700BF13
:10FDA000EDEF4000ADFC4000F40F002024100020D7
:10FDB00099EB4000FDF0400004ED00E0E1FC400064
:10FDC00030B587B0002203A92A4B18682A4B984700
:10FDD00000284CD0039B002BF4DB059C636913B116
:10FDE000201D264B984702A8254B9847039B092BBB
:10FDF000E8D801A252F823F021FE400021FE400085
:10FE000021FE4000C5FD400055FE400067FE400059
:10FE100021FE400021FE4000C5FD400055FE40008F
:10FE20000499A5690B46024629442046154DA8476A
:10FE30000028C7D0636A20469847E369012BC1D1E7
:10FE4000A269002100910B460498024420460E4C02
:10FE5000A047B7E70499A161034602460144204642
:10FE6000084CA047AEE72046084B9847AAE707B0E2
:10FE700030BD00BF24100020E5E8400051E2400002
:10FE8000ADFC400069FA4000D9FB40009DE4400011
:10FE900000B583B001A8044B98470199034B9847DC
:10FEA000034B9847F6E700BF49FA400039FD400090
:10FEB000C1FD4000064BDB6BC3F30023054A137002
:10FEC000054BDB6BC3F34033044A1370704700BF2C
:10FED00000100E402C100020000E0E402D100020AF
:10FEE00008B5054BDB6B13F4004F02D1034B984769
:10FEF00008BD034B984708BD000E0E40BD5440009E
:10FF0000E154400030B583B004460D460023019310
:10FF10002E4B984213D02E4B9C421AD02D4B9C4214
:10FF200021D02D4B9C4228D02C4B9C422FD02C4BC7
:10FF30009C4236D02B4B9C423DD003B030BD01A932
:10FF40002046294B98470028F9D19DF804302B70A2
:10FF5000E1E701A92046244B98470028F9D19DF8F4
:10FF600004302B70DAE701A920461F4B9847002880
:10FF7000F9D19DF804302B70D3E701A920461A4B24
:10FF800098470028F9D19DF804302B70CCE701A9DF
:10FF90002046154B98470028F9D19DF804302B7066
:10FFA000C5E701A92046104B98470028F9D19DF8D4
:10FFB00004302B70BEE701A920460B4B9847002860
:10FFC000F9D19DF804302B70B7E700BF00C20040A4
:10FFD00000020240004202400082014000C2014093
:10FFE000008200400002044091DE400038B5044623
:10FFF0000D46274B984213D0264B984218D0264BDB
:020000040041B9
:1000000098421DD0254B984222D0254B984227D0AC
:10001000244B98422CD0244B984231D0002038BD3C
:1000200029462046214B98470028F9D1012038BDA8
:10003000294620461D4B98470028F9D1012038BD9C
:1000400029462046194B98470028F9D1012038BD90
:1000500029462046154B98470028F9D1012038BD84
:1000600029462046114B98470028F9D1012038BD78
:10007000294620460D4B98470028F9D1012038BD6C
:1000800029462046094B98470028F9D1012038BD60
:1000900000C20040000202400042024000820140D3
:1000A00000C20140008200400002044069DE4000BE
:1000B00000B583B002A9002341F8043D084B18683D
:1000C000084B9847019B3BB14FF08052064B1A609A
:1000D000BFF34F8FBFF36F8F03B05DF804FB00BF1A
:1000E000341000209DF9400004ED00E070B58AB0A6
:1000F0001D4B0FCB0AAC04E90F001C4D1C4B1D60BF
:100100001C4A1D4B1A601D4A1D4B1A60069B00932A
:10011000079B0193089B0293099B0393002404947B
:10012000184E3046184B984701213046174B9847D8
:10013000174A69462846174B98472846164B984752
:100140002846164B9847164E336821469868154D39
:10015000A847336821465868A847336821469868FD
:10016000A8470AB070BD00BFFC4D410000820140AD
:1001700038230020EDFF40003423002005FF40001D
:10018000302300200080014051DA4000B9DB4000FC
:100190000000DC05F5DE400041DE40004DDE4000A1
:1001A0003C030020E91C410008B504460D460A4600
:1001B00001460748074B98470220074B98472946B6
:1001C0002046064B9847EFF30580054B9847FFDE26
:1001D000C04E410055134100854D4000714D400017
:1001E000914D400070B51F4B98471F4B1B68C31AB9
:1001F000632B00D870BD1C4B18601C4B18681C4D3D
:10020000A8471C4C20601C481C4EB047A8476060A3
:100210001B48B047A847A0601A48B047A847E0600D
:100220001948B047A84720611848B047A8476061FF
:100230001748B047A847A0611648B047A847E061F3
:100240001548B047A84720621448B047A8476062E5
:100250001348B047A847A0621248B047A847E062D9
:10026000C8E700BFFDEF4000301000203410002030
:1002700099F44000B4230020B44E410015F2400030
:10028000804741001C4D41003C4D4100704D4100F4
:10029000904D4100B04D4100D04C41001847410005
:1002A000E44D4100F44D4100704700002DE9F0435A
:1002B00083B04B4B98474B4A936843F0254343F434
:1002C00080139360484B9847484B9847484B984752
:1002D000484B9847484B9847484B98470446484BEB
:1002E0009847F02201462046464B9847464B984790
:1002F0004648474B03602223037123234371454D36
:100300002946454CA0474548454B03602B230371C4
:100310002A2343712946A047424B9847424B9847AE
:100320004248434B98474348434CA04743494448BD
:10033000A04744494448A047444A45494548A04746
:1003400000230193042200924FF4807242494348F3
:10035000434CA047012802D04248374B98473E48BB
:10036000414B9847414B1860414B9847414B984748
:10037000414B9847414B9847414A00210F20414E3D
:10038000B047414C03220B212046404DA847DFF8DF
:1003900010914A4600212820B0473D4F03220C21EE
:1003A0003846A8472820DFF8FC80C0470146384679
:1003B000384FB8474A4600210D20B04703220B2191
:1003C0002046A8470D20C04701462046B847324B7B
:1003D0009847324B9847002003B0BDE8F08300BF38
:1003E0006945400010140E40D1D84000897A400081
:1003F000C56E4000ED004100957640004D7840000C
:10040000557840000D77400029774000A023002058
:1004100000000240A0860100597340008C23002098
:1004200000C001406DB740008D6D4000B10041003B
:100430005D4540000C4E410055134100244E4100E3
:10044000384E410050444100444E4100584E410056
:10045000644E4100704E4100884E4100617840007A
:1004600001EF4000904E410015F240003410002092
:10047000D997400051AE4000CDA04000FD8F400014
:10048000E1FE4000D1BA4000000E0E4041BB4000EA
:1004900000100E404FD840001F50400075EF400044
:1004A000B5FE400073D8400030B583B000248DF80D
:1004B00004408DF805408DF806400F4B98470F4BD0
:1004C000984720460E4B98470E4D01A928460E4BE3
:1004D000984772B60D480E4CA0472846A0470D4BD2
:1004E00098470D4B98470D4B98470D4A136823F0DA
:1004F0000103136003B030BD557A4000EDEF4000BA
:10050000055440008C23002095634000A023002068
:10051000F1734000A9534000B9B74000A9774000EB
:1005200010E000E000487047A0230020004870471A
:100530008C23002008B5014B984708BD5D7840002A
:1005400008B5014B984708BD5F784000704701200F
:100550007047000008B50248024B984708BD00BF2D
:10056000A02300209174400008B50248024B984730
:1005700008BD00BF8C23002091744000014B187807
:10058000704700BF2D100020014B1878704700BF46
:100590002C10002070B58AB0044600F06FF8324B82
:1005A00093F900506B1C064609D02146204600F006
:1005B0008DFE20B90021204600F07EFE10B13046AD
:1005C0000AB070BD294B08902046019300F006FB4D
:1005D000CDE90401CDE902012046CDB9244B4FF00D
:1005E00060420021CDE9062300F03EFE002833D012
:1005F00002230093684600F085F9A8B1089BC3B9AF
:10060000DDE9060100F03EFB064630460AB070BD4B
:10061000184B00220021CDE9062300F025FE68B129
:1006200002239D420093E5D100F066FE2223036081
:10063000E4E700F061FE089B0360E1E70123022D7F
:1006400000930BD100F058FE212303600A4800F00C
:100650005BF9CDE90601D1E701230093684600F07C
:1006600051F90028F2D1EDE738030020D84E4100BF
:10067000FFFFEFC70000F0FFE04D41002DE9F84F0C
:1006800030F000432DD00028014604464ADBB0F18B
:10069000FF4F3BDAB0F5000F3CDB00268D4AC4F378
:1006A00016052A4402F40002E41582F07E507F3CD5
:1006B00034444FF07E51284304EBD25400F036FB13
:1006C00005F10F03C3F316030F2B064631DC00219F
:1006D00000F0CAFD002800F094804CB90020BDE86D
:1006E000F88F00214FF04C4000F0DEFCBDE8F88FA1
:1006F000204600F0D1FB7849054600F021FC7749FF
:100700000446284600F01CFC0146204600F010FB81
:10071000BDE8F88F4FF0984100F012FC6FF018061A
:100720000446BBE700F002FB002100F0BDFCBDE881
:10073000F88F4FF0804100F0FBFA0146304600F0A0
:10074000B3FC8046204600F0A7FB41468146404668
:1007500000F0F6FB0146834600F0F2FB6049DFF84B
:10076000A0A1074600F0ECFB5E4900F0E1FA394633
:1007700000F0E6FB5C4900F0DBFA394600F0E0FBF4
:100780005A4900F0D5FA594600F0DAFB5849834639
:10079000384600F0D5FB574900F0CAFA394600F058
:1007A000CFFB554900F0C4FA394600F0C9FB0146B9
:1007B000584600F0BDFAC5F55713AA4403F5227355
:1007C00043EA0A03002B074665DD4FF07C513046B3
:1007D00000F0B6FB314600F0B3FB0546002C32D1E9
:1007E0002946384600F0A4FA414600F0A9FB01462C
:1007F000284600F09BFA0146304600F097FABDE823
:10080000F88F3E49304600F09BFB01464FF07C508C
:1008100000F08CFA31460546304600F091FB014667
:10082000284600F08DFB0546002C2ED0204600F017
:1008300033FB2949074600F083FB28490446384624
:1008400000F07EFB14E02449484600F079FB29467D
:100850000446384600F06CFA414600F071FB1F492F
:100860000746484600F06CFB0146384600F060FA47
:100870000146284600F05AFA314600F057FA014680
:10088000204600F053FABDE8F88F0146304600F0EC
:100890004DFABDE8F88F7CB10F49484600F050FB97
:1008A00039460446304600F041FA414600F048FB24
:1008B0000A4905464846C3E70146304600F036FA85
:1008C000414600F03DFB0146304600F02FFABDE8FE
:1008D000F88F00BF20FB4A008071313FD1F71737F6
:1008E0009788173E25333A3E2549923EABAA2A3FC8
:1008F0004FD01C3E298E633ECDCCCC3EABAAAA3E47
:10090000305CCFFF0020704700200149704700BFD6
:100910000000F87F81F0004102E000BF83F0004357
:1009200030B54FEA41044FEA430594EA050F08BF8A
:1009300090EA020F1FBF54EA000C55EA020C7FEA4E
:10094000645C7FEA655C00F0E2804FEA5454D4EBCB
:100950005555B8BF6D420CDD2C4480EA020281EA95
:10096000030382EA000083EA010180EA020281EACD
:100970000303362D88BF30BD11F0004F4FEA01311F
:100980004FF4801C4CEA113102D0404261EB41012E
:1009900013F0004F4FEA03334CEA133302D05242B4
:1009A00063EB430394EA050F00F0A780A4F1010470
:1009B000D5F1200E0DDB02FA0EFC22FA05F28018AA
:1009C00041F1000103FA0EF2801843FA05F3594190
:1009D0000EE0A5F120050EF1200E012A03FA0EFC0F
:1009E00028BF4CF0020C43FA05F3C01851EBE37139
:1009F00001F0004507D54FF0000EDCF1000C7EEB56
:100A000000006EEB0101B1F5801F1BD3B1F5001F93
:100A10000CD349085FEA30004FEA3C0C04F10104B2
:100A20004FEA445212F5800F80F09A80BCF1004FDB
:100A300008BF5FEA500C50F1000041EB045141EA5D
:100A4000050130BD5FEA4C0C404141EB010111F45E
:100A5000801FA4F10104E9D191F0000F04BF014609
:100A60000020B1FA81F308BF2033A3F10B03B3F1E7
:100A700020020CDA0C3208DD02F1140CC2F10C0277
:100A800001FA0CF021FA02F10CE002F11402D8BFD5
:100A9000C2F1200C01FA02F120FA0CFCDCBF41EAA1
:100AA0000C019040E41AA2BF01EB0451294330BD70
:100AB0006FEA04041F3C1CDA0C340EDC04F114044D
:100AC000C4F1200220FA04F001FA02F340EA030024
:100AD00021FA04F345EA030130BDC4F10C04C4F16A
:100AE000200220FA02F001FA04F340EA030029464A
:100AF00030BD21FA04F0294630BD94F0000F83F494
:100B0000801306BF81F480110134013D4EE77FEA76
:100B1000645C18BF7FEA655C29D094EA050F08BFC2
:100B200090EA020F05D054EA000C04BF19461046A3
:100B300030BD91EA030F1EBF0021002030BD5FEAE7
:100B4000545C05D14000494128BF41F0004130BD0F
:100B500014F580043CBF01F5801130BD01F0004563
:100B600045F0FE4141F470014FF0000030BD7FEAD6
:100B7000645C1ABF194610467FEA655C1CBF0B46D1
:100B8000024650EA013406BF52EA033591EA030FE8
:100B900041F4002130BD00BF90F0000F04BF0021E0
:100BA000704730B54FF4806404F132044FF0000513
:100BB0004FF0000150E700BF90F0000F04BF00218C
:100BC000704730B54FF4806404F1320410F00045F2
:100BD00048BF40424FF000013EE700BF42004FEAED
:100BE000E2014FEA31014FEA02701FBF12F07F436A
:100BF00093F07F4F81F06051704792F0000F14BF67
:100C000093F07F4F704730B54FF4607401F00045AA
:100C100021F0004120E700BF50EA010208BF704701
:100C200030B54FF000050AE050EA010208BF7047F6
:100C300030B511F0004502D5404261EB41014FF45F
:100C4000806404F132045FEA915C3FF4DCAE4FF063
:100C500003025FEADC0C18BF03325FEADC0C18BF4A
:100C6000033202EBDC02C2F1200300FA03FC20FA9B
:100C700002F001FA03FE40EA0E0021FA02F11444E8
:100C8000C1E600BF4FEA4102B2F1E04324BFB3F531
:100C9000001CDCF1FE5C0DD901F0004C4FEAC002F3
:100CA0004CEA5070B2F1004F40EB830008BF20F0D7
:100CB0000100704711F0804F21D113F13872BCBF91
:100CC00001F00040704741F480114FEA5252C2F1E6
:100CD0001802C2F1200C10FA0CF320FA02F018BF2F
:100CE00040F001004FEAC1234FEAD32303FA0CFC82
:100CF00040EA0C0023FA02F34FEA4303CCE77FEA11
:100D0000625307D150EA01331EBF4FF0FE4040F45A
:100D10004000704701F0004040F0FE4040F4000009
:100D2000704700BF80F0004002E000BF81F000414A
:100D300042001FBF5FEA410392EA030F7FEA226C81
:100D40007FEA236C6AD04FEA1262D2EB1363C1BF11
:100D5000D218414048404140B8BF5B42192B88BF80
:100D6000704710F0004F40F4000020F07F4018BFA3
:100D7000404211F0004F41F4000121F07F4118BFC3
:100D8000494292EA030F3FD0A2F1010241FA03FC6B
:100D900010EB0C00C3F1200301FA03F100F0004353
:100DA00002D5494260EB4000B0F5000F13D3B0F11B
:100DB000807F06D340084FEA310102F10102FE2A8A
:100DC00051D2B1F1004F40EBC25008BF20F00100FA
:100DD00040EA03007047490040EB000010F4000FA8
:100DE000A2F10102EDD1B0FA80FCACF1080CB2EB3B
:100DF0000C0200FA0CF0AABF00EBC250524218439A
:100E0000BCBFD0401843704792F0000F81F400013E
:100E100006BF80F400000132013BB5E74FEA410311
:100E20007FEA226C18BF7FEA236C21D092EA030F7D
:100E300004D092F0000F08BF0846704790EA010FF7
:100E40001CBF0020704712F07F4F04D1400028BF24
:100E500040F00040704712F100723CBF00F5000006
:100E6000704700F0004343F0FE4040F4000070473C
:100E70007FEA226216BF08467FEA236301464202E8
:100E800006BF5FEA412390EA010F40F480007047FB
:100E90004FF0000304E000BF10F0004348BF4042A1
:100EA0005FEA000C08BF704743F0964301464FF0DD
:100EB00000001CE050EA010208BF70474FF0000339
:100EC0000AE000BF50EA010208BF704711F000437A
:100ED00002D5404261EB41015FEA010C02BF84464A
:100EE0000146002043F0B64308BFA3F18053A3F5A9
:100EF0000003BCFA8CF2083AA3EBC25310DB01FAF0
:100F000002FC634400FA02FCC2F12002BCF1004F73
:100F100020FA02F243EB020008BF20F00100704704
:100F200002F1200201FA02FCC2F1200250EA4C0058
:100F300021FA02F243EB020008BF20EADC7070479E
:100F40004FF0FF0C1CEAD0521EBF1CEAD15392EAAC
:100F50000C0F93EA0C0F6FD01A4480EA010C400288
:100F600018BF5FEA41211ED04FF0006343EA5010E2
:100F700043EA5111A0FB01310CF00040B1F5000F24
:100F80003EBF490041EAD3715B0040EA010062F1D3
:100F90007F02FD2A1DD8B3F1004F40EBC25008BFBD
:100FA00020F00100704790F0000F0CF0004C08BFDB
:100FB00049024CEA502040EA51207F3AC2BFD2F1A8
:100FC000FF0340EAC250704740F400004FF00003B6
:100FD000013A5DDC12F1190FDCBF00F000407047F0
:100FE000C2F10002410021FA02F1C2F1200200FA2E
:100FF00002FC5FEA310040F1000053EA4C0308BFF5
:1010000020EADC70704792F0000F00F0004C02BF45
:10101000400010F4000F013AF9D040EA0C0093F0C0
:10102000000F01F0004C02BF490011F4000F013B1A
:10103000F9D041EA0C018FE70CEAD15392EA0C0F88
:1010400018BF93EA0C0F0AD030F0004C18BF31F0F3
:10105000004CD8D180EA010000F00040704790F0C9
:10106000000F17BF90F0004F084691F0000F91F06D
:10107000004F14D092EA0C0F01D142020FD193EA33
:101080000C0F03D14B0218BF084608D180EA0100BB
:1010900000F0004040F0FE4040F40000704740F097
:1010A000FE4040F4400070474FF0FF0C1CEAD05265
:1010B0001EBF1CEAD15392EA0C0F93EA0C0F69D0C1
:1010C000A2EB030280EA010C49024FEA402037D02C
:1010D0004FF0805343EA111143EA10130CF0004023
:1010E0008B4238BF5B0042F17D024FF4000C8B4213
:1010F00024BF5B1A40EA0C00B3EB510F24BFA3EBF3
:10110000510340EA5C00B3EB910F24BFA3EB9103C2
:1011100040EA9C00B3EBD10F24BFA3EBD10340EA1C
:10112000DC001B0118BF5FEA1C1CE0D1FD2A3FF662
:1011300050AF8B4240EBC25008BF20F00100704717
:101140000CF0004C4CEA50207F32C2BFD2F1FF03BA
:1011500040EAC250704740F400004FF00003013AEB
:1011600037E792F0000F00F0004C02BF400010F48F
:10117000000F013AF9D040EA0C0093F0000F01F0A3
:10118000004C02BF490011F4000F013BF9D041EAC5
:101190000C0195E70CEAD15392EA0C0F08D14202F8
:1011A0007FF47DAF93EA0C0F7FF470AF084676E7CB
:1011B00093EA0C0F04D14B023FF44CAF08466EE7A4
:1011C00030F0004C18BF31F0004CCAD130F0004272
:1011D0007FF45CAF31F000437FF43CAF5FE700BFCA
:1011E0004FF0FF3C06E000BF4FF0010C02E000BFF3
:1011F0004FF0010C4DF804CD4FEA40024FEA410395
:101200007FEA226C18BF7FEA236C11D001B052EA4A
:10121000530C18BF90EA010F58BFB2EB030088BF10
:10122000C81738BF6FEAE17018BF40F0010070477F
:101230007FEA226C02D15FEA402C05D17FEA236C61
:10124000E4D15FEA412CE1D05DF8040B704700BFA8
:10125000844608466146FFE70FB5FFF7C9FF00283F
:1012600048BF10F1000F0FBD4DF808EDFFF7F4FF78
:101270000CBF012000205DF808FB00BF4DF808ED11
:10128000FFF7EAFF34BF012000205DF808FB00BF34
:101290004DF808EDFFF7E0FF94BF012000205DF856
:1012A00008FB00BF4DF808EDFFF7D2FF94BF012007
:1012B00000205DF808FB00BF4DF808EDFFF7C8FF00
:1012C00034BF012000205DF808FB00BF4FEA400258
:1012D0004FEA41037FEA226C02D15FEA402C08D139
:1012E0007FEA236C02D15FEA412C02D14FF000006B
:1012F00070474FF001007047014B1868704700BFFE
:101300003C03002070B50F4E0F4D761BB61018BF72
:10131000002405D0013455F8043B9847A642F9D182
:101320000A4E0B4D761B03F08FFEB61018BF00243B
:1013300006D0013455F8043B9847A642F9D170BD58
:1013400070BD00BF54504100545041005C504100FA
:10135000545041000FB400B5074983B004AB08688E
:1013600053F8042B8168019300F076FE03B05DF81A
:1013700004EB04B0704700BF3C030020024B014661
:10138000186800F00BB800BF3C030020024B014678
:10139000186801F07DBF00BF3C0300202DE9F04F2D
:1013A00001F10B06162E83B0054640F29E8036F002
:1013B000070600F1BD80B14200F2BA8000F06CFC7B
:1013C000B6F5FC7FC0F09382730A00F0B880042B5E
:1013D00000F27981B30903F1390003F1380EC3003B
:1013E000BF4F3B44A3F108015C68A14206D10CE069
:1013F000002A80F2AA80E468A14206D0636823F044
:1014000003039A1B0F2AF3DD70463C69DFF8E4E220
:10141000744500F0AB81636823F003039A1B0F2A25
:1014200000F39081002AC7F814E0C7F810E080F2BA
:101430009D80B3F5007F80F06181DB0803F1010C32
:1014400099107A6857F83C80C4F8088001238B40D3
:1014500007EBCC0113430839E1607B6047F83C405F
:10146000C8F80C408210012494409C4200F28B800A
:101470001C4206D120F0030064001C4200F104006D
:10148000FAD007EBC009CC468046DCF80C309C450E
:1014900007D16DE1002A80F27B81DB689C4500F07A
:1014A0006781596821F003018A1B0F2AF2DDD3F806
:1014B0000CC0D3F8088000939C19284646F001061A
:1014C00042F001055E60C8F80CC0CCF808807C6171
:1014D0003C61C4F80CE0C4F808E065605A5000F0C4
:1014E000E1FB009B03F108041EE0102920D800F066
:1014F000D3FB102618230220794F3B44A3F10802A6
:101500005C68944200F03D816368E168A66823F05E
:101510000303234428465A68F16042F001028E60BA
:101520005A6000F0BFFB0834204603B0BDE8F08FDE
:1015300000240C2320462B6003B0BDE8F08F402030
:101540004FF400734FF03F0E4AE72344E1685A68B6
:10155000A66842F00102F16028468E605A6000F0F1
:10156000A1FB0834204603B0BDE8F08F2344284691
:101570005A6842F001025A6000F094FB0834204699
:1015800003B0BDE8F08FBC68636823F00308B04582
:1015900004D3A8EB06030F2B00F38580DFF85891E6
:1015A000504BD9F800201B680132334404EB080A81
:1015B00000F0558103F580530F3323F47F6B2BF03C
:1015C0000F0B5946284600F07DFB411C024600F0F7
:1015D000FC80824500F2F780434B1968594419603A
:1015E00000F04D81D9F8000001301BBFA2EB0A0AC0
:1015F0005144C9F80020196012F0070100F015816C
:10160000C1F10800C1F580510244083102EB0B0919
:10161000C9F30B09A1EB0909494628460193009239
:1016200000F050FB431C9DE80C0000F04381801A41
:10163000484440F001001968BA604944BC42506017
:10164000196017D0B8F10F0F40F2FB806068A8F165
:101650000C0222F0070204EB020E00F001004FF032
:10166000050C10430F2A6060CEF804C0CEF808C005
:1016700000F217811D4BBC681A68914288BF19603F
:101680001B4B1A689142626888BF196022F00302FE
:101690009642A2EB060301D80F2B04DC284600F08B
:1016A00001FB002440E7A21943F0010346F00106C4
:1016B00066602846BA60536000F0F4FA08342046A9
:1016C00003B0BDE8F08F142B71D9542B00F2A38026
:1016D000330B03F16F0003F16E0EC30080E600BF11
:1016E00068070020681000203810002060100020DB
:1016F0006410002070070020700B00205A0A042A92
:101700005BD9142A00F2AE8002F15C01C9005B32A1
:1017100007EB010C7958ACF1080C8C4500F088807F
:101720004A6822F00302934273D289688C45F7D14C
:10173000DCF80C207B68E260C4F808C09460CCF848
:101740000C408FE6A11946F0010C42F00106C4F8E6
:1017500004C0284679613961C1F80CE0C1F808E09D
:101760004E60E25000F09EFA0834DDE67B6879E6D0
:1017700008F1010818F0030F0CF1080C7FF485AE96
:101780002DE0DC68A34208BF02303FF43EAEBBE66A
:1017900019441C464A68DB6854F8086F42F001029D
:1017A0004A602846F3609E6000F07CFABCE603F1D4
:1017B0005C0003F15B0EC30012E69A0902F13901E5
:1017C000C9003832A4E7BC4254D0BC68626822F039
:1017D00003025DE759F80839994540F0868010F01A
:1017E000030F00F1FF30F5D17B6823EA04037B602F
:1017F00064009C423FF6C7AE002C3FF4C4AE1C42CE
:1018000040467FF43EAE64001C4200F10400FAD072
:1018100037E68C468CE7B3F5AA7F15D8F30B03F1B6
:10182000780003F1770EC300DAE54FF48051EDE65E
:101830007B689210012101FA02F213437B60624639
:1018400079E70123536029E740F25452934222D8AA
:10185000B30C03F17D0003F17C0EC300C0E503F17E
:10186000100BAEE6542A29D81A0B02F16F01C900F9
:101870006E324DE7204B196859441960B2E6CAF33D
:101880000B0000287FF4AEAE08EB0B03BA6843F000
:1018900001035360EEE67F204FF47E734FF07E0E1F
:1018A0009EE504F108012846009301F0F1FC009B3D
:1018B0001968DFE601204FF00009BCE6B2F5AA7F07
:1018C00005D8DA0B02F17801C900773220E740F23F
:1018D00054518A4205D89A0C02F17D01C9007C322C
:1018E00016E74FF47E717E2212E77B6880E7F008EE
:1018F00006F1080300E600BF3810002000000000D9
:1019000001F0FF01102A2BDB10F0070F08D010F8B0
:10191000013B013A8B422DD010F0070F42B3F6D1B4
:10192000F0B441EA012141EA014122F007047FF0CD
:1019300000070023F0E80256083C85EA010586EA24
:10194000010685FA47F5A3FA87F586FA47F6A5FA60
:1019500087F68EB9EED1F0BC01F0FF0102F007026C
:1019600032B110F8013B013A83EA010313B1F8D117
:101970000020704701387047002D06BF35460338F8
:10198000073815F0010F07D1013015F4807F02BF31
:10199000013015F4C03F0130F0BC0138704700BF82
:1019A000032A70B422D940EA01039B0711D00378BF
:1019B0000C78A3421DD10A44013105E010F8013F23
:1019C00011F8014BA34214D19142F7D1002070BC11
:1019D00070470D680668AE420C46034601F10401EB
:1019E00000F1040008D1043A032AF2D8002ADED11B
:1019F000ECE7181B70BC704721461846D7E700BFBC
:101A0000844641EA000313F003036DD1403A41D309
:101A100051F8043B40F8043B51F8043B40F8043BC8
:101A200051F8043B40F8043B51F8043B40F8043BB8
:101A300051F8043B40F8043B51F8043B40F8043BA8
:101A400051F8043B40F8043B51F8043B40F8043B98
:101A500051F8043B40F8043B51F8043B40F8043B88
:101A600051F8043B40F8043B51F8043B40F8043B78
:101A700051F8043B40F8043B51F8043B40F8043B68
:101A800051F8043B40F8043B51F8043B40F8043B58
:101A9000403ABDD2303211D351F8043B40F8043BF8
:101AA00051F8043B40F8043B51F8043B40F8043B38
:101AB00051F8043B40F8043B103AEDD20C3205D308
:101AC00051F8043B40F8043B043AF9D2043208D000
:101AD000D2071CBF11F8013B00F8013B01D30B8872
:101AE00003806046704700BF082A13D38B078DD050
:101AF00010F003038AD0C3F10403D21ADB071CBF22
:101B000011F8013B00F8013B80D331F8023B20F88B
:101B1000023B7BE7043AD9D3013A11F8013B00F8C4
:101B2000013BF9D20B7803704B7843708B7883704C
:101B3000604670478842F0B50DD98B1898420AD29A
:101B40008418002A51D0224613F8014D02F8014DA5
:101B50009942F9D1F0BD0F2A48D941EA00039B0709
:101B600046D100F1100401F11003154653F8106C32
:101B700044F8106C53F80C6C44F80C6C53F8086C77
:101B800044F8086C103D53F8046C44F8046C0F2DB5
:101B900003F1100304F11004E8D8A2F1100323F0BC
:101BA0000F0302F00F0E1033BEF1030F194403446C
:101BB00021D91E1F0D467446043C55F8047B46F897
:101BC000047F032CF8D8AEF1040424F00304043499
:101BD0002144234402F0030262B1013B0A4411F89C
:101BE000014B03F8014F8A42F9D1F0BD0346F3E7F8
:101BF0000346F2E7F0BD7246EEE700BF70B4860719
:101C000046D0541E002A41D0CAB2034602E014F165
:101C1000FF343BD303F8012B9D07F8D1032C2ED9B9
:101C2000CDB245EA05250F2C45EA054519D903F142
:101C300010022646103E0F2E42F8105C42F80C5C53
:101C400042F8085C42F8045C02F11002F2D8A4F1F8
:101C5000100222F00F0204F00F041032032C134480
:101C60000DD91E462246043A032A46F8045BFAD8E8
:101C7000221F22F003020432134404F003042CB1A7
:101C8000C9B21C4403F8011B9C42FBD170BC7047D5
:101C900014460346C2E700BF014801F093BD00BFF0
:101CA00004240020014801F08FBD00BF042400205F
:101CB00010B5034B0446196801F02AFE204610BDFA
:101CC0003C03002038B5074C002305460846236036
:101CD000FCF762FA431C00D038BD2368002BFBD010
:101CE0002B6038BD1824002000290CBF02220022DE
:101CF0004FF4806300F000B82DE9F043614C256893
:101D000083B004460F4690461E4615B1AB6B002BC0
:101D100064D0B8F1020F06D0B8F1010F00F29F8035
:101D2000002EC0F29C80636ED80734D52146284629
:101D300001F030F9216B41B104F14003994202D026
:101D4000284601F0A5FA00232363B4F90C300022E1
:101D5000A26162601A063AD423F44A6323F00303B3
:101D6000B8F1020FA3811DD001AB6A462146284677
:101D700001F02CFDA3891843A081002E32D1009ED2
:101D80003046FFF7FBFA074600286BD0A38943F0E3
:101D90008003A38128E0A3899905C7D4A06D01F031
:101DA00011FDC3E70025616E002604F1430243F0F4
:101DB00002030120A660CE07A38122602261606138
:101DC00001D498053ED5284603B0BDE8F0832169CB
:101DD000284601F05DFAB4F90C30BDE7284601F061
:101DE00031F996E7002FCBD0AB6B002B33D0009BA3
:101DF000B4F90C2027609E421CBF42F40062A2810D
:101E0000B8F1010F04BF42F00102A28192B212F0B8
:101E10000803276166610ED0D1071AD5656E764238
:101E2000002315F00105A661A36009D0002528460E
:101E300003B0BDE8F083A360656E15F00105F5D130
:101E40009305C0D4A06D01F0BFFC284603B0BDE8E7
:101E5000F083A660F0E7284601F0F4F8C7E74FF0FA
:101E6000FF35B0E7DDF80090B14504D04846FFF7F4
:101E700085FA074620B9B4F90C304FF0FF3592E7E8
:101E80004E4683E73C0300200000000000000000F5
:101E90000000000000000000000000000000000042
:101EA0000000000000000000000000000000000032
:101EB0000000000000000000000000000000000022
:101EC00090F800F06DE9024520F007016FF0000C7A
:101ED00010F0070491F820F040F049804FF0000422
:101EE0006FF00700D1E9002391F840F000F10800FD
:101EF00082FA4CF2A4FA8CF283FA4CF3A2FA8CF335
:101F00004BBBD1E9022382FA4CF200F10800A4FA9B
:101F10008CF283FA4CF3A2FA8CF3E3B9D1E90423EF
:101F200082FA4CF200F10800A4FA8CF283FA4CF326
:101F3000A2FA8CF37BB9D1E9062301F1200182FAE0
:101F40004CF200F10800A4FA8CF283FA4CF3A2FAE6
:101F50008CF3002BC6D0002A04BF04301A4612BAF4
:101F6000B2FA82F2FDE8024500EBD2007047D1E9F7
:101F7000002304F00305C4F100004FEAC50514F086
:101F8000040F91F840F00CFA05F562EA05021CBF57
:101F900063EA050362464FF00004A9E7B1B1037894
:101FA000B3B10144431C994214D010B41A785C1C9C
:101FB00032B1A142234606D01A785C1C002AF8D11F
:101FC000181A10BC7047081A10BC704708467047B2
:101FD00018467047081A70472DE9F84F4B6E9C045D
:101FE00093462FD59368126853B30E46074602F105
:101FF000080919E920045FEA9A0817D0043D002473
:1020000001E0A04510D0324655F8041F384601F0D3
:10201000BBF8431C04F10104F3D10023CBF80830D2
:10202000CBF80430BDE8F88FDBF808302AF0030A5B
:10203000A3EB0A03CBF8083009F10809002BD8D12B
:102040000020EAE701F00AFA0023CBF80830CBF8C9
:102050000430BDE8F88F00BF2DE9F04FADB01D464C
:102060008B4690460793069018B1836B002B00F0C7
:10207000F380DBF86430BBF90C00DF0781B202D4D7
:102080008E0540F1FC808C040AD4DBF8643040F407
:10209000005123F40053ABF80C10CBF8643089B234
:1020A000080740F1B380DBF81030002B00F0AE8061
:1020B00001F01A030A2B00F0B58000230DF170091E
:1020C0000B93119310930393CDF83C90CA46CDF82F
:1020D00010B098F800304446FBB1252B02D11CE02B
:1020E000252B03D014F8013F002BF9D1A4EB0805F0
:1020F0009DB1109B119ACAF8008001332A44072B26
:10210000CAF80450119210937ADD002A40F0B0848E
:10211000039B10922B44CA4603932378002B00F0B4
:10212000E08300204FF000038DF8373004F1010800
:1021300062780546064603464FF0FF3408F1010871
:10214000A2F12001582900F2DE82DFE811F021021D
:10215000DC02DC022902DC02DC02DC02DC02DC0242
